 Project1

 Timestamp is 4f0eeee6 (Thu Jan 12 20:32:06 2012)

 Preferred load address is 00400000

 Start         Length     Name                   Class
 0001:00000000 00023fc9H .textbss                DATA
 0002:00000000 0004abe4H .text                   CODE
 0002:0004abf0 0000112fH .text$x                 CODE
 0003:00000000 00000104H .CRT$XCA                DATA
 0003:00000104 00000104H .CRT$XCZ                DATA
 0003:00000208 00000104H .CRT$XIA                DATA
 0003:0000030c 00000113H .CRT$XIC                DATA
 0003:00000420 00000104H .CRT$XIY                DATA
 0003:00000524 00000104H .CRT$XIZ                DATA
 0003:00000628 00000104H .CRT$XPA                DATA
 0003:0000072c 00000109H .CRT$XPX                DATA
 0003:00000838 00000104H .CRT$XPXA               DATA
 0003:0000093c 00000104H .CRT$XPZ                DATA
 0003:00000a40 00000104H .CRT$XTA                DATA
 0003:00000b44 00000104H .CRT$XTZ                DATA
 0003:00000c50 0000cb1aH .rdata                  DATA
 0003:0000d76c 00000166H .rdata$debug            DATA
 0003:0000d8d4 0000032fH .rdata$r                DATA
 0003:0000dc04 00000104H .rtc$IAA                DATA
 0003:0000dd08 00000104H .rtc$IMZ                DATA
 0003:0000de0c 00000104H .rtc$IZZ                DATA
 0003:0000df10 00000104H .rtc$TAA                DATA
 0003:0000e014 00000104H .rtc$TMZ                DATA
 0003:0000e118 00000104H .rtc$TZZ                DATA
 0003:0000e220 00000d5aH .xdata$x                DATA
 0003:0000ef7a 00000000H .edata                  DATA
 0004:00000000 000012f8H .data                   DATA
 0004:00001300 00002598H .bss                    DATA
 0005:00000000 0000003cH .idata$2                DATA
 0005:0000003c 00000014H .idata$3                DATA
 0005:00000050 00000238H .idata$4                DATA
 0005:00000288 00000238H .idata$5                DATA
 0005:000004c0 00000875H .idata$6                DATA
 0006:00000000 000001c0H .rsrc$01                DATA
 0006:000001c0 00000400H .rsrc$02                DATA

  Address         Publics by Value              Rva+Base       Lib:Object

 0000:00000000       ___safe_se_handler_table   00000000     <absolute>
 0000:00000000       ___safe_se_handler_count   00000000     <absolute>
 0000:00000000       __except_list              00000000     <absolute>
 0000:00000000       ___ImageBase               00400000     <linker-defined>
 0001:00000000       __enc$textbss$begin        00401000     <linker-defined>
 0001:00023fc9       __enc$textbss$end          00424fc9     <linker-defined>
 0002:00002270       _WinMain@16                00427270 f   Project1.obj
 0002:000022e0       ?MainHandler@@YGJPAUHWND__@@IIJ@Z 004272e0 f   Project1.obj
 0002:00002546       _GetModuleHandleA@4        00427546 f   kernel32:KERNEL32.dll
 0002:0000254c       _DialogBoxParamA@20        0042754c f   user32:USER32.dll
 0002:00002552       _SetFocus@4                00427552 f   user32:USER32.dll
 0002:00002558       _GetDlgItem@8              00427558 f   user32:USER32.dll
 0002:0000255e       _MessageBoxA@16            0042755e f   user32:USER32.dll
 0002:00002564       _GetDlgItemTextA@16        00427564 f   user32:USER32.dll
 0002:0000256a       _EndDialog@8               0042756a f   user32:USER32.dll
 0002:00002570       _VMProtectEnd@0            00427570 f   VMProtectSDK32:VMProtectSDK32.dll
 0002:00002576       _VMProtectDecryptStringA@4 00427576 f   VMProtectSDK32:VMProtectSDK32.dll
 0002:0000257c       _VMProtectBegin@4          0042757c f   VMProtectSDK32:VMProtectSDK32.dll
 0002:00002590       __RTC_CheckEsp             00427590 f   LIBCMTD:_stack_.obj
 0002:000025c0       @_RTC_CheckStackVars@8     004275c0 f   LIBCMTD:_stack_.obj
 0002:00002640       @_RTC_AllocaHelper@12      00427640 f   LIBCMTD:_stack_.obj
 0002:00002680       @_RTC_CheckStackVars2@12   00427680 f   LIBCMTD:_stack_.obj
 0002:00002790       __RTC_InitBase             00427790 f   LIBCMTD:_init_.obj
 0002:000027d0       __RTC_Shutdown             004277d0 f   LIBCMTD:_init_.obj
 0002:000027f0       _atol                      004277f0 f   LIBCMTD:atox.obj
 0002:00002810       __atol_l                   00427810 f   LIBCMTD:atox.obj
 0002:00002840       _atoi                      00427840 f   LIBCMTD:atox.obj
 0002:00002860       __atoi_l                   00427860 f   LIBCMTD:atox.obj
 0002:00002880       __atoi64                   00427880 f   LIBCMTD:atox.obj
 0002:000028a0       __atoi64_l                 004278a0 f   LIBCMTD:atox.obj
 0002:000028d0       @__security_check_cookie@4 004278d0 f   LIBCMTD:secchk.obj
 0002:000028f0       _WinMainCRTStartup         004278f0 f   LIBCMTD:wincrt0.obj
 0002:00002c10       ?_RTC_Failure@@YAXPAXH@Z   00427c10 f   LIBCMTD:_error_.obj
 0002:000030a0       ?_RTC_StackFailure@@YAXPAXPBD@Z 004280a0 f   LIBCMTD:_error_.obj
 0002:000031e0       ?_RTC_AllocaFailure@@YAXPAXPAU_RTC_ALLOCA_NODE@@H@Z 004281e0 f   LIBCMTD:_error_.obj
 0002:000033f0       __RTC_UninitUse            004283f0 f   LIBCMTD:_error_.obj
 0002:00003520       __RTC_NumErrors            00428520 f   LIBCMTD:_userapi_.obj
 0002:00003530       __RTC_GetErrDesc           00428530 f   LIBCMTD:_userapi_.obj
 0002:00003550       __RTC_SetErrorType         00428550 f   LIBCMTD:_userapi_.obj
 0002:00003580       __RTC_SetErrorFunc         00428580 f   LIBCMTD:_userapi_.obj
 0002:000035b0       __RTC_SetErrorFuncW        004285b0 f   LIBCMTD:_userapi_.obj
 0002:000035e0       ?_RTC_GetErrorFunc@@YAP6AHHPBDH00ZZPBX@Z 004285e0 f   LIBCMTD:_userapi_.obj
 0002:000035f0       ?_RTC_GetErrorFuncW@@YAP6AHHPB_WH00ZZPBX@Z 004285f0 f   LIBCMTD:_userapi_.obj
 0002:00003600       __chkesp                   00428600 f   LIBCMTD:chkesp.obj
 0002:00003650       __CRT_RTC_INIT             00428650 f   LIBCMTD:chkesp.obj
 0002:00003660       __CRT_RTC_INITW            00428660 f   LIBCMTD:chkesp.obj
 0002:00003670       _strtol                    00428670 f   LIBCMTD:strtol.obj
 0002:00003cf0       ??0_LocaleUpdate@@QAE@PAUlocaleinfo_struct@@@Z 00428cf0 f i LIBCMTD:strtol.obj
 0002:00003e00       ??1_LocaleUpdate@@QAE@XZ   00428e00 f i LIBCMTD:strtol.obj
 0002:00003e40       ?GetLocaleT@_LocaleUpdate@@QAEPAUlocaleinfo_struct@@XZ 00428e40 f i LIBCMTD:strtol.obj
 0002:00003e60       __strtol_l                 00428e60 f   LIBCMTD:strtol.obj
 0002:00003e90       _strtoul                   00428e90 f   LIBCMTD:strtol.obj
 0002:00003ef0       __strtoul_l                00428ef0 f   LIBCMTD:strtol.obj
 0002:00003f20       __strtoi64                 00428f20 f   LIBCMTD:strtoq.obj
 0002:000045f0       __strtoi64_l               004295f0 f   LIBCMTD:strtoq.obj
 0002:00004620       __strtoui64                00429620 f   LIBCMTD:strtoq.obj
 0002:00004680       __strtoui64_l              00429680 f   LIBCMTD:strtoq.obj
 0002:000046b0       ___report_gsfailure        004296b0 f   LIBCMTD:gs_report.obj
 0002:00004810       ?__CxxUnhandledExceptionFilter@@YGJPAU_EXCEPTION_POINTERS@@@Z 00429810 f   LIBCMTD:unhandld.obj
 0002:00004890       ___CxxSetUnhandledExceptionFilter 00429890 f   LIBCMTD:unhandld.obj
 0002:000048b0       ___security_init_cookie    004298b0 f   LIBCMTD:gs_support.obj
 0002:000049d0       __cinit                    004299d0 f   LIBCMTD:crt0dat.obj
 0002:00004aa0       _exit                      00429aa0 f   LIBCMTD:crt0dat.obj
 0002:00004ac0       __exit                     00429ac0 f   LIBCMTD:crt0dat.obj
 0002:00004ae0       __cexit                    00429ae0 f   LIBCMTD:crt0dat.obj
 0002:00004b00       __c_exit                   00429b00 f   LIBCMTD:crt0dat.obj
 0002:00004b20       __amsg_exit                00429b20 f   LIBCMTD:crt0dat.obj
 0002:00004b50       ___freeCrtMemory           00429b50 f   LIBCMTD:crt0dat.obj
 0002:00004f60       ___crtCorExitProcess       00429f60 f   LIBCMTD:crt0dat.obj
 0002:00004fb0       ___crtExitProcess          00429fb0 f   LIBCMTD:crt0dat.obj
 0002:00004fe0       __lockexit                 00429fe0 f   LIBCMTD:crt0dat.obj
 0002:00005000       __unlockexit               0042a000 f   LIBCMTD:crt0dat.obj
 0002:00005020       __init_pointers            0042a020 f   LIBCMTD:crt0dat.obj
 0002:000050d0       __initterm_e               0042a0d0 f   LIBCMTD:crt0dat.obj
 0002:00005120       __get_wpgmptr              0042a120 f   LIBCMTD:crt0dat.obj
 0002:00005250       __get_pgmptr               0042a250 f   LIBCMTD:crt0dat.obj
 0002:00005380       ___CppXcptFilter           0042a380 f   LIBCMTD:winxfltr.obj
 0002:000053b0       __XcptFilter               0042a3b0 f   LIBCMTD:winxfltr.obj
 0002:000056a0       __wincmdln                 0042a6a0 f   LIBCMTD:wincmdln.obj
 0002:000057a0       __setenvp                  0042a7a0 f   LIBCMTD:stdenvp.obj
 0002:000059b0       __invoke_watson_if_error   0042a9b0 f i LIBCMTD:stdenvp.obj
 0002:000059f0       __setargv                  0042a9f0 f   LIBCMTD:stdargv.obj
 0002:00005b50       __set_pgmptr               0042ab50 f i LIBCMTD:stdargv.obj
 0002:00005fb0       ___crtGetEnvironmentStringsA 0042afb0 f   LIBCMTD:a_env.obj
 0002:000060f0       __ioinit                   0042b0f0 f   LIBCMTD:ioinit.obj
 0002:00006610       __ioterm                   0042b610 f   LIBCMTD:ioinit.obj
 0002:000066e0       __RTC_Initialize           0042b6e0 f   LIBCMTD:_initsect_.obj
 0002:00006710       __RTC_Terminate            0042b710 f   LIBCMTD:_initsect_.obj
 0002:00006740       __malloc_dbg               0042b740 f   LIBCMTD:dbgheap.obj
 0002:00006780       __nh_malloc                0042b780 f   LIBCMTD:dbgheap.obj
 0002:000067b0       __nh_malloc_dbg            0042b7b0 f   LIBCMTD:dbgheap.obj
 0002:000068b0       __heap_alloc               0042b8b0 f   LIBCMTD:dbgheap.obj
 0002:00006d80       __heap_alloc_dbg           0042bd80 f   LIBCMTD:dbgheap.obj
 0002:00006df0       __calloc_dbg_impl          0042bdf0 f   LIBCMTD:dbgheap.obj
 0002:00006e90       __calloc_dbg               0042be90 f   LIBCMTD:dbgheap.obj
 0002:00006f00       __recalloc                 0042bf00 f   LIBCMTD:dbgheap.obj
 0002:00006f40       __realloc_dbg              0042bf40 f   LIBCMTD:dbgheap.obj
 0002:00007780       __recalloc_dbg             0042c780 f   LIBCMTD:dbgheap.obj
 0002:00007860       __expand                   0042c860 f   LIBCMTD:dbgheap.obj
 0002:00007890       __expand_dbg               0042c890 f   LIBCMTD:dbgheap.obj
 0002:000079e0       __free_nolock              0042c9e0 f   LIBCMTD:dbgheap.obj
 0002:00007a00       __free_dbg                 0042ca00 f   LIBCMTD:dbgheap.obj
 0002:00007aa0       __free_dbg_nolock          0042caa0 f   LIBCMTD:dbgheap.obj
 0002:000080c0       __msize                    0042d0c0 f   LIBCMTD:dbgheap.obj
 0002:000080e0       __msize_dbg                0042d0e0 f   LIBCMTD:dbgheap.obj
 0002:00008340       __CrtSetBreakAlloc         0042d340 f   LIBCMTD:dbgheap.obj
 0002:00008370       __CrtSetDbgBlockType       0042d370 f   LIBCMTD:dbgheap.obj
 0002:00008490       __CrtSetAllocHook          0042d490 f   LIBCMTD:dbgheap.obj
 0002:000084c0       __CrtGetAllocHook          0042d4c0 f   LIBCMTD:dbgheap.obj
 0002:00008520       __CrtCheckMemory           0042d520 f   LIBCMTD:dbgheap.obj
 0002:00008a90       __CrtSetDbgFlag            0042da90 f   LIBCMTD:dbgheap.obj
 0002:00008c30       __CrtDoForAllClientObjects 0042dc30 f   LIBCMTD:dbgheap.obj
 0002:00008da0       __CrtIsValidPointer        0042dda0 f   LIBCMTD:dbgheap.obj
 0002:00008dc0       __CrtIsValidHeapPointer    0042ddc0 f   LIBCMTD:dbgheap.obj
 0002:00008e20       __CrtIsMemoryBlock         0042de20 f   LIBCMTD:dbgheap.obj
 0002:00008ff0       __CrtReportBlockType       0042dff0 f   LIBCMTD:dbgheap.obj
 0002:00009030       __CrtSetDumpClient         0042e030 f   LIBCMTD:dbgheap.obj
 0002:00009060       __CrtGetDumpClient         0042e060 f   LIBCMTD:dbgheap.obj
 0002:00009070       __CrtMemCheckpoint         0042e070 f   LIBCMTD:dbgheap.obj
 0002:00009310       __CrtMemDifference         0042e310 f   LIBCMTD:dbgheap.obj
 0002:000095b0       __CrtMemDumpAllObjectsSince 0042e5b0 f   LIBCMTD:dbgheap.obj
 0002:00009be0       __invoke_watson_if_oneof   0042ebe0 f i LIBCMTD:dbgheap.obj
 0002:00009c30       __CrtDumpMemoryLeaks       0042ec30 f   LIBCMTD:dbgheap.obj
 0002:00009cd0       __CrtMemDumpStatistics     0042ecd0 f   LIBCMTD:dbgheap.obj
 0002:00009e20       __aligned_malloc           0042ee20 f   LIBCMTD:dbgheap.obj
 0002:00009e50       __aligned_malloc_dbg       0042ee50 f   LIBCMTD:dbgheap.obj
 0002:00009e80       __aligned_realloc          0042ee80 f   LIBCMTD:dbgheap.obj
 0002:00009eb0       __aligned_recalloc         0042eeb0 f   LIBCMTD:dbgheap.obj
 0002:00009ee0       __aligned_realloc_dbg      0042eee0 f   LIBCMTD:dbgheap.obj
 0002:00009f10       __aligned_recalloc_dbg     0042ef10 f   LIBCMTD:dbgheap.obj
 0002:00009f50       __aligned_offset_malloc    0042ef50 f   LIBCMTD:dbgheap.obj
 0002:00009f80       __aligned_offset_malloc_dbg 0042ef80 f   LIBCMTD:dbgheap.obj
 0002:0000a1b0       __aligned_offset_realloc   0042f1b0 f   LIBCMTD:dbgheap.obj
 0002:0000a1e0       __aligned_offset_recalloc  0042f1e0 f   LIBCMTD:dbgheap.obj
 0002:0000a210       __aligned_offset_realloc_dbg 0042f210 f   LIBCMTD:dbgheap.obj
 0002:0000a5c0       __aligned_offset_recalloc_dbg 0042f5c0 f   LIBCMTD:dbgheap.obj
 0002:0000a6b0       __aligned_free             0042f6b0 f   LIBCMTD:dbgheap.obj
 0002:0000a6d0       __aligned_free_dbg         0042f6d0 f   LIBCMTD:dbgheap.obj
 0002:0000a7b0       __CrtSetDebugFillThreshold 0042f7b0 f   LIBCMTD:dbgheap.obj
 0002:0000a7e0       __CrtSetCheckCount         0042f7e0 f   LIBCMTD:dbgheap.obj
 0002:0000a800       __CrtGetCheckCount         0042f800 f   LIBCMTD:dbgheap.obj
 0002:0000a810       __aligned_msize            0042f810 f   LIBCMTD:dbgheap.obj
 0002:0000a840       __aligned_msize_dbg        0042f840 f   LIBCMTD:dbgheap.obj
 0002:0000a990       __encoded_null             0042f990 f   LIBCMTD:tidtable.obj
 0002:0000a9b0       ___crtTlsAlloc@4           0042f9b0 f   LIBCMTD:tidtable.obj
 0002:0000a9d0       ___fls_getvalue@4          0042f9d0 f   LIBCMTD:tidtable.obj
 0002:0000aa00       ___get_flsindex            0042fa00 f   LIBCMTD:tidtable.obj
 0002:0000aa10       ___set_flsgetvalue         0042fa10 f   LIBCMTD:tidtable.obj
 0002:0000aa70       ___fls_setvalue@8          0042fa70 f   LIBCMTD:tidtable.obj
 0002:0000aaa0       __mtinit                   0042faa0 f   LIBCMTD:tidtable.obj
 0002:0000ad20       __mtterm                   0042fd20 f   LIBCMTD:tidtable.obj
 0002:0000ad90       __initptd                  0042fd90 f   LIBCMTD:tidtable.obj
 0002:0000af00       __getptd_noexit            0042ff00 f   LIBCMTD:tidtable.obj
 0002:0000aff0       __getptd                   0042fff0 f   LIBCMTD:tidtable.obj
 0002:0000b020       __freefls@4                00430020 f   LIBCMTD:tidtable.obj
 0002:0000b2b0       __freeptd                  004302b0 f   LIBCMTD:tidtable.obj
 0002:0000b350       ___threadid                00430350 f   LIBCMTD:tidtable.obj
 0002:0000b360       ___threadhandle            00430360 f   LIBCMTD:tidtable.obj
 0002:0000b370       __heap_init                00430370 f   LIBCMTD:heapinit.obj
 0002:0000b3c0       __heap_term                004303c0 f   LIBCMTD:heapinit.obj
 0002:0000b3f0       __get_heap_handle          004303f0 f   LIBCMTD:heapinit.obj
 0002:0000b430       __except_handler4          00430430 f   LIBCMTD:chandler4.obj
 0002:0000b6e0       __FF_MSGBANNER             004306e0 f   LIBCMTD:crt0msg.obj
 0002:0000b740       __GET_RTERRMSG             00430740 f   LIBCMTD:crt0msg.obj
 0002:0000b7a0       __NMSG_WRITE               004307a0 f   LIBCMTD:crt0msg.obj
 0002:0000bba0       ?_RTC_GetSrcLine@@YAHPAEPA_WKPAH1K@Z 00430ba0 f   LIBCMTD:_pdblkup_.obj
 0002:0000c180       __CrtSetReportHook2        00431180 f   LIBCMTD:dbgrpt.obj
 0002:0000c570       __CrtDbgReport             00431570 f   LIBCMTD:dbgrpt.obj
 0002:0000c5c0       __CrtDbgReportV            004315c0 f i LIBCMTD:dbgrpt.obj
 0002:0000c5f0       ___crtMessageWindowA       004315f0 f   LIBCMTD:dbgrpt.obj
 0002:0000caf0       __CrtSetReportHookW2       00431af0 f   LIBCMTD:dbgrptw.obj
 0002:0000cee0       __CrtDbgReportW            00431ee0 f   LIBCMTD:dbgrptw.obj
 0002:0000cf30       __CrtDbgReportWV           00431f30 f i LIBCMTD:dbgrptw.obj
 0002:0000cf60       ___crtMessageWindowW       00431f60 f   LIBCMTD:dbgrptw.obj
 0002:0000d460       ?_CrtDbgReportW@@YAHHPBGH00ZZ 00432460 f   LIBCMTD:dbgrptw.obj
 0002:0000d4b0       ____setlc_active_func      004324b0 f   LIBCMTD:setlocal.obj
 0002:0000d4c0       ____unguarded_readlc_active_add_func 004324c0 f   LIBCMTD:setlocal.obj
 0002:0000d4d0       __configthreadlocale       004324d0 f   LIBCMTD:setlocal.obj
 0002:0000d620       __locterm                  00432620 f   LIBCMTD:setlocal.obj
 0002:0000d6e0       __free_locale              004326e0 f   LIBCMTD:setlocal.obj
 0002:0000d870       ___free_locale             00432870 f   LIBCMTD:setlocal.obj
 0002:0000d890       __create_locale            00432890 f   LIBCMTD:setlocal.obj
 0002:0000db50       ___create_locale           00432b50 f   LIBCMTD:setlocal.obj
 0002:0000db70       __get_current_locale       00432b70 f   LIBCMTD:setlocal.obj
 0002:0000dcd0       ___get_current_locale      00432cd0 f   LIBCMTD:setlocal.obj
 0002:0000dce0       _setlocale                 00432ce0 f   LIBCMTD:setlocal.obj
 0002:0000ef40       __expandlocale             00433f40 f   LIBCMTD:setlocal.obj
 0002:0000f290       ___init_dummy              00434290 f   LIBCMTD:setlocal.obj
 0002:0000f2a0       __strcats                  004342a0 f   LIBCMTD:setlocal.obj
 0002:0000f340       ___lc_strtolc              00434340 f   LIBCMTD:setlocal.obj
 0002:0000f5c0       ___lc_lctostr              004345c0 f   LIBCMTD:setlocal.obj
 0002:0000f680       __chvalidator              00434680 f   LIBCMTD:isctype.obj
 0002:0000f6e0       __chvalidator_l            004346e0 f   LIBCMTD:isctype.obj
 0002:0000f7c0       __isctype_l                004347c0 f   LIBCMTD:isctype.obj
 0002:0000f920       __isctype                  00434920 f   LIBCMTD:isctype.obj
 0002:0000f970       __initp_misc_invarg        00434970 f   LIBCMTD:invarg.obj
 0002:0000f990       __invalid_parameter        00434990 f   LIBCMTD:invarg.obj
 0002:0000fa00       __invoke_watson            00434a00 f   LIBCMTD:invarg.obj
 0002:0000fa40       __call_reportfault         00434a40 f   LIBCMTD:invarg.obj
 0002:0000fbf0       __set_invalid_parameter_handler 00434bf0 f   LIBCMTD:invarg.obj
 0002:0000fc40       __get_invalid_parameter_handler 00434c40 f   LIBCMTD:invarg.obj
 0002:0000fc80       ?_invalid_parameter@@YAXPBG00II@Z 00434c80 f   LIBCMTD:invarg.obj
 0002:0000fcb0       ?_invoke_watson@@YAXPBG00II@Z 00434cb0 f   LIBCMTD:invarg.obj
 0002:0000fce0       __dosmaperr                00434ce0 f   LIBCMTD:dosmap.obj
 0002:0000fd20       __get_errno_from_oserr     00434d20 f   LIBCMTD:dosmap.obj
 0002:0000fdc0       __set_errno                00434dc0 f   LIBCMTD:dosmap.obj
 0002:0000fe00       __get_errno                00434e00 f   LIBCMTD:dosmap.obj
 0002:0000fea0       __set_doserrno             00434ea0 f   LIBCMTD:dosmap.obj
 0002:0000fee0       __get_doserrno             00434ee0 f   LIBCMTD:dosmap.obj
 0002:0000ff80       __errno                    00434f80 f   LIBCMTD:dosmap.obj
 0002:0000ffb0       ___doserrno                00434fb0 f   LIBCMTD:dosmap.obj
 0002:0000ffe0       ?_JumpToContinuation@@YGXPAXPAUEHRegistrationNode@@@Z 00434fe0 f   LIBCMTD:_trnsctrl_.obj
 0002:00010030       ?_CallMemberFunction0@@YGXPAX0@Z 00435030 f   LIBCMTD:_trnsctrl_.obj
 0002:00010040       ?_CallMemberFunction1@@YGXPAX00@Z 00435040 f   LIBCMTD:_trnsctrl_.obj
 0002:00010050       ?_CallMemberFunction2@@YGXPAX00H@Z 00435050 f   LIBCMTD:_trnsctrl_.obj
 0002:00010060       ?_UnwindNestedFrames@@YGXPAUEHRegistrationNode@@PAUEHExceptionRecord@@@Z 00435060 f   LIBCMTD:_trnsctrl_.obj
 0002:000100d0       ___CxxFrameHandler         004350d0 f   LIBCMTD:_trnsctrl_.obj
 0002:00010120       ___CxxFrameHandler3        00435120 f   LIBCMTD:_trnsctrl_.obj
 0002:00010170       ___CxxFrameHandler2        00435170 f   LIBCMTD:_trnsctrl_.obj
 0002:000101c0       ___CxxLongjmpUnwind@4      004351c0 f   LIBCMTD:_trnsctrl_.obj
 0002:00010200       ?_CallCatchBlock2@@YAPAXPAUEHRegistrationNode@@PBU_s_FuncInfo@@PAXHK@Z 00435200 f   LIBCMTD:_trnsctrl_.obj
 0002:000102f0       ?_CallSETranslator@@YAHPAUEHExceptionRecord@@PAUEHRegistrationNode@@PAX2PBU_s_FuncInfo@@H1@Z 004352f0 f   LIBCMTD:_trnsctrl_.obj
 0002:00010500       ?_GetRangeOfTrysToCheck@@YAPBU_s_TryBlockMapEntry@@PBU_s_FuncInfo@@HHPAI1@Z 00435500 f   LIBCMTD:_trnsctrl_.obj
 0002:000105a0       __CreateFrameInfo          004355a0 f   LIBCMTD:_trnsctrl_.obj
 0002:000105e0       __IsExceptionObjectToBeDestroyed 004355e0 f   LIBCMTD:_trnsctrl_.obj
 0002:00010620       __FindAndUnlinkFrame       00435620 f   LIBCMTD:_trnsctrl_.obj
 0002:00010690       ___updatetmbcinfo          00435690 f   LIBCMTD:mbctype.obj
 0002:000107e0       __setmbcp                  004357e0 f   LIBCMTD:mbctype.obj
 0002:00010c70       __setmbcp_nolock           00435c70 f   LIBCMTD:mbctype.obj
 0002:00011650       __getmbcp                  00436650 f   LIBCMTD:mbctype.obj
 0002:000116e0       ___initmbctable            004366e0 f   LIBCMTD:mbctype.obj
 0002:00011710       ___addlocaleref            00436710 f   LIBCMTD:localref.obj
 0002:00011880       ___removelocaleref         00436880 f   LIBCMTD:localref.obj
 0002:00011a00       ___freetlocinfo            00436a00 f   LIBCMTD:localref.obj
 0002:00011da0       __updatetlocinfoEx_nolock  00436da0 f   LIBCMTD:localref.obj
 0002:00011e40       ___updatetlocinfo          00436e40 f   LIBCMTD:localref.obj
 0002:00011f40       __allmul                   00436f40 f   LIBCMTD:llmul.obj
 0002:00011f90       __aullrem                  00436f90 f   LIBCMTD:ullrem.obj
 0002:00012030       __aulldiv                  00437030 f   LIBCMTD:ulldiv.obj
 0002:000120c0       __CrtDefaultAllocHook      004370c0 f   LIBCMTD:dbghook.obj
 0002:000120d0       __crt_debugger_hook        004370d0 f   LIBCMTD:dbghook.obj
 0002:000120f0       __initp_eh_hooks           004370f0 f   LIBCMTD:hooks.obj
 0002:00012110       ?terminate@@YAXXZ          00437110 f   LIBCMTD:hooks.obj
 0002:000121b0       ?unexpected@@YAXXZ         004371b0 f   LIBCMTD:hooks.obj
 0002:000121e0       ?_inconsistency@@YAXXZ     004371e0 f   LIBCMTD:hooks.obj
 0002:00012290       __onexit                   00437290 f   LIBCMTD:onexit.obj
 0002:000124d0       _atexit                    004374d0 f   LIBCMTD:onexit.obj
 0002:00012500       ___onexitinit              00437500 f   LIBCMTD:onexit.obj
 0002:00012570       __initp_misc_cfltcvt_tab   00437570 f   LIBCMTD:cmiscdat.obj
 0002:000125c0       __ValidateImageBase        004375c0 f   LIBCMTD:pesect.obj
 0002:00012640       __FindPESection            00437640 f   LIBCMTD:pesect.obj
 0002:000126e0       __IsNonwritableInCurrentImage 004376e0 f   LIBCMTD:pesect.obj
 0002:00012840       __mtinitlocks              00437840 f   LIBCMTD:mlock.obj
 0002:000128f0       __mtdeletelocks            004378f0 f   LIBCMTD:mlock.obj
 0002:000129e0       __mtinitlocknum            004379e0 f   LIBCMTD:mlock.obj
 0002:00012b80       __lock                     00437b80 f   LIBCMTD:mlock.obj
 0002:00012bd0       __unlock                   00437bd0 f   LIBCMTD:mlock.obj
 0002:00012bf0       __lockerr_exit             00437bf0 f   LIBCMTD:mlock.obj
 0002:00012c20       __initp_misc_winsig        00437c20 f   LIBCMTD:winsig.obj
 0002:00012c60       _signal                    00437c60 f   LIBCMTD:winsig.obj
 0002:00013210       _raise                     00438210 f   LIBCMTD:winsig.obj
 0002:00013660       ___get_sigabrt             00438660 f   LIBCMTD:winsig.obj
 0002:00013680       ___fpecode                 00438680 f   LIBCMTD:winsig.obj
 0002:000136a0       ___pxcptinfoptrs           004386a0 f   LIBCMTD:winsig.obj
 0002:000136c0       __initp_misc_rand_s        004386c0 f   LIBCMTD:rand_s.obj
 0002:000136e0       _rand_s                    004386e0 f   LIBCMTD:rand_s.obj
 0002:00013980       ___getlocaleinfo           00438980 f   LIBCMTD:inithelp.obj
 0002:00013d10       __initp_misc_purevirt      00438d10 f   LIBCMTD:inithelp.obj
 0002:00013d30       __initp_heap_handler       00438d30 f   LIBCMTD:handler.obj
 0002:00013d50       ?_set_new_handler@@YAP6AHI@ZP6AHI@Z@Z 00438d50 f   LIBCMTD:handler.obj
 0002:00013da0       ?_set_new_handler@@YAP6AHI@ZH@Z 00438da0 f   LIBCMTD:handler.obj
 0002:00013df0       ?_query_new_handler@@YAP6AHI@ZXZ 00438df0 f   LIBCMTD:handler.obj
 0002:00013e10       __callnewh                 00438e10 f   LIBCMTD:handler.obj
 0002:00013e60       __ismbbkalnum_l            00438e60 f   LIBCMTD:ismbbyte.obj
 0002:00013e90       __ismbbkalnum              00438e90 f   LIBCMTD:ismbbyte.obj
 0002:00013eb0       __ismbbkprint_l            00438eb0 f   LIBCMTD:ismbbyte.obj
 0002:00013ee0       __ismbbkprint              00438ee0 f   LIBCMTD:ismbbyte.obj
 0002:00013f00       __ismbbkpunct_l            00438f00 f   LIBCMTD:ismbbyte.obj
 0002:00013f30       __ismbbkpunct              00438f30 f   LIBCMTD:ismbbyte.obj
 0002:00013f50       __ismbbalnum_l             00438f50 f   LIBCMTD:ismbbyte.obj
 0002:00013f80       __ismbbalnum               00438f80 f   LIBCMTD:ismbbyte.obj
 0002:00013fb0       __ismbbalpha_l             00438fb0 f   LIBCMTD:ismbbyte.obj
 0002:00013fe0       __ismbbalpha               00438fe0 f   LIBCMTD:ismbbyte.obj
 0002:00014010       __ismbbgraph_l             00439010 f   LIBCMTD:ismbbyte.obj
 0002:00014040       __ismbbgraph               00439040 f   LIBCMTD:ismbbyte.obj
 0002:00014070       __ismbbprint_l             00439070 f   LIBCMTD:ismbbyte.obj
 0002:000140a0       __ismbbprint               004390a0 f   LIBCMTD:ismbbyte.obj
 0002:000140d0       __ismbbpunct_l             004390d0 f   LIBCMTD:ismbbyte.obj
 0002:00014100       __ismbbpunct               00439100 f   LIBCMTD:ismbbyte.obj
 0002:00014120       __ismbblead_l              00439120 f   LIBCMTD:ismbbyte.obj
 0002:00014150       __ismbblead                00439150 f   LIBCMTD:ismbbyte.obj
 0002:00014170       __ismbbtrail_l             00439170 f   LIBCMTD:ismbbyte.obj
 0002:000141a0       __ismbbtrail               004391a0 f   LIBCMTD:ismbbyte.obj
 0002:000141c0       __ismbbkana_l              004391c0 f   LIBCMTD:ismbbyte.obj
 0002:00014250       __ismbbkana                00439250 f   LIBCMTD:ismbbyte.obj
 0002:00014370       _strcpy_s                  00439370 f   LIBCMTD:strcpy_s.obj
 0002:00014700       _strlen                    00439700 f   LIBCMTD:strlen.obj
 0002:000147b0       _memset                    004397b0 f   LIBCMTD:memset.obj
 0002:00014850       __malloc_base              00439850 f   LIBCMTD:malloc.obj
 0002:00014900       __heap_alloc_base          00439900 f i LIBCMTD:malloc.obj
 0002:00014970       __expand_base              00439970 f   LIBCMTD:expand.obj
 0002:00014b20       __realloc_base             00439b20 f   LIBCMTD:realloc.obj
 0002:00014c60       __free_base                00439c60 f   LIBCMTD:free.obj
 0002:00014cd0       __heapchk                  00439cd0 f   LIBCMTD:heapchk.obj
 0002:00014d10       __heapset                  00439d10 f   LIBCMTD:heapchk.obj
 0002:00014d20       _sprintf                   00439d20 f   LIBCMTD:sprintf.obj
 0002:00014f20       __sprintf_l                00439f20 f   LIBCMTD:sprintf.obj
 0002:00014f60       _sprintf_s                 00439f60 f   LIBCMTD:sprintf.obj
 0002:00014fa0       __sprintf_s_l              00439fa0 f   LIBCMTD:sprintf.obj
 0002:00014fe0       __snprintf_s               00439fe0 f   LIBCMTD:sprintf.obj
 0002:00015020       __snprintf_s_l             0043a020 f   LIBCMTD:sprintf.obj
 0002:00015060       __sprintf_p                0043a060 f   LIBCMTD:sprintf.obj
 0002:000150a0       __sprintf_p_l              0043a0a0 f   LIBCMTD:sprintf.obj
 0002:000150e0       __scprintf                 0043a0e0 f   LIBCMTD:sprintf.obj
 0002:00015110       __scprintf_p               0043a110 f   LIBCMTD:sprintf.obj
 0002:00015140       __scprintf_l               0043a140 f   LIBCMTD:sprintf.obj
 0002:00015170       __scprintf_p_l             0043a170 f   LIBCMTD:sprintf.obj
 0002:000151a0       _memcpy                    0043a1a0 f   LIBCMTD:memcpy.obj
 0002:000155e0       __local_unwind4            0043a5e0 f   LIBCMTD:exsup4.obj
 0002:000156b6       __seh_longjmp_unwind4@4    0043a6b6 f   LIBCMTD:exsup4.obj
 0002:000156d2       @_EH4_CallFilterFunc@8     0043a6d2 f   LIBCMTD:exsup4.obj
 0002:000156e9       @_EH4_TransferToHandler@8  0043a6e9 f   LIBCMTD:exsup4.obj
 0002:00015702       @_EH4_GlobalUnwind2@8      0043a702 f   LIBCMTD:exsup4.obj
 0002:0001571b       @_EH4_LocalUnwind@16       0043a71b f   LIBCMTD:exsup4.obj
 0002:00015790       __set_error_mode           0043a790 f   LIBCMTD:errmode.obj
 0002:00015880       ___set_app_type            0043a880 f   LIBCMTD:errmode.obj
 0002:000158a0       ___crtMessageBoxW          0043a8a0 f   LIBCMTD:crtmboxw.obj
 0002:00015b50       _wcscat_s                  0043ab50 f   LIBCMTD:wcscat_s.obj
 0002:00016030       _wcsncpy_s                 0043b030 f   LIBCMTD:wcsncpy_s.obj
 0002:00016540       _wcslen                    0043b540 f   LIBCMTD:wcslen.obj
 0002:00016580       _wcscpy_s                  0043b580 f   LIBCMTD:wcscpy_s.obj
 0002:00016920       __CrtDbgBreak              0043b920 f   LIBCMTD:dbgrptt.obj
 0002:00016930       __CrtSetReportMode         0043b930 f   LIBCMTD:dbgrptt.obj
 0002:00016ac0       __CrtSetReportFile         0043bac0 f   LIBCMTD:dbgrptt.obj
 0002:00016bf0       __CrtSetReportHook         0043bbf0 f   LIBCMTD:dbgrptt.obj
 0002:00016c20       __CrtGetReportHook         0043bc20 f   LIBCMTD:dbgrptt.obj
 0002:00016c30       __VCrtDbgReportA           0043bc30 f   LIBCMTD:dbgrptt.obj
 0002:00017660       __VCrtDbgReportW           0043c660 f   LIBCMTD:dbgrptt.obj
 0002:000181e0       ___crtMessageBoxA          0043d1e0 f   LIBCMTD:crtmbox.obj
 0002:00018490       _memcpy_s                  0043d490 f   LIBCMTD:memcpy_s.obj
 0002:00018680       __alloca_probe             0043d680     LIBCMTD:chkstk.obj
 0002:00018680       __chkstk                   0043d680 f   LIBCMTD:chkstk.obj
 0002:000186c0       __swprintf                 0043d6c0 f   LIBCMTD:swprintf.obj
 0002:00018940       ___swprintf_l              0043d940 f   LIBCMTD:swprintf.obj
 0002:00018980       _swprintf_s                0043d980 f   LIBCMTD:swprintf.obj
 0002:000189c0       __snwprintf_s              0043d9c0 f   LIBCMTD:swprintf.obj
 0002:00018a00       __swprintf_p               0043da00 f   LIBCMTD:swprintf.obj
 0002:00018a40       __swprintf_s_l             0043da40 f   LIBCMTD:swprintf.obj
 0002:00018a80       __snwprintf_s_l            0043da80 f   LIBCMTD:swprintf.obj
 0002:00018ac0       __swprintf_p_l             0043dac0 f   LIBCMTD:swprintf.obj
 0002:00018b00       __scwprintf                0043db00 f   LIBCMTD:swprintf.obj
 0002:00018b30       __scwprintf_p              0043db30 f   LIBCMTD:swprintf.obj
 0002:00018b60       __scwprintf_l              0043db60 f   LIBCMTD:swprintf.obj
 0002:00018b90       __scwprintf_p_l            0043db90 f   LIBCMTD:swprintf.obj
 0002:00018bc0       ___pwctype_func            0043dbc0 f   LIBCMTD:ctype.obj
 0002:00018bd0       ___pctype_func             0043dbd0 f   LIBCMTD:ctype.obj
 0002:00018c30       _localeconv                0043dc30 f   LIBCMTD:lconv.obj
 0002:00018c90       ___init_time               0043dc90 f   LIBCMTD:inittime.obj
 0002:00019d00       ___free_lc_time            0043ed00 f   LIBCMTD:inittime.obj
 0002:0001a510       ___init_numeric            0043f510 f   LIBCMTD:initnum.obj
 0002:0001a9b0       ___free_lconv_num          0043f9b0 f   LIBCMTD:initnum.obj
 0002:0001aa90       ___init_monetary           0043fa90 f   LIBCMTD:initmon.obj
 0002:0001b1f0       ___free_lconv_mon          004401f0 f   LIBCMTD:initmon.obj
 0002:0001b400       ___init_ctype              00440400 f   LIBCMTD:initctyp.obj
 0002:0001bb20       ____mb_cur_max_func        00440b20 f   LIBCMTD:initctyp.obj
 0002:0001bb80       ____mb_cur_max_l_func      00440b80 f   LIBCMTD:initctyp.obj
 0002:0001bbc0       ____lc_codepage_func       00440bc0 f   LIBCMTD:initctyp.obj
 0002:0001bc20       ____lc_collate_cp_func     00440c20 f   LIBCMTD:initctyp.obj
 0002:0001bc80       ____lc_handle_func         00440c80 f   LIBCMTD:initctyp.obj
 0002:0001bce0       ___init_collate            00440ce0 f   LIBCMTD:initcoll.obj
 0002:0001bcf0       _strcmp                    00440cf0 f   LIBCMTD:strcmp.obj
 0002:0001bda0       _strncpy_s                 00440da0 f   LIBCMTD:strncpy_s.obj
 0002:0001c290       _strcspn                   00441290 f   LIBCMTD:strcspn.obj
 0002:0001c2f0       _strncmp                   004412f0 f   LIBCMTD:strncmp.obj
 0002:0001c4c0       _strpbrk                   004414c0 f   LIBCMTD:strpbrk.obj
 0002:0001c510       _memcmp                    00441510 f   LIBCMTD:memcmp.obj
 0002:0001d230       ___crtGetStringTypeA       00442230 f   LIBCMTD:a_str.obj
 0002:0001d3f0       __MarkAllocaS              004423f0 f i LIBCMTD:a_str.obj
 0002:0001d420       __freea                    00442420 f i LIBCMTD:a_str.obj
 0002:0001d4a0       _strcat_s                  004424a0 f   LIBCMTD:strcat_s.obj
 0002:0001d970       ___get_qualified_locale    00442970 f   LIBCMTD:getqloc.obj
 0002:0001eb40       __isleadbyte_l             00443b40 f i LIBCMTD:_wctype.obj
 0002:0001eba0       _isleadbyte                00443ba0 f i LIBCMTD:_wctype.obj
 0002:0001ebc0       __iswalpha_l               00443bc0 f i LIBCMTD:_wctype.obj
 0002:0001ebe0       _iswalpha                  00443be0 f i LIBCMTD:_wctype.obj
 0002:0001ec00       __iswupper_l               00443c00 f i LIBCMTD:_wctype.obj
 0002:0001ec20       _iswupper                  00443c20 f i LIBCMTD:_wctype.obj
 0002:0001ec40       __iswlower_l               00443c40 f i LIBCMTD:_wctype.obj
 0002:0001ec60       _iswlower                  00443c60 f i LIBCMTD:_wctype.obj
 0002:0001ec80       __iswdigit_l               00443c80 f i LIBCMTD:_wctype.obj
 0002:0001eca0       _iswdigit                  00443ca0 f i LIBCMTD:_wctype.obj
 0002:0001ecc0       __iswxdigit_l              00443cc0 f i LIBCMTD:_wctype.obj
 0002:0001ece0       _iswxdigit                 00443ce0 f i LIBCMTD:_wctype.obj
 0002:0001ed00       __iswspace_l               00443d00 f i LIBCMTD:_wctype.obj
 0002:0001ed20       _iswspace                  00443d20 f i LIBCMTD:_wctype.obj
 0002:0001ed40       __iswpunct_l               00443d40 f i LIBCMTD:_wctype.obj
 0002:0001ed60       _iswpunct                  00443d60 f i LIBCMTD:_wctype.obj
 0002:0001ed80       __iswalnum_l               00443d80 f i LIBCMTD:_wctype.obj
 0002:0001eda0       _iswalnum                  00443da0 f i LIBCMTD:_wctype.obj
 0002:0001edc0       __iswprint_l               00443dc0 f i LIBCMTD:_wctype.obj
 0002:0001ede0       _iswprint                  00443de0 f i LIBCMTD:_wctype.obj
 0002:0001ee00       __iswgraph_l               00443e00 f i LIBCMTD:_wctype.obj
 0002:0001ee20       _iswgraph                  00443e20 f i LIBCMTD:_wctype.obj
 0002:0001ee40       __iswcntrl_l               00443e40 f i LIBCMTD:_wctype.obj
 0002:0001ee60       _iswcntrl                  00443e60 f i LIBCMTD:_wctype.obj
 0002:0001ee80       _iswascii                  00443e80 f i LIBCMTD:_wctype.obj
 0002:0001eea0       __iswcsym_l                00443ea0 f i LIBCMTD:_wctype.obj
 0002:0001eef0       ___iswcsym                 00443ef0 f i LIBCMTD:_wctype.obj
 0002:0001ef40       __iswcsymf_l               00443f40 f i LIBCMTD:_wctype.obj
 0002:0001ef90       ___iswcsymf                00443f90 f i LIBCMTD:_wctype.obj
 0002:0001efe0       ___InternalCxxFrameHandler 00443fe0 f   LIBCMTD:frame.obj
 0002:0001f750       ??0bad_exception@std@@QAE@PBD@Z 00444750 f i LIBCMTD:frame.obj
 0002:0001f780       ??1bad_exception@std@@UAE@XZ 00444780 f i LIBCMTD:frame.obj
 0002:0001f7b0       ??_Gbad_exception@std@@UAEPAXI@Z 004447b0 f i LIBCMTD:frame.obj
 0002:0001f7b0       ??_Ebad_exception@std@@UAEPAXI@Z 004447b0 f i LIBCMTD:frame.obj
 0002:0001f7f0       ??0bad_exception@std@@QAE@ABV01@@Z 004447f0 f i LIBCMTD:frame.obj
 0002:0001fa10       ___TypeMatch               00444a10 f   LIBCMTD:frame.obj
 0002:0001faf0       ___FrameUnwindFilter       00444af0 f   LIBCMTD:frame.obj
 0002:0001fb90       ___FrameUnwindToState      00444b90 f   LIBCMTD:frame.obj
 0002:00020220       ___BuildCatchObjectHelper  00445220 f   LIBCMTD:frame.obj
 0002:00020530       ___BuildCatchObject        00445530 f   LIBCMTD:frame.obj
 0002:00020680       ___DestructExceptionObject 00445680 f   LIBCMTD:frame.obj
 0002:00020760       ___AdjustPointer           00445760 f   LIBCMTD:frame.obj
 0002:000207c0       ?__uncaught_exception@@YA_NXZ 004457c0 f   LIBCMTD:frame.obj
 0002:000207e0       ___CxxExceptionFilter      004457e0 f   LIBCMTD:frame.obj
 0002:00020a50       ___CxxRegisterExceptionObject 00445a50 f   LIBCMTD:frame.obj
 0002:00020bd0       ___CxxDetectRethrow        00445bd0 f   LIBCMTD:frame.obj
 0002:00020c80       ___CxxUnregisterExceptionObject 00445c80 f   LIBCMTD:frame.obj
 0002:00020e60       ___CxxQueryExceptionSize   00445e60 f   LIBCMTD:frame.obj
 0002:00020e70       ___CxxCallUnwindDtor       00445e70 f   LIBCMTD:frame.obj
 0002:00020f10       ___CxxCallUnwindDelDtor    00445f10 f   LIBCMTD:frame.obj
 0002:00020fb0       ___CxxCallUnwindStdDelDtor 00445fb0 f   LIBCMTD:frame.obj
 0002:00021050       ___CxxCallUnwindVecDtor    00446050 f   LIBCMTD:frame.obj
 0002:00021320       ?_is_exception_typeof@@YAHABVtype_info@@PAU_EXCEPTION_POINTERS@@@Z 00446320 f   LIBCMTD:frame.obj
 0002:00021430       __CallSettingFrame@12      00446430 f   LIBCMTD:lowhelpr.obj
 0002:00021457       __NLG_Return               00446457     LIBCMTD:lowhelpr.obj
 0002:00021490       ___crtLCMapStringA         00446490 f   LIBCMTD:a_map.obj
 0002:000218a0       _abort                     004468a0 f   LIBCMTD:abort.obj
 0002:00021920       __set_abort_behavior       00446920 f   LIBCMTD:abort.obj
 0002:00021960       __fptrap                   00446960 f   LIBCMTD:crt0fp.obj
 0002:00021980       ___crtGetLocaleInfoA       00446980 f   LIBCMTD:a_loc.obj
 0002:00021b30       __VEC_memzero              00446b30 f   LIBCMTD:p4_memset.obj
 0002:00021c20       ___sse2_available_init     00446c20 f   LIBCMTD:cpu_disp.obj
 0002:00021c40       __flsbuf                   00446c40 f   LIBCMTD:_flsbuf.obj
 0002:00021fb0       __output_l                 00446fb0 f   LIBCMTD:output.obj
 0002:000238f0       _get_int_arg               004488f0 f i LIBCMTD:output.obj
 0002:00023920       _get_int64_arg             00448920 f i LIBCMTD:output.obj
 0002:00023950       _get_short_arg             00448950 f i LIBCMTD:output.obj
 0002:00023980       __vsprintf_l               00448980 f   LIBCMTD:vsprintf.obj
 0002:00023b80       _vsprintf                  00448b80 f   LIBCMTD:vsprintf.obj
 0002:00023bb0       __vscprintf_helper         00448bb0 f   LIBCMTD:vsprintf.obj
 0002:00023cc0       __vscprintf                00448cc0 f   LIBCMTD:vsprintf.obj
 0002:00023cf0       __vscprintf_l              00448cf0 f   LIBCMTD:vsprintf.obj
 0002:00023d20       __vscprintf_p              00448d20 f   LIBCMTD:vsprintf.obj
 0002:00023d50       __vscprintf_p_l            00448d50 f   LIBCMTD:vsprintf.obj
 0002:00023d80       __vsnprintf_helper         00448d80 f   LIBCMTD:vsnprnc.obj
 0002:00023fe0       __vsnprintf_c              00448fe0 f   LIBCMTD:vsnprnc.obj
 0002:00024040       __vsnprintf_c_l            00449040 f   LIBCMTD:vsnprnc.obj
 0002:000240a0       __vsprintf_s_l             004490a0 f   LIBCMTD:vsnprnc.obj
 0002:000243a0       _vsprintf_s                004493a0 f   LIBCMTD:vsnprnc.obj
 0002:000243d0       __vsnprintf_s_l            004493d0 f   LIBCMTD:vsnprnc.obj
 0002:00024850       __vsnprintf_s              00449850 f   LIBCMTD:vsnprnc.obj
 0002:00024880       __vsprintf_p               00449880 f   LIBCMTD:vsnprnc.obj
 0002:000248e0       __vsprintf_p_l             004498e0 f   LIBCMTD:vsnprnc.obj
 0002:00024940       __VEC_memcpy               00449940 f   LIBCMTD:p4_memcpy.obj
 0002:00024a90       __global_unwind2           00449a90 f   LIBCMTD:exsup.obj
 0002:00024af5       __local_unwind2            00449af5 f   LIBCMTD:exsup.obj
 0002:00024b79       __abnormal_termination     00449b79 f   LIBCMTD:exsup.obj
 0002:00024b9c       __NLG_Notify1              00449b9c f   LIBCMTD:exsup.obj
 0002:00024ba5       __NLG_Notify               00449ba5 f   LIBCMTD:exsup.obj
 0002:00024bbc       __NLG_Dispatch             00449bbc     LIBCMTD:exsup.obj
 0002:00024bbc       __NLG_Dispatch2            00449bbc     LIBCMTD:exsup.obj
 0002:00024bc4       __NLG_Call                 00449bc4 f   LIBCMTD:exsup.obj
 0002:00024bc6       __NLG_Return2              00449bc6     LIBCMTD:exsup.obj
 0002:00024c20       __mbstowcs_l_helper        00449c20 f   LIBCMTD:mbstowcs.obj
 0002:00025050       __mbstowcs_l               0044a050 f   LIBCMTD:mbstowcs.obj
 0002:00025080       _mbstowcs                  0044a080 f   LIBCMTD:mbstowcs.obj
 0002:000250e0       __mbstowcs_s_l             0044a0e0 f   LIBCMTD:mbstowcs.obj
 0002:00025540       _mbstowcs_s                0044a540 f   LIBCMTD:mbstowcs.obj
 0002:00025570       __itoa_s                   0044a570 f   LIBCMTD:xtoas.obj
 0002:00025a20       __ltoa_s                   0044aa20 f   LIBCMTD:xtoas.obj
 0002:00025a70       __ultoa_s                  0044aa70 f   LIBCMTD:xtoas.obj
 0002:00025aa0       __i64toa_s                 0044aaa0 f   LIBCMTD:xtoas.obj
 0002:00025fa0       __ui64toa_s                0044afa0 f   LIBCMTD:xtoas.obj
 0002:00025fd0       __wcstombs_l_helper        0044afd0 f   LIBCMTD:wcstombs.obj
 0002:00026670       __wcstombs_l               0044b670 f   LIBCMTD:wcstombs.obj
 0002:000266a0       _wcstombs                  0044b6a0 f   LIBCMTD:wcstombs.obj
 0002:000266d0       __wcstombs_s_l             0044b6d0 f   LIBCMTD:wcstombs.obj
 0002:00026ac0       _wcstombs_s                0044bac0 f   LIBCMTD:wcstombs.obj
 0002:00026af0       __vswprintf_helper         0044baf0 f   LIBCMTD:vswprnc.obj
 0002:00026de0       __vswprintf_c              0044bde0 f   LIBCMTD:vswprnc.obj
 0002:00026e40       __vswprintf_c_l            0044be40 f   LIBCMTD:vswprnc.obj
 0002:00026ea0       __vswprintf_s_l            0044bea0 f   LIBCMTD:vswprnc.obj
 0002:000271a0       _vswprintf_s               0044c1a0 f   LIBCMTD:vswprnc.obj
 0002:000271d0       __vsnwprintf_s_l           0044c1d0 f   LIBCMTD:vswprnc.obj
 0002:00027670       __vsnwprintf_s             0044c670 f   LIBCMTD:vswprnc.obj
 0002:000276a0       __vswprintf_p              0044c6a0 f   LIBCMTD:vswprnc.obj
 0002:00027700       __vswprintf_p_l            0044c700 f   LIBCMTD:vswprnc.obj
 0002:00027760       __itow_s                   0044c760 f   LIBCMTD:xtows.obj
 0002:00027c30       __ltow_s                   0044cc30 f   LIBCMTD:xtows.obj
 0002:00027c80       __ultow_s                  0044cc80 f   LIBCMTD:xtows.obj
 0002:00027cb0       __i64tow_s                 0044ccb0 f   LIBCMTD:xtows.obj
 0002:000281d0       __ui64tow_s                0044d1d0 f   LIBCMTD:xtows.obj
 0002:00028200       __woutput_l                0044d200 f   LIBCMTD:woutput.obj
 0002:00029850       __vswprintf_l              0044e850 f   LIBCMTD:vswprint.obj
 0002:00029ac0       __vswprintf                0044eac0 f   LIBCMTD:vswprint.obj
 0002:00029af0       ___vswprintf_l             0044eaf0 f   LIBCMTD:vswprint.obj
 0002:00029b20       __vscwprintf_helper        0044eb20 f   LIBCMTD:vswprint.obj
 0002:00029c30       __vscwprintf               0044ec30 f   LIBCMTD:vswprint.obj
 0002:00029c60       __vscwprintf_l             0044ec60 f   LIBCMTD:vswprint.obj
 0002:00029c90       __vscwprintf_p             0044ec90 f   LIBCMTD:vswprint.obj
 0002:00029cc0       __vscwprintf_p_l           0044ecc0 f   LIBCMTD:vswprint.obj
 0002:00029cf0       _malloc                    0044ecf0 f   LIBCMTD:dbgmalloc.obj
 0002:00029d30       _free                      0044ed30 f   LIBCMTD:dbgfree.obj
 0002:00029d50       __stricmp_l                0044ed50 f   LIBCMTD:stricmp.obj
 0002:00029f60       ___ascii_stricmp           0044ef60 f   LIBCMTD:stricmp.obj
 0002:00029ff0       __stricmp                  0044eff0 f   LIBCMTD:stricmp.obj
 0002:0002a140       __strnicmp_l               0044f140 f   LIBCMTD:strnicmp.obj
 0002:0002a410       __strnicmp                 0044f410 f   LIBCMTD:strnicmp.obj
 0002:0002a600       __iswctype_l               0044f600 f   LIBCMTD:iswctype.obj
 0002:0002a620       _iswctype                  0044f620 f   LIBCMTD:iswctype.obj
 0002:0002a6a0       _is_wctype                 0044f6a0 f   LIBCMTD:iswctype.obj
 0002:0002a6c0       ?_ValidateRead@@YAHPBXI@Z  0044f6c0 f   LIBCMTD:validate.obj
 0002:0002a6f0       ?_ValidateWrite@@YAHPAXI@Z 0044f6f0 f   LIBCMTD:validate.obj
 0002:0002a720       ?_ValidateExecute@@YAHP6GHXZ@Z 0044f720 f   LIBCMTD:validate.obj
 0002:0002a750       __CxxThrowException@8      0044f750 f   LIBCMTD:throw.obj
 0002:0002a7c0       ?name@type_info@@QBEPBDPAU__type_info_node@@@Z 0044f7c0 f   LIBCMTD:typinfo.obj
 0002:0002a7f0       ??1type_info@@UAE@XZ       0044f7f0 f   LIBCMTD:typinfo.obj
 0002:0002a820       ??_Gtype_info@@UAEPAXI@Z   0044f820 f i LIBCMTD:typinfo.obj
 0002:0002a820       ??_Etype_info@@UAEPAXI@Z   0044f820 f i LIBCMTD:typinfo.obj
 0002:0002a860       ?_name_internal_method@type_info@@QBEPBDPAU__type_info_node@@@Z 0044f860 f   LIBCMTD:typinfo.obj
 0002:0002a890       ?_type_info_dtor_internal_method@type_info@@QAEXXZ 0044f890 f   LIBCMTD:typinfo.obj
 0002:0002a8b0       ??8type_info@@QBE_NABV0@@Z 0044f8b0 f   LIBCMTD:typinfo.obj
 0002:0002a8f0       ??9type_info@@QBE_NABV0@@Z 0044f8f0 f   LIBCMTD:typinfo.obj
 0002:0002a930       ?before@type_info@@QBEHABV1@@Z 0044f930 f   LIBCMTD:typinfo.obj
 0002:0002a970       ?raw_name@type_info@@QBEPBDXZ 0044f970 f   LIBCMTD:typinfo.obj
 0002:0002a990       ??0type_info@@AAE@ABV0@@Z  0044f990 f   LIBCMTD:typinfo.obj
 0002:0002a9c0       ??4type_info@@AAEAAV0@ABV0@@Z 0044f9c0 f   LIBCMTD:typinfo.obj
 0002:0002a9e0       ??0exception@std@@QAE@XZ   0044f9e0 f   LIBCMTD:stdexcpt.obj
 0002:0002aa20       ??_Eexception@std@@UAEPAXI@Z 0044fa20 f i LIBCMTD:stdexcpt.obj
 0002:0002aa20       ??_Gexception@std@@UAEPAXI@Z 0044fa20 f i LIBCMTD:stdexcpt.obj
 0002:0002aa60       ??0exception@std@@QAE@ABQBD@Z 0044fa60 f   LIBCMTD:stdexcpt.obj
 0002:0002aab0       ??0exception@std@@QAE@ABQBDH@Z 0044fab0 f   LIBCMTD:stdexcpt.obj
 0002:0002aaf0       ??0exception@std@@QAE@ABV01@@Z 0044faf0 f   LIBCMTD:stdexcpt.obj
 0002:0002ab40       ??4exception@std@@QAEAAV01@ABV01@@Z 0044fb40 f   LIBCMTD:stdexcpt.obj
 0002:0002aba0       ??1exception@std@@UAE@XZ   0044fba0 f   LIBCMTD:stdexcpt.obj
 0002:0002abd0       ?what@exception@std@@UBEPBDXZ 0044fbd0 f   LIBCMTD:stdexcpt.obj
 0002:0002ac10       ?_Copy_str@exception@std@@AAEXPBD@Z 0044fc10 f   LIBCMTD:stdexcpt.obj
 0002:0002ac90       ?_Tidy@exception@std@@AAEXXZ 0044fc90 f   LIBCMTD:stdexcpt.obj
 0002:0002ace0       ??0bad_cast@std@@QAE@PBD@Z 0044fce0 f   LIBCMTD:stdexcpt.obj
 0002:0002ad10       ??_Gbad_cast@std@@UAEPAXI@Z 0044fd10 f i LIBCMTD:stdexcpt.obj
 0002:0002ad10       ??_Ebad_cast@std@@UAEPAXI@Z 0044fd10 f i LIBCMTD:stdexcpt.obj
 0002:0002ad50       ??0bad_cast@std@@QAE@ABV01@@Z 0044fd50 f   LIBCMTD:stdexcpt.obj
 0002:0002ad80       ??1bad_cast@std@@UAE@XZ    0044fd80 f   LIBCMTD:stdexcpt.obj
 0002:0002adb0       ??0bad_typeid@std@@QAE@PBD@Z 0044fdb0 f   LIBCMTD:stdexcpt.obj
 0002:0002ade0       ??_Gbad_typeid@std@@UAEPAXI@Z 0044fde0 f i LIBCMTD:stdexcpt.obj
 0002:0002ade0       ??_Ebad_typeid@std@@UAEPAXI@Z 0044fde0 f i LIBCMTD:stdexcpt.obj
 0002:0002ae20       ??0bad_typeid@std@@QAE@ABV01@@Z 0044fe20 f   LIBCMTD:stdexcpt.obj
 0002:0002ae50       ??1bad_typeid@std@@UAE@XZ  0044fe50 f   LIBCMTD:stdexcpt.obj
 0002:0002ae80       ??0__non_rtti_object@std@@QAE@PBD@Z 0044fe80 f   LIBCMTD:stdexcpt.obj
 0002:0002aeb0       ??_G__non_rtti_object@std@@UAEPAXI@Z 0044feb0 f i LIBCMTD:stdexcpt.obj
 0002:0002aeb0       ??_E__non_rtti_object@std@@UAEPAXI@Z 0044feb0 f i LIBCMTD:stdexcpt.obj
 0002:0002aef0       ??0__non_rtti_object@std@@QAE@ABV01@@Z 0044fef0 f   LIBCMTD:stdexcpt.obj
 0002:0002af20       ??1__non_rtti_object@std@@UAE@XZ 0044ff20 f   LIBCMTD:stdexcpt.obj
 0002:0002af50       ??3@YAXPAX@Z               0044ff50 f   LIBCMTD:dbgdel.obj
 0002:0002b070       _memmove                   00450070 f   LIBCMTD:memmove.obj
 0002:0002b4b0       __lseeki64                 004504b0 f   LIBCMTD:lseeki64.obj
 0002:0002b790       __lseeki64_nolock          00450790 f   LIBCMTD:lseeki64.obj
 0002:0002b8c0       __write                    004508c0 f   LIBCMTD:write.obj
 0002:0002bb70       __write_nolock             00450b70 f   LIBCMTD:write.obj
 0002:0002c980       __getbuf                   00451980 f   LIBCMTD:_getbuf.obj
 0002:0002ca80       __isatty                   00451a80 f   LIBCMTD:isatty.obj
 0002:0002cb70       ___iob_func                00451b70 f   LIBCMTD:_file.obj
 0002:0002cb80       ___initstdio               00451b80 f   LIBCMTD:_file.obj
 0002:0002cd20       ___endstdio                00451d20 f   LIBCMTD:_file.obj
 0002:0002cd60       __lock_file                00451d60 f   LIBCMTD:_file.obj
 0002:0002cdd0       __lock_file2               00451dd0 f   LIBCMTD:_file.obj
 0002:0002ce20       __unlock_file              00451e20 f   LIBCMTD:_file.obj
 0002:0002ce90       __unlock_file2             00451e90 f   LIBCMTD:_file.obj
 0002:0002cee0       __fileno                   00451ee0 f   LIBCMTD:fileno.obj
 0002:0002cf70       _printf                    00451f70 f   LIBCMTD:printf.obj
 0002:0002d100       __printf_l                 00452100 f   LIBCMTD:printf.obj
 0002:0002d130       __printf_s_l               00452130 f   LIBCMTD:printf.obj
 0002:0002d160       _printf_s                  00452160 f   LIBCMTD:printf.obj
 0002:0002d190       __printf_p_l               00452190 f   LIBCMTD:printf.obj
 0002:0002d1c0       __printf_p                 004521c0 f   LIBCMTD:printf.obj
 0002:0002d1f0       __set_printf_count_output  004521f0 f   LIBCMTD:printf.obj
 0002:0002d250       __get_printf_count_output  00452250 f   LIBCMTD:printf.obj
 0002:0002d280       __wctomb_s_l               00452280 f   LIBCMTD:wctomb.obj
 0002:0002d640       _wctomb_s                  00452640 f   LIBCMTD:wctomb.obj
 0002:0002d670       __wctomb_l                 00452670 f   LIBCMTD:wctomb.obj
 0002:0002d710       _wctomb                    00452710 f   LIBCMTD:wctomb.obj
 0002:0002d770       __validate_param_reuseA    00452770 f   LIBCMTD:outputp.obj
 0002:0002da80       __output_p_l               00452a80 f   LIBCMTD:outputp.obj
 0002:00032530       _get_crtdouble_arg         00457530 f i LIBCMTD:outputp.obj
 0002:00032560       __output_s_l               00457560 f   LIBCMTD:outputs.obj
 0002:00034050       __woutput_s_l              00459050 f   LIBCMTD:woutputs.obj
 0002:00035850       __validate_param_reuseW    0045a850 f   LIBCMTD:woutputp.obj
 0002:00035b60       __woutput_p_l              0045ab60 f   LIBCMTD:woutputp.obj
 0002:0003a0a0       __mbtowc_l                 0045f0a0 f   LIBCMTD:mbtowc.obj
 0002:0003a340       _mbtowc                    0045f340 f   LIBCMTD:mbtowc.obj
 0002:0003a370       _fputwc                    0045f370 f   LIBCMTD:fputwc.obj
 0002:0003a4b0       __fputwc_nolock            0045f4b0 f   LIBCMTD:fputwc.obj
 0002:0003a860       _putwc                     0045f860 f   LIBCMTD:fputwc.obj
 0002:0003a880       __tolower                  0045f880 f   LIBCMTD:tolower.obj
 0002:0003a890       __tolower_l                0045f890 f   LIBCMTD:tolower.obj
 0002:0003aae0       _tolower                   0045fae0 f   LIBCMTD:tolower.obj
 0002:0003ab40       ___ascii_strnicmp          0045fb40 f   LIBCMTD:_strnicm.obj
 0002:0003abc0       ?_Type_info_dtor@type_info@@CAXPAV1@@Z 0045fbc0 f   LIBCMTD:typname.obj
 0002:0003ad10       ?_Name_base@type_info@@CAPBDPBV1@PAU__type_info_node@@@Z 0045fd10 f   LIBCMTD:typname.obj
 0002:0003af20       ?_Type_info_dtor_internal@type_info@@CAXPAV1@@Z 0045ff20 f   LIBCMTD:typname.obj
 0002:0003b070       ___unDNameHelper           00460070 f   LIBCMTD:typname.obj
 0002:0003b0c0       ?_Name_base_internal@type_info@@CAPBDPBV1@PAU__type_info_node@@@Z 004600c0 f   LIBCMTD:typname.obj
 0002:0003b2f0       ___clean_type_info_names_internal 004602f0 f   LIBCMTD:typname.obj
 0002:0003b3d0       __alloc_osfhnd             004603d0 f   LIBCMTD:osfinfo.obj
 0002:0003b730       __set_osfhnd               00460730 f   LIBCMTD:osfinfo.obj
 0002:0003b830       __free_osfhnd              00460830 f   LIBCMTD:osfinfo.obj
 0002:0003b950       __get_osfhandle            00460950 f   LIBCMTD:osfinfo.obj
 0002:0003bb10       __open_osfhandle           00460b10 f   LIBCMTD:osfinfo.obj
 0002:0003bdd0       ___lock_fhandle            00460dd0 f   LIBCMTD:osfinfo.obj
 0002:0003bf10       __unlock_fhandle           00460f10 f   LIBCMTD:osfinfo.obj
 0002:0003bf50       __putwch                   00460f50 f   LIBCMTD:putwch.obj
 0002:0003c000       __putwch_nolock            00461000 f   LIBCMTD:putwch.obj
 0002:0003c070       __fcloseall                00461070 f   LIBCMTD:closeall.obj
 0002:0003c1f0       _fflush                    004611f0 f   LIBCMTD:fflush.obj
 0002:0003c2b0       __fflush_nolock            004612b0 f   LIBCMTD:fflush.obj
 0002:0003c320       __flush                    00461320 f   LIBCMTD:fflush.obj
 0002:0003c410       __flushall                 00461410 f   LIBCMTD:fflush.obj
 0002:0003c640       __stbuf                    00461640 f   LIBCMTD:_sftbuf.obj
 0002:0003c7f0       __ftbuf                    004617f0 f   LIBCMTD:_sftbuf.obj
 0002:0003c8a0       _vprintf_helper            004618a0 f   LIBCMTD:vprintf.obj
 0002:0003ca00       __vprintf_l                00461a00 f   LIBCMTD:vprintf.obj
 0002:0003ca30       __vprintf_s_l              00461a30 f   LIBCMTD:vprintf.obj
 0002:0003ca60       __vprintf_p_l              00461a60 f   LIBCMTD:vprintf.obj
 0002:0003ca90       _vprintf                   00461a90 f   LIBCMTD:vprintf.obj
 0002:0003cac0       _vprintf_s                 00461ac0 f   LIBCMTD:vprintf.obj
 0002:0003caf0       __vprintf_p                00461af0 f   LIBCMTD:vprintf.obj
 0002:0003cb20       _wcstol                    00461b20 f   LIBCMTD:wcstol.obj
 0002:0003cfe0       __wcstol_l                 00461fe0 f   LIBCMTD:wcstol.obj
 0002:0003d010       _wcstoul                   00462010 f   LIBCMTD:wcstol.obj
 0002:0003d040       __wcstoul_l                00462040 f   LIBCMTD:wcstol.obj
 0002:0003d070       __flswbuf                  00462070 f   LIBCMTD:_flswbuf.obj
 0002:0003d400       ___unDName                 00462400 f   LIBCMTD:undname.obj
 0002:0003d510       ?Constructor@_HeapManager@@QAEXP6APAXI@ZP6AXPAX@Z@Z 00462510 f i LIBCMTD:undname.obj
 0002:0003d560       ?Destructor@_HeapManager@@QAEXXZ 00462560 f i LIBCMTD:undname.obj
 0002:0003d5c0       ___unDNameEx               004625c0 f   LIBCMTD:undname.obj
 0002:0003d6d0       ??0UnDecorator@@QAE@PADPBDHP6APADJ@ZK@Z 004626d0 f i LIBCMTD:undname.obj
 0002:0003d790       ??BUnDecorator@@QAEPADXZ   00462790 f i LIBCMTD:undname.obj
 0002:0003da50       ?dbGetString@DName@@QBEPADXZ 00462a50 f   LIBCMTD:undname.obj
 0002:0003da80       ?getDecoratedName@UnDecorator@@CA?AVDName@@XZ 00462a80 f   LIBCMTD:undname.obj
 0002:0003de60       ?getSymbolName@UnDecorator@@CA?AVDName@@XZ 00462e60 f i LIBCMTD:undname.obj
 0002:0003def0       ?getZName@UnDecorator@@CA?AVDName@@_N0@Z 00462ef0 f   LIBCMTD:undname.obj
 0002:0003e240       ?getOperatorName@UnDecorator@@CA?AVDName@@_NPA_N@Z 00463240 f i LIBCMTD:undname.obj
 0002:0003ee00       ?getStringEncoding@UnDecorator@@CA?AVDName@@PADH@Z 00463e00 f   LIBCMTD:undname.obj
 0002:0003ef40       ?getScope@UnDecorator@@CA?AVDName@@XZ 00463f40 f   LIBCMTD:undname.obj
 0002:0003f410       ?getSignedDimension@UnDecorator@@CA?AVDName@@XZ 00464410 f   LIBCMTD:undname.obj
 0002:0003f4b0       ?getDimension@UnDecorator@@CA?AVDName@@_N@Z 004644b0 f   LIBCMTD:undname.obj
 0002:0003f810       ?getNumberOfDimensions@UnDecorator@@CAHXZ 00464810 f   LIBCMTD:undname.obj
 0002:0003f950       ?getTemplateName@UnDecorator@@CA?AVDName@@_N@Z 00464950 f   LIBCMTD:undname.obj
 0002:0003fb80       ?getTemplateArgumentList@UnDecorator@@CA?AVDName@@XZ 00464b80 f   LIBCMTD:undname.obj
 0002:0003fea0       ?getTemplateConstant@UnDecorator@@CA?AVDName@@XZ 00464ea0 f   LIBCMTD:undname.obj
 0002:00040450       ?composeDeclaration@UnDecorator@@CA?AVDName@@ABV2@@Z 00465450 f i LIBCMTD:undname.obj
 0002:00041fc0       ?getTypeEncoding@UnDecorator@@CAHXZ 00466fc0 f i LIBCMTD:undname.obj
 0002:00042c90       ?getBasedType@UnDecorator@@CA?AVDName@@XZ 00467c90 f   LIBCMTD:undname.obj
 0002:00042d80       ?getScopedName@UnDecorator@@CA?AVDName@@XZ 00467d80 f   LIBCMTD:undname.obj
 0002:00042ee0       ?getCallingConvention@UnDecorator@@CA?AVDName@@XZ 00467ee0 f   LIBCMTD:undname.obj
 0002:000430b0       ?getReturnType@UnDecorator@@CA?AVDName@@PAV2@@Z 004680b0 f   LIBCMTD:undname.obj
 0002:00043110       ?getDataType@UnDecorator@@CA?AVDName@@PAV2@@Z 00468110 f   LIBCMTD:undname.obj
 0002:00043270       ?getPrimaryDataType@UnDecorator@@CA?AVDName@@ABV2@@Z 00468270 f   LIBCMTD:undname.obj
 0002:000436f0       ?getArgumentTypes@UnDecorator@@CA?AVDName@@XZ 004686f0 f   LIBCMTD:undname.obj
 0002:000438a0       ?getArgumentList@UnDecorator@@CA?AVDName@@XZ 004688a0 f   LIBCMTD:undname.obj
 0002:00043a40       ?getThrowTypes@UnDecorator@@CA?AVDName@@XZ 00468a40 f   LIBCMTD:undname.obj
 0002:00043b20       ?getBasicDataType@UnDecorator@@CA?AVDName@@ABV2@@Z 00468b20 f   LIBCMTD:undname.obj
 0002:00044250       ?getECSUDataType@UnDecorator@@CA?AVDName@@XZ 00469250 f   LIBCMTD:undname.obj
 0002:000444a0       ?getECSUName@UnDecorator@@CA?AVDName@@XZ 004694a0 f i LIBCMTD:undname.obj
 0002:000444c0       ?getEnumType@UnDecorator@@CA?AVDName@@XZ 004694c0 f i LIBCMTD:undname.obj
 0002:00044660       ?getFunctionIndirectType@UnDecorator@@CA?AVDName@@ABV2@@Z 00469660 f   LIBCMTD:undname.obj
 0002:00044bb0       ?getPtrRefType@UnDecorator@@CA?AVDName@@ABV2@0PBD@Z 00469bb0 f   LIBCMTD:undname.obj
 0002:00044d70       ?getExtendedDataIndirectType@UnDecorator@@CA?AVDName@@AAPBDAA_NH@Z 00469d70 f   LIBCMTD:undname.obj
 0002:00045020       ?getDataIndirectType@UnDecorator@@CA?AVDName@@ABV2@PBD0H@Z 0046a020 f   LIBCMTD:undname.obj
 0002:000458e0       ?getPtrRefDataType@UnDecorator@@CA?AVDName@@ABV2@H@Z 0046a8e0 f i LIBCMTD:undname.obj
 0002:00045a70       ?getArrayType@UnDecorator@@CA?AVDName@@ABV2@@Z 0046aa70 f i LIBCMTD:undname.obj
 0002:00045d30       ?getLexicalFrame@UnDecorator@@CA?AVDName@@XZ 0046ad30 f i LIBCMTD:undname.obj
 0002:00045d80       ?getThisType@UnDecorator@@CA?AVDName@@XZ 0046ad80 f i LIBCMTD:undname.obj
 0002:00045dd0       ?getPointerType@UnDecorator@@CA?AVDName@@ABV2@0@Z 0046add0 f i LIBCMTD:undname.obj
 0002:00045e10       ?getPointerTypeArray@UnDecorator@@CA?AVDName@@ABV2@0@Z 0046ae10 f i LIBCMTD:undname.obj
 0002:00045e50       ?getReferenceType@UnDecorator@@CA?AVDName@@ABV2@0PBD@Z 0046ae50 f i LIBCMTD:undname.obj
 0002:00045e80       ?getDisplacement@UnDecorator@@CA?AVDName@@XZ 0046ae80 f i LIBCMTD:undname.obj
 0002:00045ea0       ?getCallIndex@UnDecorator@@CA?AVDName@@XZ 0046aea0 f i LIBCMTD:undname.obj
 0002:00045ec0       ?getGuardNumber@UnDecorator@@CA?AVDName@@XZ 0046aec0 f i LIBCMTD:undname.obj
 0002:00045ee0       ?getVbTableType@UnDecorator@@CA?AVDName@@ABV2@@Z 0046aee0 f i LIBCMTD:undname.obj
 0002:00045f00       ?getVCallThunkType@UnDecorator@@CA?AVDName@@XZ 0046af00 f i LIBCMTD:undname.obj
 0002:00045f80       ?getVfTableType@UnDecorator@@CA?AVDName@@ABV2@@Z 0046af80 f i LIBCMTD:undname.obj
 0002:000461b0       ?getStorageConvention@UnDecorator@@CA?AVDName@@XZ 0046b1b0 f i LIBCMTD:undname.obj
 0002:000461d0       ?getDataIndirectType@UnDecorator@@CA?AVDName@@XZ 0046b1d0 f i LIBCMTD:undname.obj
 0002:00046220       ?getVdispMapType@UnDecorator@@CA?AVDName@@ABV2@@Z 0046b220 f i LIBCMTD:undname.obj
 0002:000462b0       ?getExternalDataType@UnDecorator@@CA?AVDName@@ABV2@@Z 0046b2b0 f i LIBCMTD:undname.obj
 0002:00046370       ?doMSKeywords@UnDecorator@@SAHXZ 0046b370 f i LIBCMTD:undname.obj
 0002:00046390       ?doPtr64@UnDecorator@@SAHXZ 0046b390 f i LIBCMTD:undname.obj
 0002:000463b0       ?doFunctionReturns@UnDecorator@@SAHXZ 0046b3b0 f i LIBCMTD:undname.obj
 0002:000463d0       ?doAllocationModel@UnDecorator@@SAHXZ 0046b3d0 f i LIBCMTD:undname.obj
 0002:000463f0       ?doAllocationLanguage@UnDecorator@@SAHXZ 0046b3f0 f i LIBCMTD:undname.obj
 0002:00046410       ?doThisTypes@UnDecorator@@SAHXZ 0046b410 f i LIBCMTD:undname.obj
 0002:00046430       ?doAccessSpecifiers@UnDecorator@@SAHXZ 0046b430 f i LIBCMTD:undname.obj
 0002:00046450       ?doThrowTypes@UnDecorator@@SAHXZ 0046b450 f i LIBCMTD:undname.obj
 0002:00046470       ?doMemberTypes@UnDecorator@@SAHXZ 0046b470 f i LIBCMTD:undname.obj
 0002:00046490       ?doNameOnly@UnDecorator@@SAHXZ 0046b490 f i LIBCMTD:undname.obj
 0002:000464b0       ?doTypeOnly@UnDecorator@@SAHXZ 0046b4b0 f i LIBCMTD:undname.obj
 0002:000464d0       ?haveTemplateParameters@UnDecorator@@SAHXZ 0046b4d0 f i LIBCMTD:undname.obj
 0002:000464f0       ?doEcsu@UnDecorator@@SAHXZ 0046b4f0 f i LIBCMTD:undname.obj
 0002:00046510       ?doEllipsis@UnDecorator@@SAHXZ 0046b510 f i LIBCMTD:undname.obj
 0002:00046530       ?UScore@UnDecorator@@SAPBDW4Tokens@@@Z 0046b530 f   LIBCMTD:undname.obj
 0002:00046570       ?doUnderScore@UnDecorator@@SAHXZ 0046b570 f i LIBCMTD:undname.obj
 0002:00046590       ??2@YAPAXIAAV_HeapManager@@H@Z 0046b590 f i LIBCMTD:undname.obj
 0002:000465b0       ?getMemory@_HeapManager@@QAEPAXIH@Z 0046b5b0 f   LIBCMTD:undname.obj
 0002:00046700       ??0Block@_HeapManager@@QAE@XZ 0046b700 f i LIBCMTD:undname.obj
 0002:00046720       ??H@YA?AVDName@@DABV0@@Z   0046b720 f i LIBCMTD:undname.obj
 0002:00046760       ??H@YA?AVDName@@W4DNameStatus@@ABV0@@Z 0046b760 f i LIBCMTD:undname.obj
 0002:000467a0       ??H@YA?AVDName@@PBDABV0@@Z 0046b7a0 f i LIBCMTD:undname.obj
 0002:000467e0       ??0DName@@QAE@XZ           0046b7e0 f i LIBCMTD:undname.obj
 0002:000468d0       ??0DName@@QAE@D@Z          0046b8d0 f   LIBCMTD:undname.obj
 0002:000469e0       ??0DName@@QAE@ABV0@@Z      0046b9e0 f i LIBCMTD:undname.obj
 0002:00046a10       ??0DName@@QAE@PAV0@@Z      0046ba10 f   LIBCMTD:undname.obj
 0002:00046b90       ??0DName@@QAE@PBD@Z        0046bb90 f   LIBCMTD:undname.obj
 0002:00046cc0       ??0DName@@QAE@AAPBDD@Z     0046bcc0 f   LIBCMTD:undname.obj
 0002:00047030       ?doNoIdentCharCheck@UnDecorator@@SAHXZ 0046c030 f i LIBCMTD:undname.obj
 0002:00047050       ??0DName@@QAE@_K@Z         0046c050 f   LIBCMTD:undname.obj
 0002:000471e0       ??0DName@@QAE@_J@Z         0046c1e0 f   LIBCMTD:undname.obj
 0002:000473c0       ??0DName@@QAE@W4DNameStatus@@@Z 0046c3c0 f   LIBCMTD:undname.obj
 0002:00047520       ?isValid@DName@@QBEHXZ     0046c520 f i LIBCMTD:undname.obj
 0002:00047550       ?isEmpty@DName@@QBEHXZ     0046c550 f i LIBCMTD:undname.obj
 0002:00047570       ?status@DName@@QBE?AW4DNameStatus@@XZ 0046c570 f i LIBCMTD:undname.obj
 0002:00047590       ?setPtrRef@DName@@QAEAAV1@XZ 0046c590 f i LIBCMTD:undname.obj
 0002:000475c0       ?isPtrRef@DName@@QBEHXZ    0046c5c0 f i LIBCMTD:undname.obj
 0002:000475e0       ?isUDC@DName@@QBEHXZ       0046c5e0 f i LIBCMTD:undname.obj
 0002:00047630       ?setIsUDC@DName@@QAEXXZ    0046c630 f i LIBCMTD:undname.obj
 0002:00047670       ?isUDTThunk@DName@@QBEHXZ  0046c670 f i LIBCMTD:undname.obj
 0002:000476c0       ?setIsArray@DName@@QAEXXZ  0046c6c0 f i LIBCMTD:undname.obj
 0002:000476f0       ?isArray@DName@@QBEHXZ     0046c6f0 f i LIBCMTD:undname.obj
 0002:00047710       ?isNoTE@DName@@QBEHXZ      0046c710 f i LIBCMTD:undname.obj
 0002:00047730       ?setIsNoTE@DName@@QAEXXZ   0046c730 f i LIBCMTD:undname.obj
 0002:00047760       ?isPinPtr@DName@@QBEHXZ    0046c760 f i LIBCMTD:undname.obj
 0002:00047780       ?setIsPinPtr@DName@@QAEXXZ 0046c780 f i LIBCMTD:undname.obj
 0002:000477b0       ?isComArray@DName@@QBEHXZ  0046c7b0 f i LIBCMTD:undname.obj
 0002:000477d0       ?setIsComArray@DName@@QAEXXZ 0046c7d0 f i LIBCMTD:undname.obj
 0002:00047800       ?isVCallThunk@DName@@QBEHXZ 0046c800 f i LIBCMTD:undname.obj
 0002:00047820       ?setIsVCallThunk@DName@@QAEXXZ 0046c820 f i LIBCMTD:undname.obj
 0002:00047850       ?length@DName@@QBEHXZ      0046c850 f i LIBCMTD:undname.obj
 0002:00047890       ?getLastChar@DName@@QBEDXZ 0046c890 f i LIBCMTD:undname.obj
 0002:000478d0       ?getString@DName@@QBEPADPADH@Z 0046c8d0 f i LIBCMTD:undname.obj
 0002:00047980       ?getString@DName@@QBEPADPAD0@Z 0046c980 f i LIBCMTD:undname.obj
 0002:000479d0       ??HDName@@QBE?AV0@D@Z      0046c9d0 f   LIBCMTD:undname.obj
 0002:00047a20       ??HDName@@QBE?AV0@PBD@Z    0046ca20 f   LIBCMTD:undname.obj
 0002:00047a70       ??HDName@@QBE?AV0@ABV0@@Z  0046ca70 f   LIBCMTD:undname.obj
 0002:00047ac0       ??HDName@@QBE?AV0@PAV0@@Z  0046cac0 f   LIBCMTD:undname.obj
 0002:00047b10       ??HDName@@QBE?AV0@W4DNameStatus@@@Z 0046cb10 f   LIBCMTD:undname.obj
 0002:00047b60       ?append@DName@@AAEXPAVDNameNode@@@Z 0046cb60 f   LIBCMTD:undname.obj
 0002:00047c10       ??YDName@@QAEAAV0@D@Z      0046cc10 f   LIBCMTD:undname.obj
 0002:00047cc0       ??YDName@@QAEAAV0@PBD@Z    0046ccc0 f   LIBCMTD:undname.obj
 0002:00047d80       ??YDName@@QAEAAV0@ABV0@@Z  0046cd80 f   LIBCMTD:undname.obj
 0002:00047e00       ??YDName@@QAEAAV0@PAV0@@Z  0046ce00 f   LIBCMTD:undname.obj
 0002:00047ee0       ??YDName@@QAEAAV0@W4DNameStatus@@@Z 0046cee0 f   LIBCMTD:undname.obj
 0002:00047f60       ??_5DName@@QAEAAV0@ABV0@@Z 0046cf60 f   LIBCMTD:undname.obj
 0002:00047fd0       ??4DName@@QAEAAV0@D@Z      0046cfd0 f i LIBCMTD:undname.obj
 0002:000480e0       ??4DName@@QAEAAV0@PBD@Z    0046d0e0 f   LIBCMTD:undname.obj
 0002:000481f0       ??4DName@@QAEAAV0@ABV0@@Z  0046d1f0 f   LIBCMTD:undname.obj
 0002:00048220       ??4DName@@QAEAAV0@PAV0@@Z  0046d220 f   LIBCMTD:undname.obj
 0002:000483a0       ??4DName@@QAEAAV0@W4DNameStatus@@@Z 0046d3a0 f   LIBCMTD:undname.obj
 0002:000484e0       ?doPchar@DName@@AAEXPBDH@Z 0046d4e0 f   LIBCMTD:undname.obj
 0002:00048670       ?isFull@Replicator@@QBEHXZ 0046d670 f i LIBCMTD:undname.obj
 0002:00048690       ??0Replicator@@QAE@XZ      0046d690 f i LIBCMTD:undname.obj
 0002:000486b0       ??YReplicator@@QAEAAV0@ABVDName@@@Z 0046d6b0 f   LIBCMTD:undname.obj
 0002:00048760       ??AReplicator@@QBE?AVDName@@H@Z 0046d760 f   LIBCMTD:undname.obj
 0002:000487e0       ??0DNameNode@@IAE@XZ       0046d7e0 f   LIBCMTD:undname.obj
 0002:00048800       ??0charNode@@QAE@D@Z       0046d800 f   LIBCMTD:undname.obj
 0002:00048840       ?length@charNode@@UBEHXZ   0046d840 f i LIBCMTD:undname.obj
 0002:00048860       ?getLastChar@charNode@@UBEDXZ 0046d860 f i LIBCMTD:undname.obj
 0002:00048880       ?getString@charNode@@UBEPADPAD0@Z 0046d880 f i LIBCMTD:undname.obj
 0002:000488c0       ??0pcharNode@@QAE@PBDH@Z   0046d8c0 f   LIBCMTD:undname.obj
 0002:00048980       ?length@pcharNode@@UBEHXZ  0046d980 f i LIBCMTD:undname.obj
 0002:000489a0       ?getLastChar@pcharNode@@UBEDXZ 0046d9a0 f i LIBCMTD:undname.obj
 0002:000489f0       ?getString@pcharNode@@UBEPADPAD0@Z 0046d9f0 f i LIBCMTD:undname.obj
 0002:00048a30       ?getStringHelper@@YAPADPAD00H@Z 0046da30 f i LIBCMTD:undname.obj
 0002:00048a80       ??0pDNameNode@@QAE@PAVDName@@@Z 0046da80 f   LIBCMTD:undname.obj
 0002:00048b00       ?length@pDNameNode@@UBEHXZ 0046db00 f i LIBCMTD:undname.obj
 0002:00048b40       ?getLastChar@pDNameNode@@UBEDXZ 0046db40 f i LIBCMTD:undname.obj
 0002:00048b80       ?getString@pDNameNode@@UBEPADPAD0@Z 0046db80 f i LIBCMTD:undname.obj
 0002:00048bd0       ??0DNameStatusNode@@AAE@W4DNameStatus@@@Z 0046dbd0 f   LIBCMTD:undname.obj
 0002:00048c30       ?length@DNameStatusNode@@UBEHXZ 0046dc30 f i LIBCMTD:undname.obj
 0002:00048c50       ?getLastChar@DNameStatusNode@@UBEDXZ 0046dc50 f i LIBCMTD:undname.obj
 0002:00048c80       ?getString@DNameStatusNode@@UBEPADPAD0@Z 0046dc80 f i LIBCMTD:undname.obj
 0002:00048cd0       ?make@DNameStatusNode@@SAPAV1@W4DNameStatus@@@Z 0046dcd0 f i LIBCMTD:undname.obj
 0002:00048db0       ??0pairNode@@QAE@PAVDNameNode@@0@Z 0046ddb0 f   LIBCMTD:undname.obj
 0002:00048e00       ?length@pairNode@@UBEHXZ   0046de00 f i LIBCMTD:undname.obj
 0002:00048e60       ?getLastChar@pairNode@@UBEDXZ 0046de60 f i LIBCMTD:undname.obj
 0002:00048ec0       ?getString@pairNode@@UBEPADPAD0@Z 0046dec0 f i LIBCMTD:undname.obj
 0002:00049040       ___initconout              0046e040 f   LIBCMTD:initcon.obj
 0002:00049070       ___termconout              0046e070 f   LIBCMTD:initcon.obj
 0002:000490a0       _fclose                    0046e0a0 f   LIBCMTD:fclose.obj
 0002:000491f0       __fclose_nolock            0046e1f0 f   LIBCMTD:fclose.obj
 0002:00049330       __commit                   0046e330 f   LIBCMTD:commit.obj
 0002:000495d0       __wchartodigit             0046e5d0 f   LIBCMTD:wchtodig.obj
 0002:000499c0       __allshl                   0046e9c0 f   LIBCMTD:llshl.obj
 0002:000499f0       __purecall                 0046e9f0 f   LIBCMTD:purevirt.obj
 0002:00049a40       __set_purecall_handler     0046ea40 f   LIBCMTD:purevirt.obj
 0002:00049a80       __get_purecall_handler     0046ea80 f   LIBCMTD:purevirt.obj
 0002:00049aa0       __close                    0046eaa0 f   LIBCMTD:close.obj
 0002:00049d40       __close_nolock             0046ed40 f   LIBCMTD:close.obj
 0002:00049e40       __freebuf                  0046ee40 f   LIBCMTD:_freebuf.obj
 0002:00049ee6       _GetCommandLineA@0         0046eee6 f   kernel32:KERNEL32.dll
 0002:00049eec       _HeapSetInformation@16     0046eeec f   kernel32:KERNEL32.dll
 0002:00049ef2       _GetStartupInfoW@4         0046eef2 f   kernel32:KERNEL32.dll
 0002:00049ef8       _WideCharToMultiByte@32    0046eef8 f   kernel32:KERNEL32.dll
 0002:00049efe       _IsDebuggerPresent@0       0046eefe f   kernel32:KERNEL32.dll
 0002:00049f04       _MultiByteToWideChar@24    0046ef04 f   kernel32:KERNEL32.dll
 0002:00049f0a       _RaiseException@16         0046ef0a f   kernel32:KERNEL32.dll
 0002:00049f10       _lstrlenA@4                0046ef10 f   kernel32:KERNEL32.dll
 0002:00049f16       _GetProcAddress@8          0046ef16 f   kernel32:KERNEL32.dll
 0002:00049f1c       _LoadLibraryW@4            0046ef1c f   kernel32:KERNEL32.dll
 0002:00049f22       _TerminateProcess@8        0046ef22 f   kernel32:KERNEL32.dll
 0002:00049f28       _GetCurrentProcess@0       0046ef28 f   kernel32:KERNEL32.dll
 0002:00049f2e       _UnhandledExceptionFilter@4 0046ef2e f   kernel32:KERNEL32.dll
 0002:00049f34       _SetUnhandledExceptionFilter@4 0046ef34 f   kernel32:KERNEL32.dll
 0002:00049f3a       _QueryPerformanceCounter@4 0046ef3a f   kernel32:KERNEL32.dll
 0002:00049f40       _GetTickCount@0            0046ef40 f   kernel32:KERNEL32.dll
 0002:00049f46       _GetCurrentThreadId@0      0046ef46 f   kernel32:KERNEL32.dll
 0002:00049f4c       _GetCurrentProcessId@0     0046ef4c f   kernel32:KERNEL32.dll
 0002:00049f52       _GetSystemTimeAsFileTime@4 0046ef52 f   kernel32:KERNEL32.dll
 0002:00049f58       _InterlockedIncrement@4    0046ef58 f   kernel32:KERNEL32.dll
 0002:00049f5e       _InterlockedDecrement@4    0046ef5e f   kernel32:KERNEL32.dll
 0002:00049f64       _DecodePointer@4           0046ef64 f   kernel32:KERNEL32.dll
 0002:00049f6a       _GetModuleHandleW@4        0046ef6a f   kernel32:KERNEL32.dll
 0002:00049f70       _ExitProcess@4             0046ef70 f   kernel32:KERNEL32.dll
 0002:00049f76       _GetModuleFileNameA@12     0046ef76 f   kernel32:KERNEL32.dll
 0002:00049f7c       _FreeEnvironmentStringsW@4 0046ef7c f   kernel32:KERNEL32.dll
 0002:00049f82       _GetEnvironmentStringsW@0  0046ef82 f   kernel32:KERNEL32.dll
 0002:00049f88       _SetHandleCount@4          0046ef88 f   kernel32:KERNEL32.dll
 0002:00049f8e       _GetStdHandle@4            0046ef8e f   kernel32:KERNEL32.dll
 0002:00049f94       _InitializeCriticalSectionAndSpinCount@8 0046ef94 f   kernel32:KERNEL32.dll
 0002:00049f9a       _GetFileType@4             0046ef9a f   kernel32:KERNEL32.dll
 0002:00049fa0       _DeleteCriticalSection@4   0046efa0 f   kernel32:KERNEL32.dll
 0002:00049fa6       _HeapValidate@12           0046efa6 f   kernel32:KERNEL32.dll
 0002:00049fac       _IsBadReadPtr@8            0046efac f   kernel32:KERNEL32.dll
 0002:00049fb2       _EncodePointer@4           0046efb2 f   kernel32:KERNEL32.dll
 0002:00049fb8       _TlsAlloc@0                0046efb8 f   kernel32:KERNEL32.dll
 0002:00049fbe       _TlsGetValue@4             0046efbe f   kernel32:KERNEL32.dll
 0002:00049fc4       _TlsSetValue@8             0046efc4 f   kernel32:KERNEL32.dll
 0002:00049fca       _TlsFree@4                 0046efca f   kernel32:KERNEL32.dll
 0002:00049fd0       _SetLastError@4            0046efd0 f   kernel32:KERNEL32.dll
 0002:00049fd6       _GetLastError@0            0046efd6 f   kernel32:KERNEL32.dll
 0002:00049fdc       _GetCurrentThread@0        0046efdc f   kernel32:KERNEL32.dll
 0002:00049fe2       _HeapCreate@12             0046efe2 f   kernel32:KERNEL32.dll
 0002:00049fe8       _HeapDestroy@4             0046efe8 f   kernel32:KERNEL32.dll
 0002:00049fee       _GetModuleFileNameW@12     0046efee f   kernel32:KERNEL32.dll
 0002:00049ff4       _WriteFile@20              0046eff4 f   kernel32:KERNEL32.dll
 0002:00049ffa       _HeapFree@12               0046effa f   kernel32:KERNEL32.dll
 0002:0004a000       _HeapAlloc@12              0046f000 f   kernel32:KERNEL32.dll
 0002:0004a006       _GetProcessHeap@0          0046f006 f   kernel32:KERNEL32.dll
 0002:0004a00c       _VirtualQuery@12           0046f00c f   kernel32:KERNEL32.dll
 0002:0004a012       _FreeLibrary@4             0046f012 f   kernel32:KERNEL32.dll
 0002:0004a018       _RtlUnwind@16              0046f018 f   kernel32:KERNEL32.dll
 0002:0004a01e       _GetACP@0                  0046f01e f   kernel32:KERNEL32.dll
 0002:0004a024       _GetOEMCP@0                0046f024 f   kernel32:KERNEL32.dll
 0002:0004a02a       _GetCPInfo@8               0046f02a f   kernel32:KERNEL32.dll
 0002:0004a030       _IsValidCodePage@4         0046f030 f   kernel32:KERNEL32.dll
 0002:0004a036       _EnterCriticalSection@4    0046f036 f   kernel32:KERNEL32.dll
 0002:0004a03c       _LeaveCriticalSection@4    0046f03c f   kernel32:KERNEL32.dll
 0002:0004a042       _FatalAppExitA@8           0046f042 f   kernel32:KERNEL32.dll
 0002:0004a048       _SetConsoleCtrlHandler@8   0046f048 f   kernel32:KERNEL32.dll
 0002:0004a04e       _InterlockedExchange@8     0046f04e f   kernel32:KERNEL32.dll
 0002:0004a054       _GetLocaleInfoW@16         0046f054 f   kernel32:KERNEL32.dll
 0002:0004a05a       _HeapReAlloc@16            0046f05a f   kernel32:KERNEL32.dll
 0002:0004a060       _HeapSize@12               0046f060 f   kernel32:KERNEL32.dll
 0002:0004a066       _HeapQueryInformation@20   0046f066 f   kernel32:KERNEL32.dll
 0002:0004a06c       _OutputDebugStringA@4      0046f06c f   kernel32:KERNEL32.dll
 0002:0004a072       _WriteConsoleW@20          0046f072 f   kernel32:KERNEL32.dll
 0002:0004a078       _OutputDebugStringW@4      0046f078 f   kernel32:KERNEL32.dll
 0002:0004a07e       _GetStringTypeW@16         0046f07e f   kernel32:KERNEL32.dll
 0002:0004a084       _GetLocaleInfoA@16         0046f084 f   kernel32:KERNEL32.dll
 0002:0004a08a       _IsValidLocale@8           0046f08a f   kernel32:KERNEL32.dll
 0002:0004a090       _EnumSystemLocalesA@8      0046f090 f   kernel32:KERNEL32.dll
 0002:0004a096       _GetUserDefaultLCID@0      0046f096 f   kernel32:KERNEL32.dll
 0002:0004a09c       _LCMapStringW@24           0046f09c f   kernel32:KERNEL32.dll
 0002:0004a0a2       _IsProcessorFeaturePresent@4 0046f0a2 f   kernel32:KERNEL32.dll
 0002:0004a0a8       _SetFilePointer@16         0046f0a8 f   kernel32:KERNEL32.dll
 0002:0004a0ae       _GetConsoleCP@0            0046f0ae f   kernel32:KERNEL32.dll
 0002:0004a0b4       _GetConsoleMode@8          0046f0b4 f   kernel32:KERNEL32.dll
 0002:0004a0ba       _SetStdHandle@8            0046f0ba f   kernel32:KERNEL32.dll
 0002:0004a0c0       _CreateFileW@28            0046f0c0 f   kernel32:KERNEL32.dll
 0002:0004a0c6       _CloseHandle@4             0046f0c6 f   kernel32:KERNEL32.dll
 0002:0004a0cc       _FlushFileBuffers@4        0046f0cc f   kernel32:KERNEL32.dll
 0003:00000000       ___xc_a                    00471000     LIBCMTD:crt0init.obj
 0003:00000104       ___xc_z                    00471104     LIBCMTD:crt0init.obj
 0003:00000208       ___xi_a                    00471208     LIBCMTD:crt0init.obj
 0003:00000524       ___xi_z                    00471524     LIBCMTD:crt0init.obj
 0003:00000628       ___xp_a                    00471628     LIBCMTD:crt0init.obj
 0003:0000093c       ___xp_z                    0047193c     LIBCMTD:crt0init.obj
 0003:00000a40       ___xt_a                    00471a40     LIBCMTD:crt0init.obj
 0003:00000b44       ___xt_z                    00471b44     LIBCMTD:crt0init.obj
 0003:00000c6c       ??_C@_0BD@PFGEINHE@Incorrect?5password?$AA@ 00471c6c     Project1.obj
 0003:00000c84       ??_C@_05NAOIJFC@Error?$AA@ 00471c84     Project1.obj
 0003:00000c8c       ??_C@_0BB@KFINCMHA@Correct?5password?$AA@ 00471c8c     Project1.obj
 0003:00000ca0       ??_C@_0M@EBFEGAAI@Information?$AA@ 00471ca0     Project1.obj
 0003:00000cb0       ??_C@_0M@MGHKIMEF@Test?5marker?$AA@ 00471cb0     Project1.obj
 0003:00000cc0       ??_C@_0BO@GNIAFIKK@Unknown?5Runtime?5Check?5Error?6?$AN?$AA@ 00471cc0     LIBCMTD:_error_.obj
 0003:00000ce4       ??_C@_0CM@NGINOKPC@Stack?5memory?5around?5_alloca?5was?5@ 00471ce4     LIBCMTD:_error_.obj
 0003:00000d18       ??_C@_0DG@HKJMLLLP@A?5local?5variable?5was?5used?5before@ 00471d18     LIBCMTD:_error_.obj
 0003:00000d58       ??_C@_0BN@FFOINMNJ@Stack?5memory?5was?5corrupted?6?$AN?$AA@ 00471d58     LIBCMTD:_error_.obj
 0003:00000d80       ??_C@_0BBN@GPMLNJCF@A?5cast?5to?5a?5smaller?5data?5type?5ha@ 00471d80     LIBCMTD:_error_.obj
 0003:00000ed8       ??_C@_0NN@NGPKDKPD@The?5value?5of?5ESP?5was?5not?5properl@ 00471ed8     LIBCMTD:_error_.obj
 0003:000010a0       ??_C@_0CA@IODNCDPG@Run?9Time?5Check?5Failure?5?$CD?$CFd?5?9?5?$CFs?$AA@ 004720a0     LIBCMTD:_error_.obj
 0003:000010c8       ??_C@_0BE@GNBOBNCK@Unknown?5Module?5Name?$AA@ 004720c8     LIBCMTD:_error_.obj
 0003:000010e0       ??_C@_0BB@PFFGGCJP@Unknown?5Filename?$AA@ 004720e0     LIBCMTD:_error_.obj
 0003:000010f8       ??_C@_1EA@NFKNIFJP@?$AAR?$AAu?$AAn?$AA?9?$AAT?$AAi?$AAm?$AAe?$AA?5?$AAC?$AAh?$AAe?$AAc?$AAk?$AA?5?$AAF?$AAa?$AAi?$AAl?$AAu?$AAr?$AAe?$AA?5?$AA?$CD?$AA?$CF?$AAd?$AA?5?$AA?9?$AA?5?$AA?$CF?$AAs?$AA?$AA@ 004720f8     LIBCMTD:_error_.obj
 0003:00001148       ??_C@_1GM@OLMCBDMB@?$AAR?$AAu?$AAn?$AAt?$AAi?$AAm?$AAe?$AA?5?$AAC?$AAh?$AAe?$AAc?$AAk?$AA?5?$AAE?$AAr?$AAr?$AAo?$AAr?$AA?4?$AA?6?$AA?$AN?$AA?5?$AAU?$AAn?$AAa?$AAb?$AAl?$AAe?$AA?5?$AAt?$AAo@ 00472148     LIBCMTD:_error_.obj
 0003:000011cc       ??_C@_0CG@IAFNJNEE@Stack?5corrupted?5near?5unknown?5var@ 004721cc     LIBCMTD:_error_.obj
 0003:00001200       ??_C@_0EJ@LJKNEOLN@Stack?5area?5around?5_alloca?5memory@ 00472200     LIBCMTD:_error_.obj
 0003:00001258       ??_C@_08KJEDNCKC@?$CFs?$CFs?$CFs?$CFs?$AA@ 00472258     LIBCMTD:_error_.obj
 0003:00001264       ??_C@_02LLMPMKNF@?$DO?5?$AA@ 00472264     LIBCMTD:_error_.obj
 0003:00001268       ??_C@_01EEMJAFIK@?6?$AA@   00472268     LIBCMTD:_error_.obj
 0003:0000126c       ??_C@_0BC@KIBAILCI@?$CFs?$CFs?$CFp?$CFs?$CFld?$CFs?$CFd?$CFs?$AA@ 0047226c     LIBCMTD:_error_.obj
 0003:00001288       ??_C@_0EI@CLEPFNGI@Stack?5area?5around?5_alloca?5memory@ 00472288     LIBCMTD:_error_.obj
 0003:000012e0       ??_C@_0N@MHFFIMFG@?6Address?3?50x?$AA@ 004722e0     LIBCMTD:_error_.obj
 0003:000012f0       ??_C@_07DFDJCKFN@?6Size?3?5?$AA@ 004722f0     LIBCMTD:_error_.obj
 0003:000012fc       ??_C@_0CK@DKGBICFE@?6Allocation?5number?5within?5this?5f@ 004722fc     LIBCMTD:_error_.obj
 0003:00001330       ??_C@_08OMAHNMHJ@?6Data?3?5?$DM?$AA@ 00472330     LIBCMTD:_error_.obj
 0003:0000133c       ??_C@_09FOPFMPEJ@wsprintfA?$AA@ 0047233c     LIBCMTD:_error_.obj
 0003:00001348       ??_C@_1BG@OILDLIOJ@?$AAu?$AAs?$AAe?$AAr?$AA3?$AA2?$AA?4?$AAd?$AAl?$AAl?$AA?$AA@ 00472348     LIBCMTD:_error_.obj
 0003:00001364       ??_C@_05MKKEDADM@?$CF?42X?5?$AA@ 00472364     LIBCMTD:_error_.obj
 0003:0000136c       ??_C@_0DE@OHJBPMBP@A?5variable?5is?5being?5used?5without@ 0047236c     LIBCMTD:_error_.obj
 0003:000013ac       ??_C@_0BP@OGBCLIBO@Stack?5around?5_alloca?5corrupted?$AA@ 004723ac     LIBCMTD:_userapi_.obj
 0003:000013d4       ??_C@_0CK@CNLNOEPB@Local?5variable?5used?5before?5initi@ 004723d4     LIBCMTD:_userapi_.obj
 0003:00001408       ??_C@_0BI@CIGMDCBH@Stack?5memory?5corruption?$AA@ 00472408     LIBCMTD:_userapi_.obj
 0003:00001424       ??_C@_0CK@FEGOIOPB@Cast?5to?5smaller?5type?5causing?5los@ 00472424     LIBCMTD:_userapi_.obj
 0003:00001458       ??_C@_0BJ@HEGAHDFO@Stack?5pointer?5corruption?$AA@ 00472458     LIBCMTD:_userapi_.obj
 0003:00001490       ??_C@_0DP@CBBAPGOP@f?3?2dd?2vctools?2crt_bld?2self_x86?2c@ 00472490     LIBCMTD:chkesp.obj
 0003:000014db       ??_C@_00CNPNBAHC@?$AA@     004724db     LIBCMTD:chkesp.obj
 0003:000014e0       ??_C@_0NM@DNEDKLDF@The?5value?5of?5ESP?5was?5not?5properl@ 004724e0     LIBCMTD:chkesp.obj
 0003:000015e8       ?ProcessDetach@NativeDll@<CrtImplementationDetails>@@0IB 004725e8     LIBCMTD:strtol.obj
 0003:000015ec       ?ProcessAttach@NativeDll@<CrtImplementationDetails>@@0IB 004725ec     LIBCMTD:strtol.obj
 0003:000015f0       ?ThreadAttach@NativeDll@<CrtImplementationDetails>@@0IB 004725f0     LIBCMTD:strtol.obj
 0003:000015f4       ?ThreadDetach@NativeDll@<CrtImplementationDetails>@@0IB 004725f4     LIBCMTD:strtol.obj
 0003:000015f8       ?ProcessVerifier@NativeDll@<CrtImplementationDetails>@@0IB 004725f8     LIBCMTD:strtol.obj
 0003:00001600       ??_C@_1FE@CEHLKAHD@?$AAi?$AAb?$AAa?$AAs?$AAe?$AA?5?$AA?$DN?$AA?$DN?$AA?5?$AA0?$AA?5?$AA?$HM?$AA?$HM?$AA?5?$AA?$CI?$AA2?$AA?5?$AA?$DM?$AA?$DN?$AA?5?$AAi?$AAb?$AAa?$AAs?$AAe?$AA?5?$AA?$CG?$AA?$CG?$AA?5?$AAi?$AAb?$AAa@ 00472600     LIBCMTD:strtol.obj
 0003:00001664       ??_C@_1BA@LOLAMAJG@?$AAs?$AAt?$AAr?$AAt?$AAo?$AAx?$AAl?$AA?$AA@ 00472664     LIBCMTD:strtol.obj
 0003:00001678       ??_C@_1GA@IPHKKOEI@?$AAf?$AA?3?$AA?2?$AAd?$AAd?$AA?2?$AAv?$AAc?$AAt?$AAo?$AAo?$AAl?$AAs?$AA?2?$AAc?$AAr?$AAt?$AA_?$AAb?$AAl?$AAd?$AA?2?$AAs?$AAe?$AAl?$AAf?$AA_?$AAx?$AA8?$AA6?$AA?2?$AAc@ 00472678     LIBCMTD:strtol.obj
 0003:000016ec       ??_C@_1BK@LAOAACLJ@?$AAn?$AAp?$AAt?$AAr?$AA?5?$AA?$CB?$AA?$DN?$AA?5?$AAN?$AAU?$AAL?$AAL?$AA?$AA@ 004726ec     LIBCMTD:strtol.obj
 0003:0000170c       ??_C@_1BA@BMMDEPNE@?$AAs?$AAt?$AAr?$AAt?$AAo?$AAx?$AAq?$AA?$AA@ 0047270c     LIBCMTD:strtoq.obj
 0003:00001720       ??_C@_1GA@GIMEIKLC@?$AAf?$AA?3?$AA?2?$AAd?$AAd?$AA?2?$AAv?$AAc?$AAt?$AAo?$AAo?$AAl?$AAs?$AA?2?$AAc?$AAr?$AAt?$AA_?$AAb?$AAl?$AAd?$AA?2?$AAs?$AAe?$AAl?$AAf?$AA_?$AAx?$AA8?$AA6?$AA?2?$AAc@ 00472720     LIBCMTD:strtoq.obj
 0003:000017a0       ??_C@_0P@MIGLKIOC@CorExitProcess?$AA@ 004727a0     LIBCMTD:crt0dat.obj
 0003:000017b4       ??_C@_1BI@BGOHAHKC@?$AAm?$AAs?$AAc?$AAo?$AAr?$AAe?$AAe?$AA?4?$AAd?$AAl?$AAl?$AA?$AA@ 004727b4     LIBCMTD:crt0dat.obj
 0003:000017d0       ??_C@_1CC@CDIPMFPD@?$AA_?$AAw?$AAp?$AAg?$AAm?$AAp?$AAt?$AAr?$AA?5?$AA?$CB?$AA?$DN?$AA?5?$AAN?$AAU?$AAL?$AAL?$AA?$AA@ 004727d0     LIBCMTD:crt0dat.obj
 0003:000017f8       ??_C@_1BK@PNLDCCDP@?$AA_?$AAg?$AAe?$AAt?$AA_?$AAw?$AAp?$AAg?$AAm?$AAp?$AAt?$AAr?$AA?$AA@ 004727f8     LIBCMTD:crt0dat.obj
 0003:00001818       ??_C@_1GC@DGCPEDNJ@?$AAf?$AA?3?$AA?2?$AAd?$AAd?$AA?2?$AAv?$AAc?$AAt?$AAo?$AAo?$AAl?$AAs?$AA?2?$AAc?$AAr?$AAt?$AA_?$AAb?$AAl?$AAd?$AA?2?$AAs?$AAe?$AAl?$AAf?$AA_?$AAx?$AA8?$AA6?$AA?2?$AAc@ 00472818     LIBCMTD:crt0dat.obj
 0003:00001890       ??_C@_1BO@LKEBEKJP@?$AAp?$AAV?$AAa?$AAl?$AAu?$AAe?$AA?5?$AA?$CB?$AA?$DN?$AA?5?$AAN?$AAU?$AAL?$AAL?$AA?$AA@ 00472890     LIBCMTD:crt0dat.obj
 0003:000018b4       ??_C@_1CA@BBNAFCKO@?$AA_?$AAp?$AAg?$AAm?$AAp?$AAt?$AAr?$AA?5?$AA?$CB?$AA?$DN?$AA?5?$AAN?$AAU?$AAL?$AAL?$AA?$AA@ 004728b4     LIBCMTD:crt0dat.obj
 0003:000018dc       ??_C@_1BI@COAAPHJK@?$AA_?$AAg?$AAe?$AAt?$AA_?$AAp?$AAg?$AAm?$AAp?$AAt?$AAr?$AA?$AA@ 004728dc     LIBCMTD:crt0dat.obj
 0003:000018f8       __XcptActTab               004728f8     LIBCMTD:winxfltr.obj
 0003:00001988       __First_FPE_Indx           00472988     LIBCMTD:winxfltr.obj
 0003:0000198c       __Num_FPE                  0047298c     LIBCMTD:winxfltr.obj
 0003:00001990       __XcptActTabSize           00472990     LIBCMTD:winxfltr.obj
 0003:00001994       __XcptActTabCount          00472994     LIBCMTD:winxfltr.obj
 0003:000019b8       ??_C@_1DE@MMOGFGHF@?$AAs?$AAt?$AAr?$AAc?$AAp?$AAy?$AA_?$AAs?$AA?$CI?$AA?$CK?$AAe?$AAn?$AAv?$AA?0?$AA?5?$AAc?$AAc?$AAh?$AAa?$AAr?$AAs?$AA?0?$AA?5?$AAp?$AA?$CJ?$AA?$AA@ 004729b8     LIBCMTD:stdenvp.obj
 0003:000019f8       ??_C@_1BC@GHMCNHHL@?$AA_?$AAs?$AAe?$AAt?$AAe?$AAn?$AAv?$AAp?$AA?$AA@ 004729f8     LIBCMTD:stdenvp.obj
 0003:00001a10       ??_C@_1GC@DGBFLDBN@?$AAf?$AA?3?$AA?2?$AAd?$AAd?$AA?2?$AAv?$AAc?$AAt?$AAo?$AAo?$AAl?$AAs?$AA?2?$AAc?$AAr?$AAt?$AA_?$AAb?$AAl?$AAd?$AA?2?$AAs?$AAe?$AAl?$AAf?$AA_?$AAx?$AA8?$AA6?$AA?2?$AAc@ 00472a10     LIBCMTD:stdenvp.obj
 0003:00001a88       ??_C@_0DB@BMEBJJKP@f?3?2dd?2vctools?2crt_bld?2self_x86?2c@ 00472a88     LIBCMTD:stdenvp.obj
 0003:00001ac4       ??_C@_0DB@OEPBJOLC@f?3?2dd?2vctools?2crt_bld?2self_x86?2c@ 00472ac4     LIBCMTD:stdargv.obj
 0003:00001b00       ??_C@_0CP@PPLBCJDN@f?3?2dd?2vctools?2crt_bld?2self_x86?2c@ 00472b00     LIBCMTD:a_env.obj
 0003:00001b38       ??_C@_0DA@NBLAKPEL@f?3?2dd?2vctools?2crt_bld?2self_x86?2c@ 00472b38     LIBCMTD:ioinit.obj
 0003:00001b74       ??_C@_06PJIGMIJB@Client?$AA@ 00472b74     LIBCMTD:dbgheap.obj
 0003:00001b7c       ??_C@_06KMEJCCGM@Ignore?$AA@ 00472b7c     LIBCMTD:dbgheap.obj
 0003:00001b84       ??_C@_03OGPFLFLO@CRT?$AA@  00472b84     LIBCMTD:dbgheap.obj
 0003:00001b88       ??_C@_06EFAGIKOH@Normal?$AA@ 00472b88     LIBCMTD:dbgheap.obj
 0003:00001b90       ??_C@_04HJMOFLDF@Free?$AA@ 00472b90     LIBCMTD:dbgheap.obj
 0003:00001bb0       ??_C@_0DC@JEMAGEKG@Error?3?5memory?5allocation?3?5bad?5me@ 00472bb0     LIBCMTD:dbgheap.obj
 0003:00001bec       ??_C@_0CF@BICKFLAF@Invalid?5allocation?5size?3?5?$CFIu?5byt@ 00472bec     LIBCMTD:dbgheap.obj
 0003:00001c18       ??_C@_02DKCKIIND@?$CFs?$AA@ 00472c18     LIBCMTD:dbgheap.obj
 0003:00001c1c       ??_C@_0CB@CCLOLAHO@Client?5hook?5allocation?5failure?4?6@ 00472c1c     LIBCMTD:dbgheap.obj
 0003:00001c44       ??_C@_0DF@BBEGIFEK@Client?5hook?5allocation?5failure?5a@ 00472c44     LIBCMTD:dbgheap.obj
 0003:00001c88       ??_C@_1GC@DNJKKEAA@?$AAf?$AA?3?$AA?2?$AAd?$AAd?$AA?2?$AAv?$AAc?$AAt?$AAo?$AAo?$AAl?$AAs?$AA?2?$AAc?$AAr?$AAt?$AA_?$AAb?$AAl?$AAd?$AA?2?$AAs?$AAe?$AAl?$AAf?$AA_?$AAx?$AA8?$AA6?$AA?2?$AAc@ 00472c88     LIBCMTD:dbgheap.obj
 0003:00001d00       ??_C@_1CE@LJFEPPMP@?$AA_?$AAC?$AAr?$AAt?$AAC?$AAh?$AAe?$AAc?$AAk?$AAM?$AAe?$AAm?$AAo?$AAr?$AAy?$AA?$CI?$AA?$CJ?$AA?$AA@ 00472d00     LIBCMTD:dbgheap.obj
 0003:00001d2c       ??_C@_1DE@KOOKLFBB@?$AA_?$AAp?$AAF?$AAi?$AAr?$AAs?$AAt?$AAB?$AAl?$AAo?$AAc?$AAk?$AA?5?$AA?$DN?$AA?$DN?$AA?5?$AAp?$AAO?$AAl?$AAd?$AAB?$AAl?$AAo?$AAc?$AAk?$AA?$AA@ 00472d2c     LIBCMTD:dbgheap.obj
 0003:00001d6c       ??_C@_1DC@GEFKNOOL@?$AA_?$AAp?$AAL?$AAa?$AAs?$AAt?$AAB?$AAl?$AAo?$AAc?$AAk?$AA?5?$AA?$DN?$AA?$DN?$AA?5?$AAp?$AAO?$AAl?$AAd?$AAB?$AAl?$AAo?$AAc?$AAk?$AA?$AA@ 00472d6c     LIBCMTD:dbgheap.obj
 0003:00001da8       ??_C@_1GE@PCKLOLAO@?$AAf?$AAR?$AAe?$AAa?$AAl?$AAl?$AAo?$AAc?$AA?5?$AA?$HM?$AA?$HM?$AA?5?$AA?$CI?$AA?$CB?$AAf?$AAR?$AAe?$AAa?$AAl?$AAl?$AAo?$AAc?$AA?5?$AA?$CG?$AA?$CG?$AA?5?$AAp?$AAN?$AAe?$AAw?$AAB?$AAl@ 00472da8     LIBCMTD:dbgheap.obj
 0003:00001e20       ??_C@_0DA@HFBKENN@Error?3?5possible?5heap?5corruption?5@ 00472e20     LIBCMTD:dbgheap.obj
 0003:00001e60       ??_C@_1IK@DCPKDGNH@?$AAp?$AAO?$AAl?$AAd?$AAB?$AAl?$AAo?$AAc?$AAk?$AA?9?$AA?$DO?$AAn?$AAL?$AAi?$AAn?$AAe?$AA?5?$AA?$DN?$AA?$DN?$AA?5?$AAI?$AAG?$AAN?$AAO?$AAR?$AAE?$AA_?$AAL?$AAI?$AAN?$AAE?$AA?5@ 00472e60     LIBCMTD:dbgheap.obj
 0003:00001f08       ??_C@_1EE@GFOPCECE@?$AA_?$AAC?$AAr?$AAt?$AAI?$AAs?$AAV?$AAa?$AAl?$AAi?$AAd?$AAH?$AAe?$AAa?$AAp?$AAP?$AAo?$AAi?$AAn?$AAt?$AAe?$AAr?$AA?$CI?$AAp?$AAU?$AAs?$AAe?$AAr?$AAD?$AAa?$AAt?$AAa@ 00472f08     LIBCMTD:dbgheap.obj
 0003:00001f60       ??_C@_0EM@LGFLMAGJ@The?5Block?5at?50x?$CFp?5was?5allocated?5@ 00472f60     LIBCMTD:dbgheap.obj
 0003:00001fc0       ??_C@_0FA@EFEIGJKG@Error?3?5memory?5allocation?3?5bad?5me@ 00472fc0     LIBCMTD:dbgheap.obj
 0003:00002020       ??_C@_0ED@GPCPBAGP@Invalid?5allocation?5size?3?5?$CFIu?5byt@ 00473020     LIBCMTD:dbgheap.obj
 0003:00002070       ??_C@_0CE@DOFMDOL@Client?5hook?5re?9allocation?5failur@ 00473070     LIBCMTD:dbgheap.obj
 0003:0000209c       ??_C@_0DI@KKJPDPGM@Client?5hook?5re?9allocation?5failur@ 0047309c     LIBCMTD:dbgheap.obj
 0003:000020e0       ??_C@_1BI@HAPNGHDP@?$AA_?$AAe?$AAx?$AAp?$AAa?$AAn?$AAd?$AA_?$AAd?$AAb?$AAg?$AA?$AA@ 004730e0     LIBCMTD:dbgheap.obj
 0003:000020fc       ??_C@_1CE@CJACEFBA@?$AAp?$AAU?$AAs?$AAe?$AAr?$AAD?$AAa?$AAt?$AAa?$AA?5?$AA?$CB?$AA?$DN?$AA?5?$AAN?$AAU?$AAL?$AAL?$AA?$AA@ 004730fc     LIBCMTD:dbgheap.obj
 0003:00002128       ??_C@_1CM@MMAADDMD@?$AA_?$AAp?$AAF?$AAi?$AAr?$AAs?$AAt?$AAB?$AAl?$AAo?$AAc?$AAk?$AA?5?$AA?$DN?$AA?$DN?$AA?5?$AAp?$AAH?$AAe?$AAa?$AAd?$AA?$AA@ 00473128     LIBCMTD:dbgheap.obj
 0003:0000215c       ??_C@_1CK@DMAGEMBG@?$AA_?$AAp?$AAL?$AAa?$AAs?$AAt?$AAB?$AAl?$AAo?$AAc?$AAk?$AA?5?$AA?$DN?$AA?$DN?$AA?5?$AAp?$AAH?$AAe?$AAa?$AAd?$AA?$AA@ 0047315c     LIBCMTD:dbgheap.obj
 0003:00002190       ??_C@_1DM@ODCJIDCP@?$AAp?$AAH?$AAe?$AAa?$AAd?$AA?9?$AA?$DO?$AAn?$AAB?$AAl?$AAo?$AAc?$AAk?$AAU?$AAs?$AAe?$AA?5?$AA?$DN?$AA?$DN?$AA?5?$AAn?$AAB?$AAl?$AAo?$AAc?$AAk?$AAU?$AAs?$AAe?$AA?$AA@ 00473190     LIBCMTD:dbgheap.obj
 0003:000021d8       ??_C@_1HK@HPCBMDFG@?$AAp?$AAH?$AAe?$AAa?$AAd?$AA?9?$AA?$DO?$AAn?$AAL?$AAi?$AAn?$AAe?$AA?5?$AA?$DN?$AA?$DN?$AA?5?$AAI?$AAG?$AAN?$AAO?$AAR?$AAE?$AA_?$AAL?$AAI?$AAN?$AAE?$AA?5?$AA?$CG?$AA?$CG?$AA?5?$AAp@ 004731d8     LIBCMTD:dbgheap.obj
 0003:00002270       ??_C@_0IG@LEMBDCJK@HEAP?5CORRUPTION?5DETECTED?3?5after?5@ 00473270     LIBCMTD:dbgheap.obj
 0003:00002310       ??_C@_0KE@MBMNHHHN@HEAP?5CORRUPTION?5DETECTED?3?5after?5@ 00473310     LIBCMTD:dbgheap.obj
 0003:000023d8       ??_C@_0IK@PJCGLBOB@HEAP?5CORRUPTION?5DETECTED?3?5before@ 004733d8     LIBCMTD:dbgheap.obj
 0003:00002480       ??_C@_0KI@JGFOHMEB@HEAP?5CORRUPTION?5DETECTED?3?5before@ 00473480     LIBCMTD:dbgheap.obj
 0003:00002550       ??_C@_1EO@LHDAJOCM@?$AA_?$AAB?$AAL?$AAO?$AAC?$AAK?$AA_?$AAT?$AAY?$AAP?$AAE?$AA_?$AAI?$AAS?$AA_?$AAV?$AAA?$AAL?$AAI?$AAD?$AA?$CI?$AAp?$AAH?$AAe?$AAa?$AAd?$AA?9?$AA?$DO?$AAn?$AAB?$AAl?$AAo@ 00473550     LIBCMTD:dbgheap.obj
 0003:000025b0       ??_C@_0BL@KEIPLFAC@Client?5hook?5free?5failure?4?6?$AA@ 004735b0     LIBCMTD:dbgheap.obj
 0003:000025d0       ??_C@_0EJ@HEIBCIMJ@The?5Block?5at?50x?$CFp?5was?5allocated?5@ 004735d0     LIBCMTD:dbgheap.obj
 0003:00002628       ??_C@_1BG@MBKOGDLD@?$AA_?$AAm?$AAs?$AAi?$AAz?$AAe?$AA_?$AAd?$AAb?$AAg?$AA?$AA@ 00473628     LIBCMTD:dbgheap.obj
 0003:00002644       ??_C@_0CI@JMLBEDHJ@?$CFhs?5located?5at?50x?$CFp?5is?5?$CFIu?5bytes@ 00473644     LIBCMTD:dbgheap.obj
 0003:00002678       ??_C@_0EG@DGJMPDBH@?$CFhs?5located?5at?50x?$CFp?5is?5?$CFIu?5bytes@ 00473678     LIBCMTD:dbgheap.obj
 0003:000026d0       ??_C@_0IC@BBJIOOJH@HEAP?5CORRUPTION?5DETECTED?3?5on?5top@ 004736d0     LIBCMTD:dbgheap.obj
 0003:00002770       ??_C@_0KA@IHNJJKPL@HEAP?5CORRUPTION?5DETECTED?3?5on?5top@ 00473770     LIBCMTD:dbgheap.obj
 0003:00002830       ??_C@_07OHKEFPKJ@DAMAGED?$AA@ 00473830     LIBCMTD:dbgheap.obj
 0003:0000283c       ??_C@_0CL@HNNNMKMJ@_heapchk?5fails?5with?5unknown?5retu@ 0047383c     LIBCMTD:dbgheap.obj
 0003:00002870       ??_C@_0CC@MFFCHFHO@_heapchk?5fails?5with?5_HEAPBADPTR?4@ 00473870     LIBCMTD:dbgheap.obj
 0003:00002898       ??_C@_0CC@MJGLGBDG@_heapchk?5fails?5with?5_HEAPBADEND?4@ 00473898     LIBCMTD:dbgheap.obj
 0003:000028c0       ??_C@_0CD@CPKEAPBD@_heapchk?5fails?5with?5_HEAPBADNODE@ 004738c0     LIBCMTD:dbgheap.obj
 0003:000028ec       ??_C@_0CE@MKKHMBMK@_heapchk?5fails?5with?5_HEAPBADBEGI@ 004738ec     LIBCMTD:dbgheap.obj
 0003:00002918       ??_C@_1BO@GJFDNMNF@?$AA_?$AAC?$AAr?$AAt?$AAS?$AAe?$AAt?$AAD?$AAb?$AAg?$AAF?$AAl?$AAa?$AAg?$AA?$AA@ 00473918     LIBCMTD:dbgheap.obj
 0003:00002940       ??_C@_1BHO@NNANJNF@?$AA?$CI?$AAf?$AAN?$AAe?$AAw?$AAB?$AAi?$AAt?$AAs?$AA?$DN?$AA?$DN?$AA_?$AAC?$AAR?$AAT?$AAD?$AAB?$AAG?$AA_?$AAR?$AAE?$AAP?$AAO?$AAR?$AAT?$AA_?$AAF?$AAL?$AAA?$AAG?$AA?$CJ?$AA?5@ 00473940     LIBCMTD:dbgheap.obj
 0003:00002b0c       ??_C@_1DE@GJCKCKEC@?$AA_?$AAC?$AAr?$AAt?$AAD?$AAo?$AAF?$AAo?$AAr?$AAA?$AAl?$AAl?$AAC?$AAl?$AAi?$AAe?$AAn?$AAt?$AAO?$AAb?$AAj?$AAe?$AAc?$AAt?$AAs?$AA?$AA@ 00473b0c     LIBCMTD:dbgheap.obj
 0003:00002b4c       ??_C@_1BI@CJGCEEDL@?$AAp?$AAf?$AAn?$AA?5?$AA?$CB?$AA?$DN?$AA?5?$AAN?$AAU?$AAL?$AAL?$AA?$AA@ 00473b4c     LIBCMTD:dbgheap.obj
 0003:00002b68       ??_C@_0CB@EAAIGELO@Bad?5memory?5block?5found?5at?50x?$CFp?4?6@ 00473b68     LIBCMTD:dbgheap.obj
 0003:00002b90       ??_C@_0DP@LEFMFBOD@Bad?5memory?5block?5found?5at?50x?$CFp?4?6@ 00473b90     LIBCMTD:dbgheap.obj
 0003:00002bdc       ??_C@_1CE@NJJKELF@?$AA_?$AAC?$AAr?$AAt?$AAM?$AAe?$AAm?$AAC?$AAh?$AAe?$AAc?$AAk?$AAp?$AAo?$AAi?$AAn?$AAt?$AA?$AA@ 00473bdc     LIBCMTD:dbgheap.obj
 0003:00002c08       ??_C@_1BM@MIMANDHC@?$AAs?$AAt?$AAa?$AAt?$AAe?$AA?5?$AA?$CB?$AA?$DN?$AA?5?$AAN?$AAU?$AAL?$AAL?$AA?$AA@ 00473c08     LIBCMTD:dbgheap.obj
 0003:00002c2c       ??_C@_1CC@DFPEDFBP@?$AAn?$AAe?$AAw?$AAS?$AAt?$AAa?$AAt?$AAe?$AA?5?$AA?$CB?$AA?$DN?$AA?5?$AAN?$AAU?$AAL?$AAL?$AA?$AA@ 00473c2c     LIBCMTD:dbgheap.obj
 0003:00002c54       ??_C@_1CC@DHPFEMMN@?$AAo?$AAl?$AAd?$AAS?$AAt?$AAa?$AAt?$AAe?$AA?5?$AA?$CB?$AA?$DN?$AA?5?$AAN?$AAU?$AAL?$AAL?$AA?$AA@ 00473c54     LIBCMTD:dbgheap.obj
 0003:00002c7c       ??_C@_1CE@PDIENACM@?$AA_?$AAC?$AAr?$AAt?$AAM?$AAe?$AAm?$AAD?$AAi?$AAf?$AAf?$AAe?$AAr?$AAe?$AAn?$AAc?$AAe?$AA?$AA@ 00473c7c     LIBCMTD:dbgheap.obj
 0003:00002ca8       ??_C@_0BH@GFGKJDCO@Object?5dump?5complete?4?6?$AA@ 00473ca8     LIBCMTD:dbgheap.obj
 0003:00002cc4       ??_C@_0DA@MDLBNIBM@crt?5block?5at?50x?$CFp?0?5subtype?5?$CFx?0?5?$CF@ 00473cc4     LIBCMTD:dbgheap.obj
 0003:00002d00       ??_C@_0CH@FAGDDGPN@normal?5block?5at?50x?$CFp?0?5?$CFIu?5bytes?5@ 00473d00     LIBCMTD:dbgheap.obj
 0003:00002d30       ??_C@_0DD@GHNAAKBB@client?5block?5at?50x?$CFp?0?5subtype?5?$CFx@ 00473d30     LIBCMTD:dbgheap.obj
 0003:00002d70       ??_C@_06PKLGBFGM@?$HL?$CFld?$HN?5?$AA@ 00473d70     LIBCMTD:dbgheap.obj
 0003:00002d78       ??_C@_0L@JMEFFCCJ@?$CFhs?$CI?$CFd?$CJ?5?3?5?$AA@ 00473d78     LIBCMTD:dbgheap.obj
 0003:00002d88       ??_C@_0BE@OIEFNFL@?$CDFile?5Error?$CD?$CI?$CFd?$CJ?5?3?5?$AA@ 00473d88     LIBCMTD:dbgheap.obj
 0003:00002da0       ??_C@_0BE@KCIPKCIA@Dumping?5objects?5?9?$DO?6?$AA@ 00473da0     LIBCMTD:dbgheap.obj
 0003:00002db8       ??_C@_0BA@HJBKCELP@?5Data?3?5?$DM?$CFs?$DO?5?$CFs?6?$AA@ 00473db8     LIBCMTD:dbgheap.obj
 0003:00002dcc       ??_C@_1BI@KALLJECN@?$AA?$CI?$AA?$CK?$AA_?$AAe?$AAr?$AAr?$AAn?$AAo?$AA?$CI?$AA?$CJ?$AA?$CJ?$AA?$AA@ 00473dcc     LIBCMTD:dbgheap.obj
 0003:00002de8       ??_C@_1CG@LPFIACGM@?$AA_?$AAp?$AAr?$AAi?$AAn?$AAt?$AAM?$AAe?$AAm?$AAB?$AAl?$AAo?$AAc?$AAk?$AAD?$AAa?$AAt?$AAa?$AA?$AA@ 00473de8     LIBCMTD:dbgheap.obj
 0003:00002e18       ??_C@_0BI@JBFPOEJA@Detected?5memory?5leaks?$CB?6?$AA@ 00473e18     LIBCMTD:dbgheap.obj
 0003:00002e34       ??_C@_0BP@DEDHGGGI@Total?5allocations?3?5?$CFId?5bytes?4?6?$AA@ 00473e34     LIBCMTD:dbgheap.obj
 0003:00002e5c       ??_C@_0CB@BLHDAFNE@Largest?5number?5used?3?5?$CFId?5bytes?4?6@ 00473e5c     LIBCMTD:dbgheap.obj
 0003:00002e84       ??_C@_0BO@DACNIABB@?$CFId?5bytes?5in?5?$CFId?5?$CFhs?5Blocks?4?6?$AA@ 00473e84     LIBCMTD:dbgheap.obj
 0003:00002ea8       ??_C@_1CM@MPNIBKGK@?$AA_?$AAC?$AAr?$AAt?$AAM?$AAe?$AAm?$AAD?$AAu?$AAm?$AAp?$AAS?$AAt?$AAa?$AAt?$AAi?$AAs?$AAt?$AAi?$AAc?$AAs?$AA?$AA@ 00473ea8     LIBCMTD:dbgheap.obj
 0003:00002edc       ??_C@_1DK@LFLKFPDA@?$AAo?$AAf?$AAf?$AAs?$AAe?$AAt?$AA?5?$AA?$DN?$AA?$DN?$AA?5?$AA0?$AA?5?$AA?$HM?$AA?$HM?$AA?5?$AAo?$AAf?$AAf?$AAs?$AAe?$AAt?$AA?5?$AA?$DM?$AA?5?$AAs?$AAi?$AAz?$AAe?$AA?$AA@ 00473edc     LIBCMTD:dbgheap.obj
 0003:00002f24       ??_C@_1DG@DONCJBBJ@?$AA_?$AAa?$AAl?$AAi?$AAg?$AAn?$AAe?$AAd?$AA_?$AAo?$AAf?$AAf?$AAs?$AAe?$AAt?$AA_?$AAm?$AAa?$AAl?$AAl?$AAo?$AAc?$AA_?$AAd?$AAb?$AAg?$AA?$AA@ 00473f24     LIBCMTD:dbgheap.obj
 0003:00002f64       ??_C@_1CE@NPMGPNNP@?$AAI?$AAS?$AA_?$AA2?$AA_?$AAP?$AAO?$AAW?$AA_?$AAN?$AA?$CI?$AAa?$AAl?$AAi?$AAg?$AAn?$AA?$CJ?$AA?$AA@ 00473f64     LIBCMTD:dbgheap.obj
 0003:00002f90       ??_C@_1DI@NINIKFFK@?$AA_?$AAa?$AAl?$AAi?$AAg?$AAn?$AAe?$AAd?$AA_?$AAo?$AAf?$AAf?$AAs?$AAe?$AAt?$AA_?$AAr?$AAe?$AAa?$AAl?$AAl?$AAo?$AAc?$AA_?$AAd?$AAb?$AAg?$AA?$AA@ 00473f90     LIBCMTD:dbgheap.obj
 0003:00002fd4       ??_C@_0DL@PGHMMKNE@Damage?5before?50x?$CFp?5which?5was?5all@ 00473fd4     LIBCMTD:dbgheap.obj
 0003:00003020       ??_C@_0EI@NDNJMAJK@The?5block?5at?50x?$CFp?5was?5not?5alloca@ 00474020     LIBCMTD:dbgheap.obj
 0003:00003078       ??_C@_0EF@PGELACII@The?5block?5at?50x?$CFp?5was?5not?5alloca@ 00474078     LIBCMTD:dbgheap.obj
 0003:000030cc       ??_C@_1CG@CEGMHIMN@?$AA_?$AAa?$AAl?$AAi?$AAg?$AAn?$AAe?$AAd?$AA_?$AAm?$AAs?$AAi?$AAz?$AAe?$AA_?$AAd?$AAb?$AAg?$AA?$AA@ 004740cc     LIBCMTD:dbgheap.obj
 0003:000030fc       ??_C@_1CC@MOBIKHH@?$AAm?$AAe?$AAm?$AAb?$AAl?$AAo?$AAc?$AAk?$AA?5?$AA?$CB?$AA?$DN?$AA?5?$AAN?$AAU?$AAL?$AAL?$AA?$AA@ 004740fc     LIBCMTD:dbgheap.obj
 0003:00003124       ??_C@_0DC@LMJHGCKC@f?3?2dd?2vctools?2crt_bld?2self_x86?2c@ 00474124     LIBCMTD:tidtable.obj
 0003:00003160       ??_C@_07PEJMOBNF@FlsFree?$AA@ 00474160     LIBCMTD:tidtable.obj
 0003:0000316c       ??_C@_0M@JCPCPOEF@FlsSetValue?$AA@ 0047416c     LIBCMTD:tidtable.obj
 0003:0000317c       ??_C@_0M@GDNOONDI@FlsGetValue?$AA@ 0047417c     LIBCMTD:tidtable.obj
 0003:0000318c       ??_C@_08KNHFBNJ@FlsAlloc?$AA@ 0047418c     LIBCMTD:tidtable.obj
 0003:00003198       ??_C@_1BK@DBDEIDLH@?$AAK?$AAE?$AAR?$AAN?$AAE?$AAL?$AA3?$AA2?$AA?4?$AAD?$AAL?$AAL?$AA?$AA@ 00474198     LIBCMTD:tidtable.obj
 0003:000031b8       ??_C@_1GE@JDDMFOID@?$AAf?$AA?3?$AA?2?$AAd?$AAd?$AA?2?$AAv?$AAc?$AAt?$AAo?$AAo?$AAl?$AAs?$AA?2?$AAc?$AAr?$AAt?$AA_?$AAb?$AAl?$AAd?$AA?2?$AAs?$AAe?$AAl?$AAf?$AA_?$AAx?$AA8?$AA6?$AA?2?$AAc@ 004741b8     LIBCMTD:heapinit.obj
 0003:00003230       ??_C@_1BC@DENNNKIM@?$AA_?$AAc?$AAr?$AAt?$AAh?$AAe?$AAa?$AAp?$AA?$AA@ 00474230     LIBCMTD:heapinit.obj
 0003:00003248       ??_C@_1BO@BKOMIGKJ@?$AAr?$AAu?$AAn?$AAt?$AAi?$AAm?$AAe?$AA?5?$AAe?$AAr?$AAr?$AAo?$AAr?$AA?5?$AA?$AA@ 00474248     LIBCMTD:crt0msg.obj
 0003:0000326c       ??_C@_15JNBOKNOG@?$AA?$AN?$AA?6?$AA?$AA@ 0047426c     LIBCMTD:crt0msg.obj
 0003:00003274       ??_C@_1BM@JBBEPPHI@?$AAT?$AAL?$AAO?$AAS?$AAS?$AA?5?$AAe?$AAr?$AAr?$AAo?$AAr?$AA?$AN?$AA?6?$AA?$AA@ 00474274     LIBCMTD:crt0msg.obj
 0003:00003298       ??_C@_1BK@KMOMNAAI@?$AAS?$AAI?$AAN?$AAG?$AA?5?$AAe?$AAr?$AAr?$AAo?$AAr?$AA?$AN?$AA?6?$AA?$AA@ 00474298     LIBCMTD:crt0msg.obj
 0003:000032b8       ??_C@_1BO@BFCDCGC@?$AAD?$AAO?$AAM?$AAA?$AAI?$AAN?$AA?5?$AAe?$AAr?$AAr?$AAo?$AAr?$AA?$AN?$AA?6?$AA?$AA@ 004742b8     LIBCMTD:crt0msg.obj
 0003:000032e0       ??_C@_1BOO@KGEDBGAJ@?$AAR?$AA6?$AA0?$AA3?$AA3?$AA?$AN?$AA?6?$AA?9?$AA?5?$AAA?$AAt?$AAt?$AAe?$AAm?$AAp?$AAt?$AA?5?$AAt?$AAo?$AA?5?$AAu?$AAs?$AAe?$AA?5?$AAM?$AAS?$AAI?$AAL?$AA?5?$AAc?$AAo?$AAd@ 004742e0     LIBCMTD:crt0msg.obj
 0003:00003530       ??_C@_1GG@GOPILAJP@?$AAR?$AA6?$AA0?$AA3?$AA2?$AA?$AN?$AA?6?$AA?9?$AA?5?$AAn?$AAo?$AAt?$AA?5?$AAe?$AAn?$AAo?$AAu?$AAg?$AAh?$AA?5?$AAs?$AAp?$AAa?$AAc?$AAe?$AA?5?$AAf?$AAo?$AAr?$AA?5?$AAl?$AAo@ 00474530     LIBCMTD:crt0msg.obj
 0003:000035b0       ??_C@_1MG@ENCOOIDF@?$AAR?$AA6?$AA0?$AA3?$AA1?$AA?$AN?$AA?6?$AA?9?$AA?5?$AAA?$AAt?$AAt?$AAe?$AAm?$AAp?$AAt?$AA?5?$AAt?$AAo?$AA?5?$AAi?$AAn?$AAi?$AAt?$AAi?$AAa?$AAl?$AAi?$AAz?$AAe?$AA?5?$AAt@ 004745b0     LIBCMTD:crt0msg.obj
 0003:000036a0       ??_C@_1DO@BMFCDCD@?$AAR?$AA6?$AA0?$AA3?$AA0?$AA?$AN?$AA?6?$AA?9?$AA?5?$AAC?$AAR?$AAT?$AA?5?$AAn?$AAo?$AAt?$AA?5?$AAi?$AAn?$AAi?$AAt?$AAi?$AAa?$AAl?$AAi?$AAz?$AAe?$AAd?$AA?$AN?$AA?6?$AA?$AA@ 004746a0     LIBCMTD:crt0msg.obj
 0003:000036f0       ??_C@_1EK@HHFLMAOL@?$AAR?$AA6?$AA0?$AA2?$AA8?$AA?$AN?$AA?6?$AA?9?$AA?5?$AAu?$AAn?$AAa?$AAb?$AAl?$AAe?$AA?5?$AAt?$AAo?$AA?5?$AAi?$AAn?$AAi?$AAt?$AAi?$AAa?$AAl?$AAi?$AAz?$AAe?$AA?5?$AAh?$AAe@ 004746f0     LIBCMTD:crt0msg.obj
 0003:00003748       ??_C@_1GK@MFGOKLAG@?$AAR?$AA6?$AA0?$AA2?$AA7?$AA?$AN?$AA?6?$AA?9?$AA?5?$AAn?$AAo?$AAt?$AA?5?$AAe?$AAn?$AAo?$AAu?$AAg?$AAh?$AA?5?$AAs?$AAp?$AAa?$AAc?$AAe?$AA?5?$AAf?$AAo?$AAr?$AA?5?$AAl?$AAo@ 00474748     LIBCMTD:crt0msg.obj
 0003:000037c8       ??_C@_1GK@MCAAGJMO@?$AAR?$AA6?$AA0?$AA2?$AA6?$AA?$AN?$AA?6?$AA?9?$AA?5?$AAn?$AAo?$AAt?$AA?5?$AAe?$AAn?$AAo?$AAu?$AAg?$AAh?$AA?5?$AAs?$AAp?$AAa?$AAc?$AAe?$AA?5?$AAf?$AAo?$AAr?$AA?5?$AAs?$AAt@ 004747c8     LIBCMTD:crt0msg.obj
 0003:00003848       ??_C@_1EM@MAADIHMB@?$AAR?$AA6?$AA0?$AA2?$AA5?$AA?$AN?$AA?6?$AA?9?$AA?5?$AAp?$AAu?$AAr?$AAe?$AA?5?$AAv?$AAi?$AAr?$AAt?$AAu?$AAa?$AAl?$AA?5?$AAf?$AAu?$AAn?$AAc?$AAt?$AAi?$AAo?$AAn?$AA?5?$AAc@ 00474848     LIBCMTD:crt0msg.obj
 0003:000038a8       ??_C@_1GK@FHCKBEFA@?$AAR?$AA6?$AA0?$AA2?$AA4?$AA?$AN?$AA?6?$AA?9?$AA?5?$AAn?$AAo?$AAt?$AA?5?$AAe?$AAn?$AAo?$AAu?$AAg?$AAh?$AA?5?$AAs?$AAp?$AAa?$AAc?$AAe?$AA?5?$AAf?$AAo?$AAr?$AA?5?$AA_?$AAo@ 004748a8     LIBCMTD:crt0msg.obj
 0003:00003928       ??_C@_1FC@ECHBIFBC@?$AAR?$AA6?$AA0?$AA1?$AA9?$AA?$AN?$AA?6?$AA?9?$AA?5?$AAu?$AAn?$AAa?$AAb?$AAl?$AAe?$AA?5?$AAt?$AAo?$AA?5?$AAo?$AAp?$AAe?$AAn?$AA?5?$AAc?$AAo?$AAn?$AAs?$AAo?$AAl?$AAe?$AA?5@ 00474928     LIBCMTD:crt0msg.obj
 0003:00003990       ??_C@_1EC@JIBHAOPH@?$AAR?$AA6?$AA0?$AA1?$AA8?$AA?$AN?$AA?6?$AA?9?$AA?5?$AAu?$AAn?$AAe?$AAx?$AAp?$AAe?$AAc?$AAt?$AAe?$AAd?$AA?5?$AAh?$AAe?$AAa?$AAp?$AA?5?$AAe?$AAr?$AAr?$AAo?$AAr?$AA?$AN?$AA?6@ 00474990     LIBCMTD:crt0msg.obj
 0003:000039e0       ??_C@_1FK@BEOGODMC@?$AAR?$AA6?$AA0?$AA1?$AA7?$AA?$AN?$AA?6?$AA?9?$AA?5?$AAu?$AAn?$AAe?$AAx?$AAp?$AAe?$AAc?$AAt?$AAe?$AAd?$AA?5?$AAm?$AAu?$AAl?$AAt?$AAi?$AAt?$AAh?$AAr?$AAe?$AAa?$AAd?$AA?5@ 004749e0     LIBCMTD:crt0msg.obj
 0003:00003a50       ??_C@_1FI@LOGNIKDM@?$AAR?$AA6?$AA0?$AA1?$AA6?$AA?$AN?$AA?6?$AA?9?$AA?5?$AAn?$AAo?$AAt?$AA?5?$AAe?$AAn?$AAo?$AAu?$AAg?$AAh?$AA?5?$AAs?$AAp?$AAa?$AAc?$AAe?$AA?5?$AAf?$AAo?$AAr?$AA?5?$AAt?$AAh@ 00474a50     LIBCMTD:crt0msg.obj
 0003:00003ac0       ??_C@_1EG@BEHAGFJD@?$AAR?$AA6?$AA0?$AA1?$AA0?$AA?$AN?$AA?6?$AA?9?$AA?5?$AAa?$AAb?$AAo?$AAr?$AAt?$AA?$CI?$AA?$CJ?$AA?5?$AAh?$AAa?$AAs?$AA?5?$AAb?$AAe?$AAe?$AAn?$AA?5?$AAc?$AAa?$AAl?$AAl?$AAe?$AAd@ 00474ac0     LIBCMTD:crt0msg.obj
 0003:00003b18       ??_C@_1FI@HONFMGBI@?$AAR?$AA6?$AA0?$AA0?$AA9?$AA?$AN?$AA?6?$AA?9?$AA?5?$AAn?$AAo?$AAt?$AA?5?$AAe?$AAn?$AAo?$AAu?$AAg?$AAh?$AA?5?$AAs?$AAp?$AAa?$AAc?$AAe?$AA?5?$AAf?$AAo?$AAr?$AA?5?$AAe?$AAn@ 00474b18     LIBCMTD:crt0msg.obj
 0003:00003b88       ??_C@_1FE@LLNEDJMD@?$AAR?$AA6?$AA0?$AA0?$AA8?$AA?$AN?$AA?6?$AA?9?$AA?5?$AAn?$AAo?$AAt?$AA?5?$AAe?$AAn?$AAo?$AAu?$AAg?$AAh?$AA?5?$AAs?$AAp?$AAa?$AAc?$AAe?$AA?5?$AAf?$AAo?$AAr?$AA?5?$AAa?$AAr@ 00474b88     LIBCMTD:crt0msg.obj
 0003:00003bf0       ??_C@_1FK@PGACCAFB@?$AAR?$AA6?$AA0?$AA0?$AA2?$AA?$AN?$AA?6?$AA?9?$AA?5?$AAf?$AAl?$AAo?$AAa?$AAt?$AAi?$AAn?$AAg?$AA?5?$AAp?$AAo?$AAi?$AAn?$AAt?$AA?5?$AAs?$AAu?$AAp?$AAp?$AAo?$AAr?$AAt?$AA?5@ 00474bf0     LIBCMTD:crt0msg.obj
 0003:00003d38       ??_C@_1EK@MBDPDCGA@?$AAM?$AAi?$AAc?$AAr?$AAo?$AAs?$AAo?$AAf?$AAt?$AA?5?$AAV?$AAi?$AAs?$AAu?$AAa?$AAl?$AA?5?$AAC?$AA?$CL?$AA?$CL?$AA?5?$AAR?$AAu?$AAn?$AAt?$AAi?$AAm?$AAe?$AA?5?$AAL?$AAi?$AAb@ 00474d38     LIBCMTD:crt0msg.obj
 0003:00003d90       ??_C@_1IG@NMONDPP@?$AAw?$AAc?$AAs?$AAc?$AAa?$AAt?$AA_?$AAs?$AA?$CI?$AAo?$AAu?$AAt?$AAm?$AAs?$AAg?$AA?0?$AA?5?$AA?$CI?$AAs?$AAi?$AAz?$AAe?$AAo?$AAf?$AA?$CI?$AAo?$AAu?$AAt?$AAm?$AAs?$AAg?$AA?$CJ@ 00474d90     LIBCMTD:crt0msg.obj
 0003:00003e30       ??_C@_15IABLJNFO@?$AA?6?$AA?6?$AA?$AA@ 00474e30     LIBCMTD:crt0msg.obj
 0003:00003e38       ??_C@_1IA@DCJGKHFO@?$AAw?$AAc?$AAs?$AAc?$AAa?$AAt?$AA_?$AAs?$AA?$CI?$AAo?$AAu?$AAt?$AAm?$AAs?$AAg?$AA?0?$AA?5?$AA?$CI?$AAs?$AAi?$AAz?$AAe?$AAo?$AAf?$AA?$CI?$AAo?$AAu?$AAt?$AAm?$AAs?$AAg?$AA?$CJ@ 00474e38     LIBCMTD:crt0msg.obj
 0003:00003ed4       ??_C@_17LGKOMLJ@?$AA?4?$AA?4?$AA?4?$AA?$AA@ 00474ed4     LIBCMTD:crt0msg.obj
 0003:00003ee0       ??_C@_1HI@FLHKGEBE@?$AAw?$AAc?$AAs?$AAn?$AAc?$AAp?$AAy?$AA_?$AAs?$AA?$CI?$AAp?$AAc?$AAh?$AA?0?$AA?5?$AAp?$AAr?$AAo?$AAg?$AAn?$AAa?$AAm?$AAe?$AA_?$AAs?$AAi?$AAz?$AAe?$AA?5?$AA?9?$AA?5?$AA?$CI@ 00474ee0     LIBCMTD:crt0msg.obj
 0003:00003f70       ??_C@_1CO@EAEJAADC@?$AA?$DM?$AAp?$AAr?$AAo?$AAg?$AAr?$AAa?$AAm?$AA?5?$AAn?$AAa?$AAm?$AAe?$AA?5?$AAu?$AAn?$AAk?$AAn?$AAo?$AAw?$AAn?$AA?$DO?$AA?$AA@ 00474f70     LIBCMTD:crt0msg.obj
 0003:00003fa8       ??_C@_1HK@FJJNAABO@?$AAw?$AAc?$AAs?$AAc?$AAp?$AAy?$AA_?$AAs?$AA?$CI?$AAp?$AAr?$AAo?$AAg?$AAn?$AAa?$AAm?$AAe?$AA?0?$AA?5?$AAp?$AAr?$AAo?$AAg?$AAn?$AAa?$AAm?$AAe?$AA_?$AAs?$AAi?$AAz?$AAe@ 00474fa8     LIBCMTD:crt0msg.obj
 0003:0000403c       ??_C@_1DE@JNGNBFGO@?$AAR?$AAu?$AAn?$AAt?$AAi?$AAm?$AAe?$AA?5?$AAE?$AAr?$AAr?$AAo?$AAr?$AA?$CB?$AA?6?$AA?6?$AAP?$AAr?$AAo?$AAg?$AAr?$AAa?$AAm?$AA?3?$AA?5?$AA?$AA@ 0047503c     LIBCMTD:crt0msg.obj
 0003:00004080       ??_C@_1KO@BKLCKNFL@?$AAw?$AAc?$AAs?$AAc?$AAp?$AAy?$AA_?$AAs?$AA?$CI?$AAo?$AAu?$AAt?$AAm?$AAs?$AAg?$AA?0?$AA?5?$AA?$CI?$AAs?$AAi?$AAz?$AAe?$AAo?$AAf?$AA?$CI?$AAo?$AAu?$AAt?$AAm?$AAs?$AAg?$AA?$CJ@ 00475080     LIBCMTD:crt0msg.obj
 0003:00004150       ??_C@_1BI@EAHMBMEC@?$AA_?$AAN?$AAM?$AAS?$AAG?$AA_?$AAW?$AAR?$AAI?$AAT?$AAE?$AA?$AA@ 00475150     LIBCMTD:crt0msg.obj
 0003:00004170       ??_C@_1GC@HKOJBOFF@?$AAf?$AA?3?$AA?2?$AAd?$AAd?$AA?2?$AAv?$AAc?$AAt?$AAo?$AAo?$AAl?$AAs?$AA?2?$AAc?$AAr?$AAt?$AA_?$AAb?$AAl?$AAd?$AA?2?$AAs?$AAe?$AAl?$AAf?$AA_?$AAx?$AA8?$AA6?$AA?2?$AAc@ 00475170     LIBCMTD:crt0msg.obj
 0003:00004208       ??_C@_01KDCPPGHE@r?$AA@    00475208     LIBCMTD:_pdblkup_.obj
 0003:0000420c       ??_C@_0BB@KCIACLNC@PDBOpenValidate5?$AA@ 0047520c     LIBCMTD:_pdblkup_.obj
 0003:00004220       ??_C@_1CK@HHHCOJPD@?$AAE?$AAn?$AAv?$AAi?$AAr?$AAo?$AAn?$AAm?$AAe?$AAn?$AAt?$AAD?$AAi?$AAr?$AAe?$AAc?$AAt?$AAo?$AAr?$AAy?$AA?$AA@ 00475220     LIBCMTD:_pdblkup_.obj
 0003:00004258       ??_C@_1FM@DNCABAP@?$AAS?$AAO?$AAF?$AAT?$AAW?$AAA?$AAR?$AAE?$AA?2?$AAM?$AAi?$AAc?$AAr?$AAo?$AAs?$AAo?$AAf?$AAt?$AA?2?$AAV?$AAi?$AAs?$AAu?$AAa?$AAl?$AAS?$AAt?$AAu?$AAd?$AAi?$AAo?$AA?2@ 00475258     LIBCMTD:_pdblkup_.obj
 0003:000042c8       ??_C@_0M@HLOHPNFA@RegCloseKey?$AA@ 004752c8     LIBCMTD:_pdblkup_.obj
 0003:000042d8       ??_C@_0BB@GLNAEDBD@RegQueryValueExW?$AA@ 004752d8     LIBCMTD:_pdblkup_.obj
 0003:000042ec       ??_C@_0O@COHOBMLB@RegOpenKeyExW?$AA@ 004752ec     LIBCMTD:_pdblkup_.obj
 0003:000042fc       ??_C@_1BK@GAEMIDIL@?$AAA?$AAD?$AAV?$AAA?$AAP?$AAI?$AA3?$AA2?$AA?4?$AAD?$AAL?$AAL?$AA?$AA@ 004752fc     LIBCMTD:_pdblkup_.obj
 0003:0000431c       ??_C@_03KHICJKCI@?4?4?4?$AA@ 0047531c     LIBCMTD:dbgrpt.obj
 0003:00004320       ??_C@_0BB@NAGLCMLI@Assertion?5Failed?$AA@ 00475320     LIBCMTD:dbgrpt.obj
 0003:00004334       ??_C@_07KGMMFLDN@Warning?$AA@ 00475334     LIBCMTD:dbgrpt.obj
 0003:00004350       ??_C@_0DA@PCCBBBID@f?3?2dd?2vctools?2crt_bld?2self_x86?2c@ 00475350     LIBCMTD:dbgrpt.obj
 0003:00004390       ??_C@_1FI@PHIAFFHM@?$AA?$CI?$AA?$CC?$AAT?$AAh?$AAe?$AA?5?$AAh?$AAo?$AAo?$AAk?$AA?5?$AAf?$AAu?$AAn?$AAc?$AAt?$AAi?$AAo?$AAn?$AA?5?$AAi?$AAs?$AA?5?$AAn?$AAo?$AAt?$AA?5?$AAi?$AAn?$AA?5?$AAt?$AAh@ 00475390     LIBCMTD:dbgrpt.obj
 0003:000043fc       ??_C@_1CG@JBJEFOCM@?$AAp?$AAf?$AAn?$AAN?$AAe?$AAw?$AAH?$AAo?$AAo?$AAk?$AA?5?$AA?$CB?$AA?$DN?$AA?5?$AAN?$AAU?$AAL?$AAL?$AA?$AA@ 004753fc     LIBCMTD:dbgrpt.obj
 0003:0000442c       ??_C@_1CG@GNMJDMIO@?$AA_?$AAC?$AAr?$AAt?$AAS?$AAe?$AAt?$AAR?$AAe?$AAp?$AAo?$AAr?$AAt?$AAH?$AAo?$AAo?$AAk?$AA2?$AA?$AA@ 0047542c     LIBCMTD:dbgrpt.obj
 0003:00004460       ??_C@_1GA@IBJGKIFE@?$AAf?$AA?3?$AA?2?$AAd?$AAd?$AA?2?$AAv?$AAc?$AAt?$AAo?$AAo?$AAl?$AAs?$AA?2?$AAc?$AAr?$AAt?$AA_?$AAb?$AAl?$AAd?$AA?2?$AAs?$AAe?$AAl?$AAf?$AA_?$AAx?$AA8?$AA6?$AA?2?$AAc@ 00475460     LIBCMTD:dbgrpt.obj
 0003:000044d8       ??_C@_1HI@OFEHGPPC@?$AAm?$AAo?$AAd?$AAe?$AA?5?$AA?$DN?$AA?$DN?$AA?5?$AA_?$AAC?$AAR?$AAT?$AA_?$AAR?$AAP?$AAT?$AAH?$AAO?$AAO?$AAK?$AA_?$AAI?$AAN?$AAS?$AAT?$AAA?$AAL?$AAL?$AA?5?$AA?$HM?$AA?$HM?$AA?5@ 004754d8     LIBCMTD:dbgrpt.obj
 0003:00004568       ??_C@_0CD@EBCGLDDL@Microsoft?5Visual?5C?$CL?$CL?5Debug?5Libra@ 00475568     LIBCMTD:dbgrpt.obj
 0003:00004594       ??_C@_0CL@EACFGMNB@_CrtDbgReport?3?5String?5too?5long?5o@ 00475594     LIBCMTD:dbgrpt.obj
 0003:000045c8       ??_C@_1JG@CPKCIOEE@?$AAs?$AAt?$AAr?$AAc?$AAp?$AAy?$AA_?$AAs?$AA?$CI?$AAs?$AAz?$AAO?$AAu?$AAt?$AAM?$AAe?$AAs?$AAs?$AAa?$AAg?$AAe?$AA?0?$AA?5?$AA4?$AA0?$AA9?$AA6?$AA?0?$AA?5?$AA?$CC?$AA_?$AAC@ 004755c8     LIBCMTD:dbgrpt.obj
 0003:00004680       ??_C@_0FF@CCONDJCB@Debug?5?$CFs?$CB?6?6Program?3?5?$CFs?$CFs?$CFs?$CFs?$CFs?$CFs@ 00475680     LIBCMTD:dbgrpt.obj
 0003:000046e8       ??_C@_09OFBFHMBK@?6Module?3?5?$AA@ 004756e8     LIBCMTD:dbgrpt.obj
 0003:000046f4       ??_C@_07OPHPPLBG@?6File?3?5?$AA@ 004756f4     LIBCMTD:dbgrpt.obj
 0003:00004700       ??_C@_07DBMPPHDI@?6Line?3?5?$AA@ 00475700     LIBCMTD:dbgrpt.obj
 0003:0000470c       ??_C@_02PHMGELLB@?6?6?$AA@ 0047570c     LIBCMTD:dbgrpt.obj
 0003:00004710       ??_C@_0N@MEECIJGN@Expression?3?5?$AA@ 00475710     LIBCMTD:dbgrpt.obj
 0003:00004720       ??_C@_0HD@GNBNFCCL@?6?6For?5information?5on?5how?5your?5pr@ 00475720     LIBCMTD:dbgrpt.obj
 0003:000047b0       ??_C@_1NO@LECLLHOL@?$AAm?$AAe?$AAm?$AAc?$AAp?$AAy?$AA_?$AAs?$AA?$CI?$AAs?$AAz?$AAS?$AAh?$AAo?$AAr?$AAt?$AAP?$AAr?$AAo?$AAg?$AAN?$AAa?$AAm?$AAe?$AA?0?$AA?5?$AAs?$AAi?$AAz?$AAe?$AAo?$AAf@ 004757b0     LIBCMTD:dbgrpt.obj
 0003:000048bc       ??_C@_0BH@DNAGHKFM@?$DMprogram?5name?5unknown?$DO?$AA@ 004758bc     LIBCMTD:dbgrpt.obj
 0003:000048d8       ??_C@_1GG@DLDHOIGE@?$AAs?$AAt?$AAr?$AAc?$AAp?$AAy?$AA_?$AAs?$AA?$CI?$AAs?$AAz?$AAE?$AAx?$AAe?$AAN?$AAa?$AAm?$AAe?$AA?0?$AA?5?$AA2?$AA6?$AA0?$AA?0?$AA?5?$AA?$CC?$AA?$DM?$AAp?$AAr?$AAo?$AAg?$AAr@ 004758d8     LIBCMTD:dbgrpt.obj
 0003:00004954       ??_C@_1CI@IDOKFLAJ@?$AA_?$AA_?$AAc?$AAr?$AAt?$AAM?$AAe?$AAs?$AAs?$AAa?$AAg?$AAe?$AAW?$AAi?$AAn?$AAd?$AAo?$AAw?$AAA?$AA?$AA@ 00475954     LIBCMTD:dbgrpt.obj
 0003:00004984       ??_C@_1CC@CGHMNGDG@?$AAA?$AAs?$AAs?$AAe?$AAr?$AAt?$AAi?$AAo?$AAn?$AA?5?$AAF?$AAa?$AAi?$AAl?$AAe?$AAd?$AA?$AA@ 00475984     LIBCMTD:dbgrptw.obj
 0003:000049ac       ??_C@_1M@ILHOPKA@?$AAE?$AAr?$AAr?$AAo?$AAr?$AA?$AA@ 004759ac     LIBCMTD:dbgrptw.obj
 0003:000049bc       ??_C@_1BA@GLMCNLEM@?$AAW?$AAa?$AAr?$AAn?$AAi?$AAn?$AAg?$AA?$AA@ 004759bc     LIBCMTD:dbgrptw.obj
 0003:000049e0       ??_C@_1CI@IIHEAKEI@?$AA_?$AAC?$AAr?$AAt?$AAS?$AAe?$AAt?$AAR?$AAe?$AAp?$AAo?$AAr?$AAt?$AAH?$AAo?$AAo?$AAk?$AAW?$AA2?$AA?$AA@ 004759e0     LIBCMTD:dbgrptw.obj
 0003:00004a10       ??_C@_1EG@PEOEAKBB@?$AAM?$AAi?$AAc?$AAr?$AAo?$AAs?$AAo?$AAf?$AAt?$AA?5?$AAV?$AAi?$AAs?$AAu?$AAa?$AAl?$AA?5?$AAC?$AA?$CL?$AA?$CL?$AA?5?$AAD?$AAe?$AAb?$AAu?$AAg?$AA?5?$AAL?$AAi?$AAb?$AAr?$AAa@ 00475a10     LIBCMTD:dbgrptw.obj
 0003:00004a68       ??_C@_1FG@BBOLDHGF@?$AA_?$AAC?$AAr?$AAt?$AAD?$AAb?$AAg?$AAR?$AAe?$AAp?$AAo?$AAr?$AAt?$AA?3?$AA?5?$AAS?$AAt?$AAr?$AAi?$AAn?$AAg?$AA?5?$AAt?$AAo?$AAo?$AA?5?$AAl?$AAo?$AAn?$AAg?$AA?5?$AAo@ 00475a68     LIBCMTD:dbgrptw.obj
 0003:00004ad0       ??_C@_1JI@EACPGHID@?$AAw?$AAc?$AAs?$AAc?$AAp?$AAy?$AA_?$AAs?$AA?$CI?$AAs?$AAz?$AAO?$AAu?$AAt?$AAM?$AAe?$AAs?$AAs?$AAa?$AAg?$AAe?$AA?0?$AA?5?$AA4?$AA0?$AA9?$AA6?$AA?0?$AA?5?$AAL?$AA?$CC?$AA_@ 00475ad0     LIBCMTD:dbgrptw.obj
 0003:00004b88       ??_C@_1KK@MEFMPOLM@?$AAD?$AAe?$AAb?$AAu?$AAg?$AA?5?$AA?$CF?$AAs?$AA?$CB?$AA?6?$AA?6?$AAP?$AAr?$AAo?$AAg?$AAr?$AAa?$AAm?$AA?3?$AA?5?$AA?$CF?$AAs?$AA?$CF?$AAs?$AA?$CF?$AAs?$AA?$CF?$AAs?$AA?$CF?$AAs?$AA?$CF?$AAs@ 00475b88     LIBCMTD:dbgrptw.obj
 0003:00004c54       ??_C@_1BE@CGCJKGHI@?$AA?6?$AAM?$AAo?$AAd?$AAu?$AAl?$AAe?$AA?3?$AA?5?$AA?$AA@ 00475c54     LIBCMTD:dbgrptw.obj
 0003:00004c6c       ??_C@_1BA@LNHECFIM@?$AA?6?$AAF?$AAi?$AAl?$AAe?$AA?3?$AA?5?$AA?$AA@ 00475c6c     LIBCMTD:dbgrptw.obj
 0003:00004c80       ??_C@_1BA@GLLGCPCK@?$AA?6?$AAL?$AAi?$AAn?$AAe?$AA?3?$AA?5?$AA?$AA@ 00475c80     LIBCMTD:dbgrptw.obj
 0003:00004c94       ??_C@_1BK@PEDCIPMA@?$AAE?$AAx?$AAp?$AAr?$AAe?$AAs?$AAs?$AAi?$AAo?$AAn?$AA?3?$AA?5?$AA?$AA@ 00475c94     LIBCMTD:dbgrptw.obj
 0003:00004cb4       ??_C@_11LOCGONAA@?$AA?$AA@ 00475cb4     LIBCMTD:dbgrptw.obj
 0003:00004cb8       ??_C@_1OG@PMPPFHAF@?$AA?6?$AA?6?$AAF?$AAo?$AAr?$AA?5?$AAi?$AAn?$AAf?$AAo?$AAr?$AAm?$AAa?$AAt?$AAi?$AAo?$AAn?$AA?5?$AAo?$AAn?$AA?5?$AAh?$AAo?$AAw?$AA?5?$AAy?$AAo?$AAu?$AAr?$AA?5?$AAp?$AAr@ 00475cb8     LIBCMTD:dbgrptw.obj
 0003:00004dd0       ??_C@_1GI@DEDNNLCI@?$AAw?$AAc?$AAs?$AAc?$AAp?$AAy?$AA_?$AAs?$AA?$CI?$AAs?$AAz?$AAE?$AAx?$AAe?$AAN?$AAa?$AAm?$AAe?$AA?0?$AA?5?$AA2?$AA6?$AA0?$AA?0?$AA?5?$AAL?$AA?$CC?$AA?$DM?$AAp?$AAr?$AAo?$AAg@ 00475dd0     LIBCMTD:dbgrptw.obj
 0003:00004e4c       ??_C@_1CI@PGJIFDEK@?$AA_?$AA_?$AAc?$AAr?$AAt?$AAM?$AAe?$AAs?$AAs?$AAa?$AAg?$AAe?$AAW?$AAi?$AAn?$AAd?$AAo?$AAw?$AAW?$AA?$AA@ 00475e4c     LIBCMTD:dbgrptw.obj
 0003:00004e7c       ??_C@_1BC@GDGBMEMK@?$AAH?$AAH?$AA?3?$AAm?$AAm?$AA?3?$AAs?$AAs?$AA?$AA@ 00475e7c     LIBCMTD:nlsdata2.obj
 0003:00004e94       ??_C@_1CI@KNAKOEBC@?$AAd?$AAd?$AAd?$AAd?$AA?0?$AA?5?$AAM?$AAM?$AAM?$AAM?$AA?5?$AAd?$AAd?$AA?0?$AA?5?$AAy?$AAy?$AAy?$AAy?$AA?$AA@ 00475e94     LIBCMTD:nlsdata2.obj
 0003:00004ec4       ??_C@_1BC@IEBCMHCM@?$AAM?$AAM?$AA?1?$AAd?$AAd?$AA?1?$AAy?$AAy?$AA?$AA@ 00475ec4     LIBCMTD:nlsdata2.obj
 0003:00004edc       ??_C@_15CLMNNGEL@?$AAP?$AAM?$AA?$AA@ 00475edc     LIBCMTD:nlsdata2.obj
 0003:00004ee4       ??_C@_15ODEHAHHF@?$AAA?$AAM?$AA?$AA@ 00475ee4     LIBCMTD:nlsdata2.obj
 0003:00004eec       ??_C@_1BC@FEMKIFH@?$AAD?$AAe?$AAc?$AAe?$AAm?$AAb?$AAe?$AAr?$AA?$AA@ 00475eec     LIBCMTD:nlsdata2.obj
 0003:00004f04       ??_C@_1BC@BGLIFPF@?$AAN?$AAo?$AAv?$AAe?$AAm?$AAb?$AAe?$AAr?$AA?$AA@ 00475f04     LIBCMTD:nlsdata2.obj
 0003:00004f1c       ??_C@_1BA@EPANDLNG@?$AAO?$AAc?$AAt?$AAo?$AAb?$AAe?$AAr?$AA?$AA@ 00475f1c     LIBCMTD:nlsdata2.obj
 0003:00004f30       ??_C@_1BE@DKAAMBJL@?$AAS?$AAe?$AAp?$AAt?$AAe?$AAm?$AAb?$AAe?$AAr?$AA?$AA@ 00475f30     LIBCMTD:nlsdata2.obj
 0003:00004f48       ??_C@_1O@PAHLKOAC@?$AAA?$AAu?$AAg?$AAu?$AAs?$AAt?$AA?$AA@ 00475f48     LIBCMTD:nlsdata2.obj
 0003:00004f58       ??_C@_19BIFMLPCD@?$AAJ?$AAu?$AAl?$AAy?$AA?$AA@ 00475f58     LIBCMTD:nlsdata2.obj
 0003:00004f64       ??_C@_19EPFLPGAP@?$AAJ?$AAu?$AAn?$AAe?$AA?$AA@ 00475f64     LIBCMTD:nlsdata2.obj
 0003:00004f70       ??_C@_1M@GJNLMHFD@?$AAA?$AAp?$AAr?$AAi?$AAl?$AA?$AA@ 00475f70     LIBCMTD:nlsdata2.obj
 0003:00004f80       ??_C@_1M@IKEENEDF@?$AAM?$AAa?$AAr?$AAc?$AAh?$AA?$AA@ 00475f80     LIBCMTD:nlsdata2.obj
 0003:00004f90       ??_C@_1BC@JGDDFFAM@?$AAF?$AAe?$AAb?$AAr?$AAu?$AAa?$AAr?$AAy?$AA?$AA@ 00475f90     LIBCMTD:nlsdata2.obj
 0003:00004fa8       ??_C@_1BA@EFMEIEBA@?$AAJ?$AAa?$AAn?$AAu?$AAa?$AAr?$AAy?$AA?$AA@ 00475fa8     LIBCMTD:nlsdata2.obj
 0003:00004fbc       ??_C@_17EGKACKIF@?$AAD?$AAe?$AAc?$AA?$AA@ 00475fbc     LIBCMTD:nlsdata2.obj
 0003:00004fc8       ??_C@_17BBDMLCIG@?$AAN?$AAo?$AAv?$AA?$AA@ 00475fc8     LIBCMTD:nlsdata2.obj
 0003:00004fd4       ??_C@_17FNLKOI@?$AAO?$AAc?$AAt?$AA?$AA@ 00475fd4     LIBCMTD:nlsdata2.obj
 0003:00004fe0       ??_C@_17HCHCOKMG@?$AAS?$AAe?$AAp?$AA?$AA@ 00475fe0     LIBCMTD:nlsdata2.obj
 0003:00004fec       ??_C@_17ICPELBCN@?$AAA?$AAu?$AAg?$AA?$AA@ 00475fec     LIBCMTD:nlsdata2.obj
 0003:00004ff8       ??_C@_17IJPCKHK@?$AAJ?$AAu?$AAl?$AA?$AA@ 00475ff8     LIBCMTD:nlsdata2.obj
 0003:00005004       ??_C@_17KCJGOCPB@?$AAJ?$AAu?$AAn?$AA?$AA@ 00476004     LIBCMTD:nlsdata2.obj
 0003:00005010       ??_C@_17PNNKMEED@?$AAM?$AAa?$AAy?$AA?$AA@ 00476010     LIBCMTD:nlsdata2.obj
 0003:0000501c       ??_C@_17LFPOIHDD@?$AAA?$AAp?$AAr?$AA?$AA@ 0047601c     LIBCMTD:nlsdata2.obj
 0003:00005028       ??_C@_17CKNLEDEC@?$AAM?$AAa?$AAr?$AA?$AA@ 00476028     LIBCMTD:nlsdata2.obj
 0003:00005034       ??_C@_17LMDJEKJN@?$AAF?$AAe?$AAb?$AA?$AA@ 00476034     LIBCMTD:nlsdata2.obj
 0003:00005040       ??_C@_17DKNBKCHM@?$AAJ?$AAa?$AAn?$AA?$AA@ 00476040     LIBCMTD:nlsdata2.obj
 0003:0000504c       ??_C@_1BC@ENMNNPAJ@?$AAS?$AAa?$AAt?$AAu?$AAr?$AAd?$AAa?$AAy?$AA?$AA@ 0047604c     LIBCMTD:nlsdata2.obj
 0003:00005064       ??_C@_1O@PDICJHAG@?$AAF?$AAr?$AAi?$AAd?$AAa?$AAy?$AA?$AA@ 00476064     LIBCMTD:nlsdata2.obj
 0003:00005074       ??_C@_1BC@HHMNLIHE@?$AAT?$AAh?$AAu?$AAr?$AAs?$AAd?$AAa?$AAy?$AA?$AA@ 00476074     LIBCMTD:nlsdata2.obj
 0003:0000508c       ??_C@_1BE@EBOGMDOH@?$AAW?$AAe?$AAd?$AAn?$AAe?$AAs?$AAd?$AAa?$AAy?$AA?$AA@ 0047608c     LIBCMTD:nlsdata2.obj
 0003:000050a4       ??_C@_1BA@ENFBFFEK@?$AAT?$AAu?$AAe?$AAs?$AAd?$AAa?$AAy?$AA?$AA@ 004760a4     LIBCMTD:nlsdata2.obj
 0003:000050b8       ??_C@_1O@MMNBFLIA@?$AAM?$AAo?$AAn?$AAd?$AAa?$AAy?$AA?$AA@ 004760b8     LIBCMTD:nlsdata2.obj
 0003:000050c8       ??_C@_1O@IHNHDHPB@?$AAS?$AAu?$AAn?$AAd?$AAa?$AAy?$AA?$AA@ 004760c8     LIBCMTD:nlsdata2.obj
 0003:000050d8       ??_C@_17GGIBDPIH@?$AAS?$AAa?$AAt?$AA?$AA@ 004760d8     LIBCMTD:nlsdata2.obj
 0003:000050e4       ??_C@_17HFOLPPLP@?$AAF?$AAr?$AAi?$AA?$AA@ 004760e4     LIBCMTD:nlsdata2.obj
 0003:000050f0       ??_C@_17PDPHAADD@?$AAT?$AAh?$AAu?$AA?$AA@ 004760f0     LIBCMTD:nlsdata2.obj
 0003:000050fc       ??_C@_17CJEDCEPE@?$AAW?$AAe?$AAd?$AA?$AA@ 004760fc     LIBCMTD:nlsdata2.obj
 0003:00005108       ??_C@_17BMKGEGOJ@?$AAT?$AAu?$AAe?$AA?$AA@ 00476108     LIBCMTD:nlsdata2.obj
 0003:00005114       ??_C@_17KBOMKBF@?$AAM?$AAo?$AAn?$AA?$AA@ 00476114     LIBCMTD:nlsdata2.obj
 0003:00005120       ??_C@_17MBGCMIPB@?$AAS?$AAu?$AAn?$AA?$AA@ 00476120     LIBCMTD:nlsdata2.obj
 0003:0000512c       ??_C@_08JCCMCCIL@HH?3mm?3ss?$AA@ 0047612c     LIBCMTD:nlsdata2.obj
 0003:00005138       ??_C@_0BE@CKGJFCPC@dddd?0?5MMMM?5dd?0?5yyyy?$AA@ 00476138     LIBCMTD:nlsdata2.obj
 0003:00005150       ??_C@_08BPBNCDIB@MM?1dd?1yy?$AA@ 00476150     LIBCMTD:nlsdata2.obj
 0003:0000515c       ??_C@_02CJNFDJBF@PM?$AA@   0047615c     LIBCMTD:nlsdata2.obj
 0003:00005160       ??_C@_02DEDBPAFC@AM?$AA@   00476160     LIBCMTD:nlsdata2.obj
 0003:00005164       ??_C@_08EDHMEBNP@December?$AA@ 00476164     LIBCMTD:nlsdata2.obj
 0003:00005170       ??_C@_08HCHEGEOA@November?$AA@ 00476170     LIBCMTD:nlsdata2.obj
 0003:0000517c       ??_C@_07JJNFCEND@October?$AA@ 0047617c     LIBCMTD:nlsdata2.obj
 0003:00005188       ??_C@_09BHHEALKD@September?$AA@ 00476188     LIBCMTD:nlsdata2.obj
 0003:00005194       ??_C@_06LBBHFDDG@August?$AA@ 00476194     LIBCMTD:nlsdata2.obj
 0003:0000519c       ??_C@_04MIEPOIFP@July?$AA@ 0047619c     LIBCMTD:nlsdata2.obj
 0003:000051a4       ??_C@_04CNLMGBGM@June?$AA@ 004761a4     LIBCMTD:nlsdata2.obj
 0003:000051ac       ??_C@_05DMJDNLEJ@April?$AA@ 004761ac     LIBCMTD:nlsdata2.obj
 0003:000051b4       ??_C@_05HPCKOFNC@March?$AA@ 004761b4     LIBCMTD:nlsdata2.obj
 0003:000051bc       ??_C@_08GNJGEPFN@February?$AA@ 004761bc     LIBCMTD:nlsdata2.obj
 0003:000051c8       ??_C@_07CGJPFGJA@January?$AA@ 004761c8     LIBCMTD:nlsdata2.obj
 0003:000051d4       ??_C@_03MKABNOCG@Dec?$AA@  004761d4     LIBCMTD:nlsdata2.obj
 0003:000051d8       ??_C@_03JPJOFNIA@Nov?$AA@  004761d8     LIBCMTD:nlsdata2.obj
 0003:000051dc       ??_C@_03BMAOKBAD@Oct?$AA@  004761dc     LIBCMTD:nlsdata2.obj
 0003:000051e0       ??_C@_03GGCAPAJC@Sep?$AA@  004761e0     LIBCMTD:nlsdata2.obj
 0003:000051e4       ??_C@_03IFJFEIGA@Aug?$AA@  004761e4     LIBCMTD:nlsdata2.obj
 0003:000051e8       ??_C@_03LBGABGKK@Jul?$AA@  004761e8     LIBCMTD:nlsdata2.obj
 0003:000051ec       ??_C@_03IDFGHECI@Jun?$AA@  004761ec     LIBCMTD:nlsdata2.obj
 0003:000051f0       ??_C@_03CNMDKL@May?$AA@    004761f0     LIBCMTD:nlsdata2.obj
 0003:000051f4       ??_C@_03LEOLGMJP@Apr?$AA@  004761f4     LIBCMTD:nlsdata2.obj
 0003:000051f8       ??_C@_03ODNJBKGA@Mar?$AA@  004761f8     LIBCMTD:nlsdata2.obj
 0003:000051fc       ??_C@_03HJBDCHOM@Feb?$AA@  004761fc     LIBCMTD:nlsdata2.obj
 0003:00005200       ??_C@_03JIHJHPIE@Jan?$AA@  00476200     LIBCMTD:nlsdata2.obj
 0003:00005204       ??_C@_08INBOOONO@Saturday?$AA@ 00476204     LIBCMTD:nlsdata2.obj
 0003:00005210       ??_C@_06JECMNKMI@Friday?$AA@ 00476210     LIBCMTD:nlsdata2.obj
 0003:00005218       ??_C@_08HACCIKIA@Thursday?$AA@ 00476218     LIBCMTD:nlsdata2.obj
 0003:00005224       ??_C@_09DLIGFAKA@Wednesday?$AA@ 00476224     LIBCMTD:nlsdata2.obj
 0003:00005230       ??_C@_07BAAGCFCM@Tuesday?$AA@ 00476230     LIBCMTD:nlsdata2.obj
 0003:0000523c       ??_C@_06JLEDEDGH@Monday?$AA@ 0047623c     LIBCMTD:nlsdata2.obj
 0003:00005244       ??_C@_06OOPIFAJ@Sunday?$AA@ 00476244     LIBCMTD:nlsdata2.obj
 0003:0000524c       ??_C@_03FEFJNEK@Sat?$AA@   0047624c     LIBCMTD:nlsdata2.obj
 0003:00005250       ??_C@_03IDIOELNC@Fri?$AA@  00476250     LIBCMTD:nlsdata2.obj
 0003:00005254       ??_C@_03IOFIKPDN@Thu?$AA@  00476254     LIBCMTD:nlsdata2.obj
 0003:00005258       ??_C@_03MHOMLAJA@Wed?$AA@  00476258     LIBCMTD:nlsdata2.obj
 0003:0000525c       ??_C@_03NAGEINEP@Tue?$AA@  0047625c     LIBCMTD:nlsdata2.obj
 0003:00005260       ??_C@_03PDAGKDH@Mon?$AA@   00476260     LIBCMTD:nlsdata2.obj
 0003:00005264       ??_C@_03KOEHGMDN@Sun?$AA@  00476264     LIBCMTD:nlsdata2.obj
 0003:00005268       ??_C@_07LCBHPJJN@LC_TIME?$AA@ 00476268     LIBCMTD:setlocal.obj
 0003:00005274       ??_C@_0L@DLHIECNL@LC_NUMERIC?$AA@ 00476274     LIBCMTD:setlocal.obj
 0003:00005284       ??_C@_0M@MIENIKLA@LC_MONETARY?$AA@ 00476284     LIBCMTD:setlocal.obj
 0003:00005294       ??_C@_08EADHIDAD@LC_CTYPE?$AA@ 00476294     LIBCMTD:setlocal.obj
 0003:000052a0       ??_C@_0L@KFJHEKIK@LC_COLLATE?$AA@ 004762a0     LIBCMTD:setlocal.obj
 0003:000052b0       ??_C@_06NEFDFEKB@LC_ALL?$AA@ 004762b0     LIBCMTD:setlocal.obj
 0003:000052b8       ___lc_category             004762b8     LIBCMTD:setlocal.obj
 0003:000053a8       ??_C@_1CI@FGIONOJM@?$AA_?$AAc?$AAo?$AAn?$AAf?$AAi?$AAg?$AAt?$AAh?$AAr?$AAe?$AAa?$AAd?$AAl?$AAo?$AAc?$AAa?$AAl?$AAe?$AA?$AA@ 004763a8     LIBCMTD:setlocal.obj
 0003:000053d8       ??_C@_1GE@OLEIGPBJ@?$AAf?$AA?3?$AA?2?$AAd?$AAd?$AA?2?$AAv?$AAc?$AAt?$AAo?$AAo?$AAl?$AAs?$AA?2?$AAc?$AAr?$AAt?$AA_?$AAb?$AAl?$AAd?$AA?2?$AAs?$AAe?$AAl?$AAf?$AA_?$AAx?$AA8?$AA6?$AA?2?$AAc@ 004763d8     LIBCMTD:setlocal.obj
 0003:00005450       ??_C@_1GA@LDEGDKD@?$AA?$CI?$AA?$CC?$AAI?$AAn?$AAv?$AAa?$AAl?$AAi?$AAd?$AA?5?$AAp?$AAa?$AAr?$AAa?$AAm?$AAe?$AAt?$AAe?$AAr?$AA?5?$AAf?$AAo?$AAr?$AA?5?$AA_?$AAc?$AAo?$AAn?$AAf?$AAi?$AAg?$AAt@ 00476450     LIBCMTD:setlocal.obj
 0003:000054c4       ??_C@_0DC@JCPFNMID@f?3?2dd?2vctools?2crt_bld?2self_x86?2c@ 004764c4     LIBCMTD:setlocal.obj
 0003:00005500       ??_C@_1BE@DBJGBOJC@?$AAs?$AAe?$AAt?$AAl?$AAo?$AAc?$AAa?$AAl?$AAe?$AA?$AA@ 00476500     LIBCMTD:setlocal.obj
 0003:00005518       ??_C@_1FG@OHLFEKMC@?$AAL?$AAC?$AA_?$AAM?$AAI?$AAN?$AA?5?$AA?$DM?$AA?$DN?$AA?5?$AA_?$AAc?$AAa?$AAt?$AAe?$AAg?$AAo?$AAr?$AAy?$AA?5?$AA?$CG?$AA?$CG?$AA?5?$AA_?$AAc?$AAa?$AAt?$AAe?$AAg?$AAo?$AAr?$AAy@ 00476518     LIBCMTD:setlocal.obj
 0003:00005580       ??_C@_1IA@PFIKKKFB@?$AAs?$AAt?$AAr?$AAn?$AAc?$AAp?$AAy?$AA_?$AAs?$AA?$CI?$AAl?$AAc?$AAt?$AAe?$AAm?$AAp?$AA?0?$AA?5?$AA?$CI?$AAs?$AAi?$AAz?$AAe?$AAo?$AAf?$AA?$CI?$AAl?$AAc?$AAt?$AAe?$AAm?$AAp@ 00476580     LIBCMTD:setlocal.obj
 0003:0000561c       ??_C@_1CE@OFNHIOO@?$AA_?$AAs?$AAe?$AAt?$AAl?$AAo?$AAc?$AAa?$AAl?$AAe?$AA_?$AAn?$AAo?$AAl?$AAo?$AAc?$AAk?$AA?$AA@ 0047661c     LIBCMTD:setlocal.obj
 0003:00005648       ??_C@_01ICJEACDI@?$DL?$AA@ 00476648     LIBCMTD:setlocal.obj
 0003:0000564c       ??_C@_02BALPLPBG@?$DN?$DL?$AA@ 0047664c     LIBCMTD:setlocal.obj
 0003:00005650       ??_C@_1GO@JALHLJEH@?$AAs?$AAt?$AAr?$AAc?$AAp?$AAy?$AA_?$AAs?$AA?$CI?$AAp?$AAc?$AAh?$AA?5?$AA?$CL?$AA?5?$AAs?$AAi?$AAz?$AAe?$AAo?$AAf?$AA?$CI?$AAi?$AAn?$AAt?$AA?$CJ?$AA?0?$AA?5?$AAc?$AAc?$AAh?$AA?5@ 00476650     LIBCMTD:setlocal.obj
 0003:000056d4       ??_C@_1CG@IEFIICPK@?$AA_?$AAs?$AAe?$AAt?$AAl?$AAo?$AAc?$AAa?$AAl?$AAe?$AA_?$AAs?$AAe?$AAt?$AA_?$AAc?$AAa?$AAt?$AA?$AA@ 004766d4     LIBCMTD:setlocal.obj
 0003:00005704       ??_C@_1DA@GDKKLCLM@?$AAs?$AAt?$AAr?$AAc?$AAa?$AAt?$AA_?$AAs?$AA?$CI?$AAp?$AAc?$AAh?$AA?0?$AA?5?$AAc?$AAc?$AAh?$AA?0?$AA?5?$AA?$CC?$AA?$DL?$AA?$CC?$AA?$CJ?$AA?$AA@ 00476704     LIBCMTD:setlocal.obj
 0003:00005740       ??_C@_1CG@NNFIJLDA@?$AA_?$AAs?$AAe?$AAt?$AAl?$AAo?$AAc?$AAa?$AAl?$AAe?$AA_?$AAg?$AAe?$AAt?$AA_?$AAa?$AAl?$AAl?$AA?$AA@ 00476740     LIBCMTD:setlocal.obj
 0003:00005770       ??_C@_01NEMOKFLO@?$DN?$AA@ 00476770     LIBCMTD:setlocal.obj
 0003:00005778       ??_C@_1FA@MHAOOIBO@?$AAs?$AAt?$AAr?$AAc?$AAp?$AAy?$AA_?$AAs?$AA?$CI?$AAo?$AAu?$AAt?$AAp?$AAu?$AAt?$AA?0?$AA?5?$AAs?$AAi?$AAz?$AAe?$AAI?$AAn?$AAC?$AAh?$AAa?$AAr?$AAs?$AA?0?$AA?5?$AAc?$AAa@ 00476778     LIBCMTD:setlocal.obj
 0003:000057d8       ??_C@_1IA@ONNFOEDA@?$AAs?$AAt?$AAr?$AAn?$AAc?$AAp?$AAy?$AA_?$AAs?$AA?$CI?$AAc?$AAa?$AAc?$AAh?$AAe?$AAi?$AAn?$AA?0?$AA?5?$AAc?$AAa?$AAc?$AAh?$AAe?$AAi?$AAn?$AAS?$AAi?$AAz?$AAe?$AA?0?$AA?5@ 004767d8     LIBCMTD:setlocal.obj
 0003:00005874       ??_C@_01GFHCPBMG@C?$AA@    00476874     LIBCMTD:setlocal.obj
 0003:00005878       ??_C@_1EG@MOMHKOD@?$AAs?$AAt?$AAr?$AAc?$AAp?$AAy?$AA_?$AAs?$AA?$CI?$AAo?$AAu?$AAt?$AAp?$AAu?$AAt?$AA?0?$AA?5?$AAs?$AAi?$AAz?$AAe?$AAI?$AAn?$AAC?$AAh?$AAa?$AAr?$AAs?$AA?0?$AA?5?$AA?$CC?$AAC@ 00476878     LIBCMTD:setlocal.obj
 0003:000058cc       ??_C@_1BM@OIIBLEFG@?$AA_?$AAe?$AAx?$AAp?$AAa?$AAn?$AAd?$AAl?$AAo?$AAc?$AAa?$AAl?$AAe?$AA?$AA@ 004768cc     LIBCMTD:setlocal.obj
 0003:000058f0       ??_C@_1BGM@IJDLABMC@?$AAs?$AAt?$AAr?$AAc?$AAa?$AAt?$AA_?$AAs?$AA?$CI?$AAo?$AAu?$AAt?$AAs?$AAt?$AAr?$AA?0?$AA?5?$AAs?$AAi?$AAz?$AAe?$AAI?$AAn?$AAB?$AAy?$AAt?$AAe?$AAs?$AA?0?$AA?5?$AA?$CI?$AA?5@ 004768f0     LIBCMTD:setlocal.obj
 0003:00005aa4       ??_C@_1BC@PIABMDIP@?$AA_?$AAs?$AAt?$AAr?$AAc?$AAa?$AAt?$AAs?$AA?$AA@ 00476aa4     LIBCMTD:setlocal.obj
 0003:00005ac0       ??_C@_1MM@NOPMGFHF@?$AAs?$AAt?$AAr?$AAn?$AAc?$AAp?$AAy?$AA_?$AAs?$AA?$CI?$AAn?$AAa?$AAm?$AAe?$AAs?$AA?9?$AA?$DO?$AAs?$AAz?$AAC?$AAo?$AAd?$AAe?$AAP?$AAa?$AAg?$AAe?$AA?0?$AA?5?$AA?$CI?$AAs?$AAi@ 00476ac0     LIBCMTD:setlocal.obj
 0003:00005bb8       ??_C@_1MG@PHNILIAG@?$AAs?$AAt?$AAr?$AAn?$AAc?$AAp?$AAy?$AA_?$AAs?$AA?$CI?$AAn?$AAa?$AAm?$AAe?$AAs?$AA?9?$AA?$DO?$AAs?$AAz?$AAC?$AAo?$AAu?$AAn?$AAt?$AAr?$AAy?$AA?0?$AA?5?$AA?$CI?$AAs?$AAi?$AAz@ 00476bb8     LIBCMTD:setlocal.obj
 0003:00005ca8       ??_C@_1MM@BFEECMAF@?$AAs?$AAt?$AAr?$AAn?$AAc?$AAp?$AAy?$AA_?$AAs?$AA?$CI?$AAn?$AAa?$AAm?$AAe?$AAs?$AA?9?$AA?$DO?$AAs?$AAz?$AAL?$AAa?$AAn?$AAg?$AAu?$AAa?$AAg?$AAe?$AA?0?$AA?5?$AA?$CI?$AAs?$AAi@ 00476ca8     LIBCMTD:setlocal.obj
 0003:00005d9c       ??_C@_03EGDHDPFD@_?4?0?$AA@ 00476d9c     LIBCMTD:setlocal.obj
 0003:00005da0       ??_C@_1NG@FMOPGKGG@?$AAs?$AAt?$AAr?$AAn?$AAc?$AAp?$AAy?$AA_?$AAs?$AA?$CI?$AAn?$AAa?$AAm?$AAe?$AAs?$AA?9?$AA?$DO?$AAs?$AAz?$AAC?$AAo?$AAd?$AAe?$AAP?$AAa?$AAg?$AAe?$AA?0?$AA?5?$AA?$CI?$AAs?$AAi@ 00476da0     LIBCMTD:setlocal.obj
 0003:00005ea0       ??_C@_1BK@CBMMLAGJ@?$AA_?$AA_?$AAl?$AAc?$AA_?$AAs?$AAt?$AAr?$AAt?$AAo?$AAl?$AAc?$AA?$AA@ 00476ea0     LIBCMTD:setlocal.obj
 0003:00005ec0       ??_C@_01LFCBOECM@?4?$AA@   00476ec0     LIBCMTD:setlocal.obj
 0003:00005ec4       ??_C@_01IDAFKMJL@_?$AA@    00476ec4     LIBCMTD:setlocal.obj
 0003:00005ec8       ??_C@_1HC@IBDBLKCB@?$AAs?$AAt?$AAr?$AAc?$AAp?$AAy?$AA_?$AAs?$AA?$CI?$AAl?$AAo?$AAc?$AAa?$AAl?$AAe?$AA?0?$AA?5?$AAs?$AAi?$AAz?$AAe?$AAI?$AAn?$AAB?$AAy?$AAt?$AAe?$AAs?$AA?0?$AA?5?$AA?$CI?$AAc@ 00476ec8     LIBCMTD:setlocal.obj
 0003:00005f50       ??_C@_1BK@FGDJDEPG@?$AA_?$AA_?$AAl?$AAc?$AA_?$AAl?$AAc?$AAt?$AAo?$AAs?$AAt?$AAr?$AA?$AA@ 00476f50     LIBCMTD:setlocal.obj
 0003:00005f70       ??_C@_1GC@CHGJNMHG@?$AAf?$AA?3?$AA?2?$AAd?$AAd?$AA?2?$AAv?$AAc?$AAt?$AAo?$AAo?$AAl?$AAs?$AA?2?$AAc?$AAr?$AAt?$AA_?$AAb?$AAl?$AAd?$AA?2?$AAs?$AAe?$AAl?$AAf?$AA_?$AAx?$AA8?$AA6?$AA?2?$AAc@ 00476f70     LIBCMTD:isctype.obj
 0003:00005fe8       ??_C@_1DC@BPLPALML@?$AA?$CI?$AAu?$AAn?$AAs?$AAi?$AAg?$AAn?$AAe?$AAd?$AA?$CJ?$AA?$CI?$AAc?$AA?5?$AA?$CL?$AA?5?$AA1?$AA?$CJ?$AA?5?$AA?$DM?$AA?$DN?$AA?5?$AA2?$AA5?$AA6?$AA?$AA@ 00476fe8     LIBCMTD:isctype.obj
 0003:00006024       ??_C@_1BG@KCMPBBDK@?$AA_?$AAg?$AAe?$AAt?$AA_?$AAe?$AAr?$AAr?$AAn?$AAo?$AA?$AA@ 00477024     LIBCMTD:dosmap.obj
 0003:00006040       ??_C@_1GA@MFGIMPNL@?$AAf?$AA?3?$AA?2?$AAd?$AAd?$AA?2?$AAv?$AAc?$AAt?$AAo?$AAo?$AAl?$AAs?$AA?2?$AAc?$AAr?$AAt?$AA_?$AAb?$AAl?$AAd?$AA?2?$AAs?$AAe?$AAl?$AAf?$AA_?$AAx?$AA8?$AA6?$AA?2?$AAc@ 00477040     LIBCMTD:dosmap.obj
 0003:000060b4       ??_C@_1BM@INIPHHDD@?$AA_?$AAg?$AAe?$AAt?$AA_?$AAd?$AAo?$AAs?$AAe?$AAr?$AAr?$AAn?$AAo?$AA?$AA@ 004770b4     LIBCMTD:dosmap.obj
 0003:000060d8       ??_C@_0DB@MHMEONEC@f?3?2dd?2vctools?2crt_bld?2self_x86?2c@ 004770d8     LIBCMTD:mbctype.obj
 0003:00006118       ??_C@_1GE@HMAALBPJ@?$AAf?$AA?3?$AA?2?$AAd?$AAd?$AA?2?$AAv?$AAc?$AAt?$AAo?$AAo?$AAl?$AAs?$AA?2?$AAc?$AAr?$AAt?$AA_?$AAb?$AAl?$AAd?$AA?2?$AAs?$AAe?$AAl?$AAf?$AA_?$AAx?$AA8?$AA6?$AA?2?$AAc@ 00477118     LIBCMTD:localref.obj
 0003:00006190       ??_C@_1BKC@GGIENNAK@?$AA?$CI?$AA?$CI?$AAp?$AAt?$AAl?$AAo?$AAc?$AAi?$AA?9?$AA?$DO?$AAl?$AAc?$AA_?$AAc?$AAa?$AAt?$AAe?$AAg?$AAo?$AAr?$AAy?$AA?$FL?$AAc?$AAa?$AAt?$AAe?$AAg?$AAo?$AAr?$AAy?$AA?$FN?$AA?4@ 00477190     LIBCMTD:localref.obj
 0003:00006388       ??_C@_0DA@HMCPFNKN@f?3?2dd?2vctools?2crt_bld?2self_x86?2c@ 00477388     LIBCMTD:onexit.obj
 0003:000063c4       ??_C@_0CP@MKONOLCI@f?3?2dd?2vctools?2crt_bld?2self_x86?2c@ 004773c4     LIBCMTD:mlock.obj
 0003:000063fc       ??_C@_1O@EJLDHPPL@?$AAs?$AAi?$AAg?$AAn?$AAa?$AAl?$AA?$AA@ 004773fc     LIBCMTD:winsig.obj
 0003:00006410       ??_C@_1GA@DBECNFG@?$AAf?$AA?3?$AA?2?$AAd?$AAd?$AA?2?$AAv?$AAc?$AAt?$AAo?$AAo?$AAl?$AAs?$AA?2?$AAc?$AAr?$AAt?$AA_?$AAb?$AAl?$AAd?$AA?2?$AAs?$AAe?$AAl?$AAf?$AA_?$AAx?$AA8?$AA6?$AA?2?$AAc@ 00477410     LIBCMTD:winsig.obj
 0003:00006484       ??_C@_1DO@MLNEDKGB@?$AA?$CI?$AA?$CC?$AAI?$AAn?$AAv?$AAa?$AAl?$AAi?$AAd?$AA?5?$AAs?$AAi?$AAg?$AAn?$AAa?$AAl?$AA?5?$AAo?$AAr?$AA?5?$AAe?$AAr?$AAr?$AAo?$AAr?$AA?$CC?$AA?0?$AA?5?$AA0?$AA?$CJ?$AA?$AA@ 00477484     LIBCMTD:winsig.obj
 0003:000064d0       ??_C@_0DA@ELJOOIJF@f?3?2dd?2vctools?2crt_bld?2self_x86?2c@ 004774d0     LIBCMTD:winsig.obj
 0003:0000650c       ??_C@_1M@DMJEIKHL@?$AAr?$AAa?$AAi?$AAs?$AAe?$AA?$AA@ 0047750c     LIBCMTD:winsig.obj
 0003:0000651c       ??_C@_0BC@JEAENNKH@SystemFunction036?$AA@ 0047751c     LIBCMTD:rand_s.obj
 0003:00006538       ??_C@_1GA@EBEDGGGB@?$AA?$CI?$AA?$CC?$AAr?$AAa?$AAn?$AAd?$AA_?$AAs?$AA?5?$AAi?$AAs?$AA?5?$AAn?$AAo?$AAt?$AA?5?$AAa?$AAv?$AAa?$AAi?$AAl?$AAa?$AAb?$AAl?$AAe?$AA?5?$AAo?$AAn?$AA?5?$AAt?$AAh?$AAi@ 00477538     LIBCMTD:rand_s.obj
 0003:000065ac       ??_C@_1O@IJGPPOGF@?$AAr?$AAa?$AAn?$AAd?$AA_?$AAs?$AA?$AA@ 004775ac     LIBCMTD:rand_s.obj
 0003:000065c0       ??_C@_1GA@HBGBBKCD@?$AAf?$AA?3?$AA?2?$AAd?$AAd?$AA?2?$AAv?$AAc?$AAt?$AAo?$AAo?$AAl?$AAs?$AA?2?$AAc?$AAr?$AAt?$AA_?$AAb?$AAl?$AAd?$AA?2?$AAs?$AAe?$AAl?$AAf?$AA_?$AAx?$AA8?$AA6?$AA?2?$AAc@ 004775c0     LIBCMTD:rand_s.obj
 0003:00006634       ??_C@_1CK@GFDNDKK@?$AA_?$AAR?$AAa?$AAn?$AAd?$AAo?$AAm?$AAV?$AAa?$AAl?$AAu?$AAe?$AA?5?$AA?$CB?$AA?$DN?$AA?5?$AAN?$AAU?$AAL?$AAL?$AA?$AA@ 00477634     LIBCMTD:rand_s.obj
 0003:00006668       ??_C@_1GO@NGIGJNHH@?$AAs?$AAt?$AAr?$AAn?$AAc?$AAp?$AAy?$AA_?$AAs?$AA?$CI?$AA?$CK?$AAs?$AAt?$AAr?$AAa?$AAd?$AAd?$AAr?$AAe?$AAs?$AAs?$AA?0?$AA?5?$AAo?$AAu?$AAt?$AAs?$AAi?$AAz?$AAe?$AA?0?$AA?5@ 00477668     LIBCMTD:inithelp.obj
 0003:000066ec       ??_C@_1CA@KHHCPEI@?$AA_?$AA_?$AAg?$AAe?$AAt?$AAl?$AAo?$AAc?$AAa?$AAl?$AAe?$AAi?$AAn?$AAf?$AAo?$AA?$AA@ 004776ec     LIBCMTD:inithelp.obj
 0003:00006718       ??_C@_1GE@PLPIMDHG@?$AAf?$AA?3?$AA?2?$AAd?$AAd?$AA?2?$AAv?$AAc?$AAt?$AAo?$AAo?$AAl?$AAs?$AA?2?$AAc?$AAr?$AAt?$AA_?$AAb?$AAl?$AAd?$AA?2?$AAs?$AAe?$AAl?$AAf?$AA_?$AAx?$AA8?$AA6?$AA?2?$AAc@ 00477718     LIBCMTD:inithelp.obj
 0003:00006790       ??_C@_0DC@CFDMMFIG@f?3?2dd?2vctools?2crt_bld?2self_x86?2c@ 00477790     LIBCMTD:inithelp.obj
 0003:000067d0       ??_C@_1GG@CDHAPCGF@?$AAf?$AA?3?$AA?2?$AAd?$AAd?$AA?2?$AAv?$AAc?$AAt?$AAo?$AAo?$AAl?$AAs?$AA?2?$AAc?$AAr?$AAt?$AA_?$AAb?$AAl?$AAd?$AA?2?$AAs?$AAe?$AAl?$AAf?$AA_?$AAx?$AA8?$AA6?$AA?2?$AAc@ 004777d0     LIBCMTD:handler.obj
 0003:0000684c       ??_C@_1BC@JLLICHIC@?$AAp?$AAn?$AAh?$AA?5?$AA?$DN?$AA?$DN?$AA?5?$AA0?$AA?$AA@ 0047784c     LIBCMTD:handler.obj
 0003:00006864       ??_C@_1DM@MADKGDLO@?$AA?$CI?$AAL?$AA?$CC?$AAB?$AAu?$AAf?$AAf?$AAe?$AAr?$AA?5?$AAi?$AAs?$AA?5?$AAt?$AAo?$AAo?$AA?5?$AAs?$AAm?$AAa?$AAl?$AAl?$AA?$CC?$AA?5?$AA?$CG?$AA?$CG?$AA?5?$AA0?$AA?$CJ?$AA?$AA@ 00477864     LIBCMTD:strcpy_s.obj
 0003:000068ac       ??_C@_1CI@HCPHDDLE@?$AAB?$AAu?$AAf?$AAf?$AAe?$AAr?$AA?5?$AAi?$AAs?$AA?5?$AAt?$AAo?$AAo?$AA?5?$AAs?$AAm?$AAa?$AAl?$AAl?$AA?$AA@ 004778ac     LIBCMTD:strcpy_s.obj
 0003:000068dc       ??_C@_1CG@OFBJMIGJ@?$AA?$CI?$AA?$CI?$AA?$CI?$AA_?$AAS?$AAr?$AAc?$AA?$CJ?$AA?$CJ?$AA?$CJ?$AA?5?$AA?$CB?$AA?$DN?$AA?5?$AAN?$AAU?$AAL?$AAL?$AA?$AA@ 004778dc     LIBCMTD:strcpy_s.obj
 0003:0000690c       ??_C@_1BC@CFJEPFGF@?$AAs?$AAt?$AAr?$AAc?$AAp?$AAy?$AA_?$AAs?$AA?$AA@ 0047790c     LIBCMTD:strcpy_s.obj
 0003:00006928       ??_C@_1GI@BGBNCIMA@?$AAf?$AA?3?$AA?2?$AAd?$AAd?$AA?2?$AAv?$AAc?$AAt?$AAo?$AAo?$AAl?$AAs?$AA?2?$AAc?$AAr?$AAt?$AA_?$AAb?$AAl?$AAd?$AA?2?$AAs?$AAe?$AAl?$AAf?$AA_?$AAx?$AA8?$AA6?$AA?2?$AAc@ 00477928     LIBCMTD:strcpy_s.obj
 0003:000069a8       ??_C@_1FC@NCPEPIBI@?$AA?$CI?$AA?$CI?$AA_?$AAD?$AAs?$AAt?$AA?$CJ?$AA?$CJ?$AA?5?$AA?$CB?$AA?$DN?$AA?5?$AAN?$AAU?$AAL?$AAL?$AA?5?$AA?$CG?$AA?$CG?$AA?5?$AA?$CI?$AA?$CI?$AA_?$AAS?$AAi?$AAz?$AAe?$AAI?$AAn?$AAB?$AAy?$AAt@ 004779a8     LIBCMTD:strcpy_s.obj
 0003:00006a0c       ??_C@_1BK@JMCGJOCC@?$AA_?$AAe?$AAx?$AAp?$AAa?$AAn?$AAd?$AA_?$AAb?$AAa?$AAs?$AAe?$AA?$AA@ 00477a0c     LIBCMTD:expand.obj
 0003:00006a30       ??_C@_1GA@EBHFLDNH@?$AAf?$AA?3?$AA?2?$AAd?$AAd?$AA?2?$AAv?$AAc?$AAt?$AAo?$AAo?$AAl?$AAs?$AA?2?$AAc?$AAr?$AAt?$AA_?$AAb?$AAl?$AAd?$AA?2?$AAs?$AAe?$AAl?$AAf?$AA_?$AAx?$AA8?$AA6?$AA?2?$AAc@ 00477a30     LIBCMTD:expand.obj
 0003:00006aa4       ??_C@_1BO@KFIJIAEA@?$AAp?$AAB?$AAl?$AAo?$AAc?$AAk?$AA?5?$AA?$CB?$AA?$DN?$AA?5?$AAN?$AAU?$AAL?$AAL?$AA?$AA@ 00477aa4     LIBCMTD:expand.obj
 0003:00006ac8       ??_C@_1CC@OLIJCKA@?$AA?$CI?$AAs?$AAt?$AAr?$AAi?$AAn?$AAg?$AA?5?$AA?$CB?$AA?$DN?$AA?5?$AAN?$AAU?$AAL?$AAL?$AA?$CJ?$AA?$AA@ 00477ac8     LIBCMTD:sprintf.obj
 0003:00006af0       ??_C@_1BA@KBJJGFFE@?$AAs?$AAp?$AAr?$AAi?$AAn?$AAt?$AAf?$AA?$AA@ 00477af0     LIBCMTD:sprintf.obj
 0003:00006b08       ??_C@_1GC@BMNPEKNN@?$AAf?$AA?3?$AA?2?$AAd?$AAd?$AA?2?$AAv?$AAc?$AAt?$AAo?$AAo?$AAl?$AAs?$AA?2?$AAc?$AAr?$AAt?$AA_?$AAb?$AAl?$AAd?$AA?2?$AAs?$AAe?$AAl?$AAf?$AA_?$AAx?$AA8?$AA6?$AA?2?$AAc@ 00477b08     LIBCMTD:sprintf.obj
 0003:00006b80       ??_C@_1CC@MGIEJOME@?$AA?$CI?$AAf?$AAo?$AAr?$AAm?$AAa?$AAt?$AA?5?$AA?$CB?$AA?$DN?$AA?5?$AAN?$AAU?$AAL?$AAL?$AA?$CJ?$AA?$AA@ 00477b80     LIBCMTD:sprintf.obj
 0003:00006ba8       ??_C@_1CA@LFDHAMEM@?$AA_?$AAs?$AAe?$AAt?$AA_?$AAe?$AAr?$AAr?$AAo?$AAr?$AA_?$AAm?$AAo?$AAd?$AAe?$AA?$AA@ 00477ba8     LIBCMTD:errmode.obj
 0003:00006bd0       ??_C@_1GC@FGMGFCNB@?$AAf?$AA?3?$AA?2?$AAd?$AAd?$AA?2?$AAv?$AAc?$AAt?$AAo?$AAo?$AAl?$AAs?$AA?2?$AAc?$AAr?$AAt?$AA_?$AAb?$AAl?$AAd?$AA?2?$AAs?$AAe?$AAl?$AAf?$AA_?$AAx?$AA8?$AA6?$AA?2?$AAc@ 00477bd0     LIBCMTD:errmode.obj
 0003:00006c48       ??_C@_1DE@BCNCAIK@?$AA?$CI?$AA?$CC?$AAI?$AAn?$AAv?$AAa?$AAl?$AAi?$AAd?$AA?5?$AAe?$AAr?$AAr?$AAo?$AAr?$AA_?$AAm?$AAo?$AAd?$AAe?$AA?$CC?$AA?0?$AA?5?$AA0?$AA?$CJ?$AA?$AA@ 00477c48     LIBCMTD:errmode.obj
 0003:00006c88       ??_C@_0BI@DFKBFLJE@GetProcessWindowStation?$AA@ 00477c88     LIBCMTD:crtmboxw.obj
 0003:00006ca4       ??_C@_0BK@DEKFELLI@GetUserObjectInformationW?$AA@ 00477ca4     LIBCMTD:crtmboxw.obj
 0003:00006cc4       ??_C@_0BD@HHGDFDBJ@GetLastActivePopup?$AA@ 00477cc4     LIBCMTD:crtmboxw.obj
 0003:00006cdc       ??_C@_0BA@HNOPNCHB@GetActiveWindow?$AA@ 00477cdc     LIBCMTD:crtmboxw.obj
 0003:00006cf0       ??_C@_0M@DLDCCGNP@MessageBoxW?$AA@ 00477cf0     LIBCMTD:crtmboxw.obj
 0003:00006d00       ??_C@_1BG@GOEBHBDC@?$AAU?$AAS?$AAE?$AAR?$AA3?$AA2?$AA?4?$AAD?$AAL?$AAL?$AA?$AA@ 00477d00     LIBCMTD:crtmboxw.obj
 0003:00006d20       ??_C@_1FA@MJKDNFFB@?$AA?$CI?$AAL?$AA?$CC?$AAS?$AAt?$AAr?$AAi?$AAn?$AAg?$AA?5?$AAi?$AAs?$AA?5?$AAn?$AAo?$AAt?$AA?5?$AAn?$AAu?$AAl?$AAl?$AA?5?$AAt?$AAe?$AAr?$AAm?$AAi?$AAn?$AAa?$AAt?$AAe?$AAd@ 00477d20     LIBCMTD:wcscat_s.obj
 0003:00006d80       ??_C@_1DM@FHLMIEG@?$AAS?$AAt?$AAr?$AAi?$AAn?$AAg?$AA?5?$AAi?$AAs?$AA?5?$AAn?$AAo?$AAt?$AA?5?$AAn?$AAu?$AAl?$AAl?$AA?5?$AAt?$AAe?$AAr?$AAm?$AAi?$AAn?$AAa?$AAt?$AAe?$AAd?$AA?$AA@ 00477d80     LIBCMTD:wcscat_s.obj
 0003:00006dc8       ??_C@_1BC@PLIEPKPJ@?$AAw?$AAc?$AAs?$AAc?$AAa?$AAt?$AA_?$AAs?$AA?$AA@ 00477dc8     LIBCMTD:wcscat_s.obj
 0003:00006de0       ??_C@_1GI@NOKGIAGA@?$AAf?$AA?3?$AA?2?$AAd?$AAd?$AA?2?$AAv?$AAc?$AAt?$AAo?$AAo?$AAl?$AAs?$AA?2?$AAc?$AAr?$AAt?$AA_?$AAb?$AAl?$AAd?$AA?2?$AAs?$AAe?$AAl?$AAf?$AA_?$AAx?$AA8?$AA6?$AA?2?$AAc@ 00477de0     LIBCMTD:wcscat_s.obj
 0003:00006e60       ??_C@_1FC@PFMLEHKI@?$AA?$CI?$AA?$CI?$AA_?$AAD?$AAs?$AAt?$AA?$CJ?$AA?$CJ?$AA?5?$AA?$CB?$AA?$DN?$AA?5?$AAN?$AAU?$AAL?$AAL?$AA?5?$AA?$CG?$AA?$CG?$AA?5?$AA?$CI?$AA?$CI?$AA_?$AAS?$AAi?$AAz?$AAe?$AAI?$AAn?$AAW?$AAo?$AAr@ 00477e60     LIBCMTD:wcscat_s.obj
 0003:00006ec4       ??_C@_1BE@PMMBFFCC@?$AAw?$AAc?$AAs?$AAn?$AAc?$AAp?$AAy?$AA_?$AAs?$AA?$AA@ 00477ec4     LIBCMTD:wcsncpy_s.obj
 0003:00006ee0       ??_C@_1GK@PAJJBKJF@?$AAf?$AA?3?$AA?2?$AAd?$AAd?$AA?2?$AAv?$AAc?$AAt?$AAo?$AAo?$AAl?$AAs?$AA?2?$AAc?$AAr?$AAt?$AA_?$AAb?$AAl?$AAd?$AA?2?$AAs?$AAe?$AAl?$AAf?$AA_?$AAx?$AA8?$AA6?$AA?2?$AAc@ 00477ee0     LIBCMTD:wcsncpy_s.obj
 0003:00006f60       ??_C@_1BC@KIONAFPO@?$AAw?$AAc?$AAs?$AAc?$AAp?$AAy?$AA_?$AAs?$AA?$AA@ 00477f60     LIBCMTD:wcscpy_s.obj
 0003:00006f78       ??_C@_1NK@LOFHIHFC@?$AAf?$AAM?$AAo?$AAd?$AAe?$AA?5?$AA?$DN?$AA?$DN?$AA?5?$AA_?$AAC?$AAR?$AAT?$AAD?$AAB?$AAG?$AA_?$AAR?$AAE?$AAP?$AAO?$AAR?$AAT?$AA_?$AAM?$AAO?$AAD?$AAE?$AA?5?$AA?$HM?$AA?$HM?$AA?5@ 00477f78     LIBCMTD:dbgrptt.obj
 0003:00007080       ??_C@_1CE@FIHIECNJ@?$AA_?$AAC?$AAr?$AAt?$AAS?$AAe?$AAt?$AAR?$AAe?$AAp?$AAo?$AAr?$AAt?$AAM?$AAo?$AAd?$AAe?$AA?$AA@ 00478080     LIBCMTD:dbgrptt.obj
 0003:000070b0       ??_C@_1GC@FIGJJMEN@?$AAf?$AA?3?$AA?2?$AAd?$AAd?$AA?2?$AAv?$AAc?$AAt?$AAo?$AAo?$AAl?$AAs?$AA?2?$AAc?$AAr?$AAt?$AA_?$AAb?$AAl?$AAd?$AA?2?$AAs?$AAe?$AAl?$AAf?$AA_?$AAx?$AA8?$AA6?$AA?2?$AAc@ 004780b0     LIBCMTD:dbgrptt.obj
 0003:00007128       ??_C@_1FA@IFFFOLDJ@?$AAn?$AAR?$AAp?$AAt?$AAT?$AAy?$AAp?$AAe?$AA?5?$AA?$DO?$AA?$DN?$AA?5?$AA0?$AA?5?$AA?$CG?$AA?$CG?$AA?5?$AAn?$AAR?$AAp?$AAt?$AAT?$AAy?$AAp?$AAe?$AA?5?$AA?$DM?$AA?5?$AA_?$AAC?$AAR?$AAT@ 00478128     LIBCMTD:dbgrptt.obj
 0003:00007188       ??_C@_1CE@IKKEDCME@?$AA_?$AAC?$AAr?$AAt?$AAS?$AAe?$AAt?$AAR?$AAe?$AAp?$AAo?$AAr?$AAt?$AAF?$AAi?$AAl?$AAe?$AA?$AA@ 00478188     LIBCMTD:dbgrptt.obj
 0003:000071b8       ??_C@_1HO@PJOFIKFE@?$AA_?$AAC?$AAr?$AAt?$AAD?$AAb?$AAg?$AAR?$AAe?$AAp?$AAo?$AAr?$AAt?$AA?3?$AA?5?$AAS?$AAt?$AAr?$AAi?$AAn?$AAg?$AA?5?$AAt?$AAo?$AAo?$AA?5?$AAl?$AAo?$AAn?$AAg?$AA?5?$AAo@ 004781b8     LIBCMTD:dbgrptt.obj
 0003:00007250       ??_C@_1MC@IGEECMDB@?$AAw?$AAc?$AAs?$AAc?$AAp?$AAy?$AA_?$AAs?$AA?$CI?$AAs?$AAz?$AAO?$AAu?$AAt?$AAM?$AAe?$AAs?$AAs?$AAa?$AAg?$AAe?$AA2?$AA?0?$AA?5?$AA4?$AA0?$AA9?$AA6?$AA?0?$AA?5?$AAL?$AA?$CC@ 00478250     LIBCMTD:dbgrptt.obj
 0003:00007338       ??_C@_1IM@OOKIFKOH@?$AAe?$AA?5?$AA?$DN?$AA?5?$AAm?$AAb?$AAs?$AAt?$AAo?$AAw?$AAc?$AAs?$AA_?$AAs?$AA?$CI?$AA?$CG?$AAr?$AAe?$AAt?$AA?0?$AA?5?$AAs?$AAz?$AAO?$AAu?$AAt?$AAM?$AAe?$AAs?$AAs?$AAa?$AAg@ 00478338     LIBCMTD:dbgrptt.obj
 0003:000073e0       ??_C@_1FI@IBIOIHEG@?$AAs?$AAt?$AAr?$AAc?$AAp?$AAy?$AA_?$AAs?$AA?$CI?$AAs?$AAz?$AAO?$AAu?$AAt?$AAM?$AAe?$AAs?$AAs?$AAa?$AAg?$AAe?$AA?0?$AA?5?$AA4?$AA0?$AA9?$AA6?$AA?0?$AA?5?$AAs?$AAz?$AAL@ 004783e0     LIBCMTD:dbgrptt.obj
 0003:0000744c       ??_C@_0M@IPILFDFN@?$CFs?$CI?$CFd?$CJ?5?3?5?$CFs?$AA@ 0047844c     LIBCMTD:dbgrptt.obj
 0003:00007460       ??_C@_1EI@LDHJEDO@?$AAs?$AAt?$AAr?$AAc?$AAa?$AAt?$AA_?$AAs?$AA?$CI?$AAs?$AAz?$AAL?$AAi?$AAn?$AAe?$AAM?$AAe?$AAs?$AAs?$AAa?$AAg?$AAe?$AA?0?$AA?5?$AA4?$AA0?$AA9?$AA6?$AA?0?$AA?5?$AA?$CC?$AA?2@ 00478460     LIBCMTD:dbgrptt.obj
 0003:000074b8       ??_C@_01LIIJDEN@?$AN?$AA@  004784b8     LIBCMTD:dbgrptt.obj
 0003:000074c0       ??_C@_1EI@CACDLAFK@?$AAs?$AAt?$AAr?$AAc?$AAa?$AAt?$AA_?$AAs?$AA?$CI?$AAs?$AAz?$AAL?$AAi?$AAn?$AAe?$AAM?$AAe?$AAs?$AAs?$AAa?$AAg?$AAe?$AA?0?$AA?5?$AA4?$AA0?$AA9?$AA6?$AA?0?$AA?5?$AA?$CC?$AA?2@ 004784c0     LIBCMTD:dbgrptt.obj
 0003:00007518       ??_C@_1FK@NPGBPOFO@?$AAs?$AAt?$AAr?$AAc?$AAa?$AAt?$AA_?$AAs?$AA?$CI?$AAs?$AAz?$AAL?$AAi?$AAn?$AAe?$AAM?$AAe?$AAs?$AAs?$AAa?$AAg?$AAe?$AA?0?$AA?5?$AA4?$AA0?$AA9?$AA6?$AA?0?$AA?5?$AAs?$AAz@ 00478518     LIBCMTD:dbgrptt.obj
 0003:00007588       ??_C@_1KK@GIGAEDMO@?$AAs?$AAt?$AAr?$AAc?$AAp?$AAy?$AA_?$AAs?$AA?$CI?$AAs?$AAz?$AAL?$AAi?$AAn?$AAe?$AAM?$AAe?$AAs?$AAs?$AAa?$AAg?$AAe?$AA?0?$AA?5?$AA4?$AA0?$AA9?$AA6?$AA?0?$AA?5?$AAs?$AAz@ 00478588     LIBCMTD:dbgrptt.obj
 0003:00007654       ??_C@_0BC@LAIDCHCH@Assertion?5failed?$CB?$AA@ 00478654     LIBCMTD:dbgrptt.obj
 0003:0000766c       ??_C@_0BD@CAENFOHP@Assertion?5failed?3?5?$AA@ 0047866c     LIBCMTD:dbgrptt.obj
 0003:00007688       ??_C@_1JI@GAALPGBM@?$AAs?$AAt?$AAr?$AAc?$AAp?$AAy?$AA_?$AAs?$AA?$CI?$AAs?$AAz?$AAU?$AAs?$AAe?$AAr?$AAM?$AAe?$AAs?$AAs?$AAa?$AAg?$AAe?$AA?0?$AA?5?$AA4?$AA0?$AA9?$AA6?$AA?0?$AA?5?$AA?$CC?$AA_@ 00478688     LIBCMTD:dbgrptt.obj
 0003:00007740       ??_C@_07BHGABMGB@?0?5Line?5?$AA@ 00478740     LIBCMTD:dbgrptt.obj
 0003:0000774c       ??_C@_0P@DFJNDPOP@?$DMfile?5unknown?$DO?$AA@ 0047874c     LIBCMTD:dbgrptt.obj
 0003:00007760       ??_C@_0CG@BNGLOCEO@Second?5Chance?5Assertion?5Failed?3?5@ 00478760     LIBCMTD:dbgrptt.obj
 0003:00007790       ??_C@_1FA@JPHJBHEM@?$AA_?$AAi?$AAt?$AAo?$AAa?$AA_?$AAs?$AA?$CI?$AAn?$AAL?$AAi?$AAn?$AAe?$AA?0?$AA?5?$AAs?$AAz?$AAL?$AAi?$AAn?$AAe?$AAM?$AAe?$AAs?$AAs?$AAa?$AAg?$AAe?$AA?0?$AA?5?$AA4?$AA0@ 00478790     LIBCMTD:dbgrptt.obj
 0003:000077f0       ??_C@_1CA@KHJHLKA@?$AA_?$AAV?$AAC?$AAr?$AAt?$AAD?$AAb?$AAg?$AAR?$AAe?$AAp?$AAo?$AAr?$AAt?$AAA?$AA?$AA@ 004787f0     LIBCMTD:dbgrptt.obj
 0003:00007818       ??_C@_1IE@CPGKIAGP@?$AAw?$AAc?$AAs?$AAt?$AAo?$AAm?$AAb?$AAs?$AA_?$AAs?$AA?$CI?$AA?$CG?$AAr?$AAe?$AAt?$AA?0?$AA?5?$AAs?$AAz?$AAa?$AAO?$AAu?$AAt?$AAM?$AAe?$AAs?$AAs?$AAa?$AAg?$AAe?$AA?0?$AA?5@ 00478818     LIBCMTD:dbgrptt.obj
 0003:000078b8       ??_C@_0DP@GNPEPHJD@_CrtDbgReport?3?5String?5too?5long?5o@ 004788b8     LIBCMTD:dbgrptt.obj
 0003:00007908       ??_C@_1MA@LBAMNNOB@?$AAs?$AAt?$AAr?$AAc?$AAp?$AAy?$AA_?$AAs?$AA?$CI?$AAs?$AAz?$AAO?$AAu?$AAt?$AAM?$AAe?$AAs?$AAs?$AAa?$AAg?$AAe?$AA2?$AA?0?$AA?5?$AA4?$AA0?$AA9?$AA6?$AA?0?$AA?5?$AA?$CC?$AA_@ 00478908     LIBCMTD:dbgrptt.obj
 0003:000079f0       ??_C@_1JC@EOAPFDLN@?$AAw?$AAc?$AAs?$AAt?$AAo?$AAm?$AAb?$AAs?$AA_?$AAs?$AA?$CI?$AA?$CI?$AA?$CI?$AAv?$AAo?$AAi?$AAd?$AA?5?$AA?$CK?$AA?$CJ?$AA0?$AA?$CJ?$AA?0?$AA?5?$AAs?$AAz?$AAO?$AAu?$AAt?$AAM?$AAe?$AAs@ 004789f0     LIBCMTD:dbgrptt.obj
 0003:00007aa0       ??_C@_1FI@DBAIJPJE@?$AAw?$AAc?$AAs?$AAc?$AAp?$AAy?$AA_?$AAs?$AA?$CI?$AAs?$AAz?$AAO?$AAu?$AAt?$AAM?$AAe?$AAs?$AAs?$AAa?$AAg?$AAe?$AA?0?$AA?5?$AA4?$AA0?$AA9?$AA6?$AA?0?$AA?5?$AAs?$AAz?$AAL@ 00478aa0     LIBCMTD:dbgrptt.obj
 0003:00007b0c       ??_C@_1BI@JIDBEPIG@?$AA?$CF?$AAs?$AA?$CI?$AA?$CF?$AAd?$AA?$CJ?$AA?5?$AA?3?$AA?5?$AA?$CF?$AAs?$AA?$AA@ 00478b0c     LIBCMTD:dbgrptt.obj
 0003:00007b28       ??_C@_1EK@PHCBEDKB@?$AAw?$AAc?$AAs?$AAc?$AAa?$AAt?$AA_?$AAs?$AA?$CI?$AAs?$AAz?$AAL?$AAi?$AAn?$AAe?$AAM?$AAe?$AAs?$AAs?$AAa?$AAg?$AAe?$AA?0?$AA?5?$AA4?$AA0?$AA9?$AA6?$AA?0?$AA?5?$AAL?$AA?$CC@ 00478b28     LIBCMTD:dbgrptt.obj
 0003:00007b80       ??_C@_13CMNBPIDO@?$AA?$AN?$AA?$AA@ 00478b80     LIBCMTD:dbgrptt.obj
 0003:00007b88       ??_C@_1EK@NMDFGHMF@?$AAw?$AAc?$AAs?$AAc?$AAa?$AAt?$AA_?$AAs?$AA?$CI?$AAs?$AAz?$AAL?$AAi?$AAn?$AAe?$AAM?$AAe?$AAs?$AAs?$AAa?$AAg?$AAe?$AA?0?$AA?5?$AA4?$AA0?$AA9?$AA6?$AA?0?$AA?5?$AAL?$AA?$CC@ 00478b88     LIBCMTD:dbgrptt.obj
 0003:00007be0       ??_C@_1FK@HPADHBBD@?$AAw?$AAc?$AAs?$AAc?$AAa?$AAt?$AA_?$AAs?$AA?$CI?$AAs?$AAz?$AAL?$AAi?$AAn?$AAe?$AAM?$AAe?$AAs?$AAs?$AAa?$AAg?$AAe?$AA?0?$AA?5?$AA4?$AA0?$AA9?$AA6?$AA?0?$AA?5?$AAs?$AAz@ 00478be0     LIBCMTD:dbgrptt.obj
 0003:00007c50       ??_C@_1KO@DGAHENCH@?$AAw?$AAc?$AAs?$AAc?$AAp?$AAy?$AA_?$AAs?$AA?$CI?$AAs?$AAz?$AAL?$AAi?$AAn?$AAe?$AAM?$AAe?$AAs?$AAs?$AAa?$AAg?$AAe?$AA?0?$AA?5?$AA4?$AA0?$AA9?$AA6?$AA?0?$AA?5?$AAs?$AAz@ 00478c50     LIBCMTD:dbgrptt.obj
 0003:00007d20       ??_C@_1CE@OJBNHDMO@?$AAA?$AAs?$AAs?$AAe?$AAr?$AAt?$AAi?$AAo?$AAn?$AA?5?$AAf?$AAa?$AAi?$AAl?$AAe?$AAd?$AA?$CB?$AA?$AA@ 00478d20     LIBCMTD:dbgrptt.obj
 0003:00007d4c       ??_C@_1CG@FFFGGODN@?$AAA?$AAs?$AAs?$AAe?$AAr?$AAt?$AAi?$AAo?$AAn?$AA?5?$AAf?$AAa?$AAi?$AAl?$AAe?$AAd?$AA?3?$AA?5?$AA?$AA@ 00478d4c     LIBCMTD:dbgrptt.obj
 0003:00007d80       ??_C@_1JK@KHFABAEO@?$AAw?$AAc?$AAs?$AAc?$AAp?$AAy?$AA_?$AAs?$AA?$CI?$AAs?$AAz?$AAU?$AAs?$AAe?$AAr?$AAM?$AAe?$AAs?$AAs?$AAa?$AAg?$AAe?$AA?0?$AA?5?$AA4?$AA0?$AA9?$AA6?$AA?0?$AA?5?$AAL?$AA?$CC@ 00478d80     LIBCMTD:dbgrptt.obj
 0003:00007e38       ??_C@_13LBAGMAIH@?$AA?6?$AA?$AA@ 00478e38     LIBCMTD:dbgrptt.obj
 0003:00007e3c       ??_C@_1BA@ELMMDCFC@?$AA?0?$AA?5?$AAL?$AAi?$AAn?$AAe?$AA?5?$AA?$AA@ 00478e3c     LIBCMTD:dbgrptt.obj
 0003:00007e50       ??_C@_1BO@OCHMLCAG@?$AA?$DM?$AAf?$AAi?$AAl?$AAe?$AA?5?$AAu?$AAn?$AAk?$AAn?$AAo?$AAw?$AAn?$AA?$DO?$AA?$AA@ 00478e50     LIBCMTD:dbgrptt.obj
 0003:00007e78       ??_C@_1EM@MJFLEDMB@?$AAS?$AAe?$AAc?$AAo?$AAn?$AAd?$AA?5?$AAC?$AAh?$AAa?$AAn?$AAc?$AAe?$AA?5?$AAA?$AAs?$AAs?$AAe?$AAr?$AAt?$AAi?$AAo?$AAn?$AA?5?$AAF?$AAa?$AAi?$AAl?$AAe?$AAd?$AA?3?$AA?5@ 00478e78     LIBCMTD:dbgrptt.obj
 0003:00007ed8       ??_C@_1FA@CNLLOMHI@?$AA_?$AAi?$AAt?$AAo?$AAw?$AA_?$AAs?$AA?$CI?$AAn?$AAL?$AAi?$AAn?$AAe?$AA?0?$AA?5?$AAs?$AAz?$AAL?$AAi?$AAn?$AAe?$AAM?$AAe?$AAs?$AAs?$AAa?$AAg?$AAe?$AA?0?$AA?5?$AA4?$AA0@ 00478ed8     LIBCMTD:dbgrptt.obj
 0003:00007f38       ??_C@_1CA@HPALHDOD@?$AA_?$AAV?$AAC?$AAr?$AAt?$AAD?$AAb?$AAg?$AAR?$AAe?$AAp?$AAo?$AAr?$AAt?$AAW?$AA?$AA@ 00478f38     LIBCMTD:dbgrptt.obj
 0003:00007f60       ??_C@_0BK@CIDNPOGP@GetUserObjectInformationA?$AA@ 00478f60     LIBCMTD:crtmbox.obj
 0003:00007f80       ??_C@_0M@CHKKJDAI@MessageBoxA?$AA@ 00478f80     LIBCMTD:crtmbox.obj
 0003:00007f90       ??_C@_1CK@DDKKOLAN@?$AAs?$AAi?$AAz?$AAe?$AAI?$AAn?$AAB?$AAy?$AAt?$AAe?$AAs?$AA?5?$AA?$DO?$AA?$DN?$AA?5?$AAc?$AAo?$AAu?$AAn?$AAt?$AA?$AA@ 00478f90     LIBCMTD:memcpy_s.obj
 0003:00007fc4       ??_C@_1BI@DCHLDCPP@?$AAs?$AAr?$AAc?$AA?5?$AA?$CB?$AA?$DN?$AA?5?$AAN?$AAU?$AAL?$AAL?$AA?$AA@ 00478fc4     LIBCMTD:memcpy_s.obj
 0003:00007fe0       ??_C@_1BC@GKHDJMGB@?$AAm?$AAe?$AAm?$AAc?$AAp?$AAy?$AA_?$AAs?$AA?$AA@ 00478fe0     LIBCMTD:memcpy_s.obj
 0003:00007ff8       ??_C@_1GE@NEOPGGBM@?$AAf?$AA?3?$AA?2?$AAd?$AAd?$AA?2?$AAv?$AAc?$AAt?$AAo?$AAo?$AAl?$AAs?$AA?2?$AAc?$AAr?$AAt?$AA_?$AAb?$AAl?$AAd?$AA?2?$AAs?$AAe?$AAl?$AAf?$AA_?$AAx?$AA8?$AA6?$AA?2?$AAc@ 00478ff8     LIBCMTD:memcpy_s.obj
 0003:00008070       ??_C@_1BI@GKKCBDMD@?$AAd?$AAs?$AAt?$AA?5?$AA?$CB?$AA?$DN?$AA?5?$AAN?$AAU?$AAL?$AAL?$AA?$AA@ 00479070     LIBCMTD:memcpy_s.obj
 0003:0000808c       ??_C@_1BE@BMIJMLDD@?$AA_?$AAs?$AAw?$AAp?$AAr?$AAi?$AAn?$AAt?$AAf?$AA?$AA@ 0047908c     LIBCMTD:swprintf.obj
 0003:000080a8       ??_C@_1GE@DKGHLBLP@?$AAf?$AA?3?$AA?2?$AAd?$AAd?$AA?2?$AAv?$AAc?$AAt?$AAo?$AAo?$AAl?$AAs?$AA?2?$AAc?$AAr?$AAt?$AA_?$AAb?$AAl?$AAd?$AA?2?$AAs?$AAe?$AAl?$AAf?$AA_?$AAx?$AA8?$AA6?$AA?2?$AAc@ 004790a8     LIBCMTD:swprintf.obj
 0003:00008120       ___newctype                00479120     LIBCMTD:ctype.obj
 0003:00008420       __wctype                   00479420     LIBCMTD:ctype.obj
 0003:00008628       ___newclmap                00479628     LIBCMTD:ctype.obj
 0003:000087a8       ___newcumap                004797a8     LIBCMTD:ctype.obj
 0003:00008ac8       ??_C@_1GE@GJCMHHMH@?$AAf?$AA?3?$AA?2?$AAd?$AAd?$AA?2?$AAv?$AAc?$AAt?$AAo?$AAo?$AAl?$AAs?$AA?2?$AAc?$AAr?$AAt?$AA_?$AAb?$AAl?$AAd?$AA?2?$AAs?$AAe?$AAl?$AAf?$AA_?$AAx?$AA8?$AA6?$AA?2?$AAc@ 00479ac8     LIBCMTD:inittime.obj
 0003:00008b40       ??_C@_1EE@FDHCFDHN@?$AAp?$AAl?$AAo?$AAc?$AAi?$AA?9?$AA?$DO?$AAl?$AAc?$AA_?$AAt?$AAi?$AAm?$AAe?$AA_?$AAc?$AAu?$AAr?$AAr?$AA?9?$AA?$DO?$AAr?$AAe?$AAf?$AAc?$AAo?$AAu?$AAn?$AAt?$AA?5?$AA?$DO?$AA?5@ 00479b40     LIBCMTD:inittime.obj
 0003:00008b94       ??_C@_0DC@KICHHNFK@f?3?2dd?2vctools?2crt_bld?2self_x86?2c@ 00479b94     LIBCMTD:inittime.obj
 0003:00008bd0       ??_C@_1GC@EDJOCBCL@?$AAf?$AA?3?$AA?2?$AAd?$AAd?$AA?2?$AAv?$AAc?$AAt?$AAo?$AAo?$AAl?$AAs?$AA?2?$AAc?$AAr?$AAt?$AA_?$AAb?$AAl?$AAd?$AA?2?$AAs?$AAe?$AAl?$AAf?$AA_?$AAx?$AA8?$AA6?$AA?2?$AAc@ 00479bd0     LIBCMTD:initnum.obj
 0003:00008c48       ??_C@_1DM@IFKAINNE@?$AAp?$AAl?$AAo?$AAc?$AAi?$AA?9?$AA?$DO?$AAl?$AAc?$AAo?$AAn?$AAv?$AA_?$AAn?$AAu?$AAm?$AA_?$AAr?$AAe?$AAf?$AAc?$AAo?$AAu?$AAn?$AAt?$AA?5?$AA?$DO?$AA?5?$AA0?$AA?$AA@ 00479c48     LIBCMTD:initnum.obj
 0003:00008c90       ??_C@_0DB@KKFMDHFI@f?3?2dd?2vctools?2crt_bld?2self_x86?2c@ 00479c90     LIBCMTD:initnum.obj
 0003:00008cd0       ??_C@_1GC@IKADOFBJ@?$AAf?$AA?3?$AA?2?$AAd?$AAd?$AA?2?$AAv?$AAc?$AAt?$AAo?$AAo?$AAl?$AAs?$AA?2?$AAc?$AAr?$AAt?$AA_?$AAb?$AAl?$AAd?$AA?2?$AAs?$AAe?$AAl?$AAf?$AA_?$AAx?$AA8?$AA6?$AA?2?$AAc@ 00479cd0     LIBCMTD:initmon.obj
 0003:00008d48       ??_C@_1DM@GKAPAMDO@?$AAp?$AAl?$AAo?$AAc?$AAi?$AA?9?$AA?$DO?$AAl?$AAc?$AAo?$AAn?$AAv?$AA_?$AAm?$AAo?$AAn?$AA_?$AAr?$AAe?$AAf?$AAc?$AAo?$AAu?$AAn?$AAt?$AA?5?$AA?$DO?$AA?5?$AA0?$AA?$AA@ 00479d48     LIBCMTD:initmon.obj
 0003:00008d90       ??_C@_0DB@BECNGFDL@f?3?2dd?2vctools?2crt_bld?2self_x86?2c@ 00479d90     LIBCMTD:initmon.obj
 0003:00008dcc       ??_C@_1DG@NMBGBDM@?$AAp?$AAl?$AAo?$AAc?$AAi?$AA?9?$AA?$DO?$AAc?$AAt?$AAy?$AAp?$AAe?$AA1?$AA_?$AAr?$AAe?$AAf?$AAc?$AAo?$AAu?$AAn?$AAt?$AA?5?$AA?$DO?$AA?5?$AA0?$AA?$AA@ 00479dcc     LIBCMTD:initctyp.obj
 0003:00008e10       ??_C@_1GE@OCPKBDKE@?$AAf?$AA?3?$AA?2?$AAd?$AAd?$AA?2?$AAv?$AAc?$AAt?$AAo?$AAo?$AAl?$AAs?$AA?2?$AAc?$AAr?$AAt?$AA_?$AAb?$AAl?$AAd?$AA?2?$AAs?$AAe?$AAl?$AAf?$AA_?$AAx?$AA8?$AA6?$AA?2?$AAc@ 00479e10     LIBCMTD:initctyp.obj
 0003:00008e88       ??_C@_0DC@EHLBFILA@f?3?2dd?2vctools?2crt_bld?2self_x86?2c@ 00479e88     LIBCMTD:initctyp.obj
 0003:00008ec4       ??_C@_1BE@NDMJHJJG@?$AAs?$AAt?$AAr?$AAn?$AAc?$AAp?$AAy?$AA_?$AAs?$AA?$AA@ 00479ec4     LIBCMTD:strncpy_s.obj
 0003:00008ee0       ??_C@_1GA@INJGGEBC@?$AAf?$AA?3?$AA?2?$AAd?$AAd?$AA?2?$AAv?$AAc?$AAt?$AAo?$AAo?$AAl?$AAs?$AA?2?$AAc?$AAr?$AAt?$AA_?$AAb?$AAl?$AAd?$AA?2?$AAs?$AAe?$AAl?$AAf?$AA_?$AAx?$AA8?$AA6?$AA?2?$AAc@ 00479ee0     LIBCMTD:a_str.obj
 0003:00008f58       ??_C@_1FE@KNPCCODH@?$AA?$CI?$AA?$CC?$AAC?$AAo?$AAr?$AAr?$AAu?$AAp?$AAt?$AAe?$AAd?$AA?5?$AAp?$AAo?$AAi?$AAn?$AAt?$AAe?$AAr?$AA?5?$AAp?$AAa?$AAs?$AAs?$AAe?$AAd?$AA?5?$AAt?$AAo?$AA?5?$AA_?$AAf@ 00479f58     LIBCMTD:a_str.obj
 0003:00008fbc       ??_C@_1BC@HGPNAKGC@?$AAs?$AAt?$AAr?$AAc?$AAa?$AAt?$AA_?$AAs?$AA?$AA@ 00479fbc     LIBCMTD:strcat_s.obj
 0003:00008fd4       ??_C@_0O@FMJNFNKE@united?9states?$AA@ 00479fd4     LIBCMTD:getqloc.obj
 0003:00008fe4       ??_C@_0P@NDHFFKCA@united?9kingdom?$AA@ 00479fe4     LIBCMTD:getqloc.obj
 0003:00008ff8       ??_C@_0BC@HHDADLGF@trinidad?5?$CG?5tobago?$AA@ 00479ff8     LIBCMTD:getqloc.obj
 0003:00009010       ??_C@_0M@IOAEBDAC@south?9korea?$AA@ 0047a010     LIBCMTD:getqloc.obj
 0003:00009020       ??_C@_0N@FIELFKIJ@south?9africa?$AA@ 0047a020     LIBCMTD:getqloc.obj
 0003:00009030       ??_C@_0M@OPNDHCMC@south?5korea?$AA@ 0047a030     LIBCMTD:getqloc.obj
 0003:00009040       ??_C@_0N@MDEOEPFI@south?5africa?$AA@ 0047a040     LIBCMTD:getqloc.obj
 0003:00009050       ??_C@_06FKAPCJLB@slovak?$AA@ 0047a050     LIBCMTD:getqloc.obj
 0003:00009058       ??_C@_0M@EFJANOAL@puerto?9rico?$AA@ 0047a058     LIBCMTD:getqloc.obj
 0003:00009068       ??_C@_08PGOJKDAI@pr?9china?$AA@ 0047a068     LIBCMTD:getqloc.obj
 0003:00009074       ??_C@_08JHDOMCMI@pr?5china?$AA@ 0047a074     LIBCMTD:getqloc.obj
 0003:00009080       ??_C@_02JHCHFBLL@nz?$AA@   0047a080     LIBCMTD:getqloc.obj
 0003:00009084       ??_C@_0M@LINHDHKP@new?9zealand?$AA@ 0047a084     LIBCMTD:getqloc.obj
 0003:00009094       ??_C@_09IIIPPBDB@hong?9kong?$AA@ 0047a094     LIBCMTD:getqloc.obj
 0003:000090a0       ??_C@_07HJLCKBG@holland?$AA@ 0047a0a0     LIBCMTD:getqloc.obj
 0003:000090ac       ??_C@_0O@LEHGMHAG@great?5britain?$AA@ 0047a0ac     LIBCMTD:getqloc.obj
 0003:000090bc       ??_C@_07FACOMELA@england?$AA@ 0047a0bc     LIBCMTD:getqloc.obj
 0003:000090c8       ??_C@_05JIHCEICB@czech?$AA@ 0047a0c8     LIBCMTD:getqloc.obj
 0003:000090d0       ??_C@_05BBJOBLGB@china?$AA@ 0047a0d0     LIBCMTD:getqloc.obj
 0003:000090d8       ??_C@_07GPKPHICP@britain?$AA@ 0047a0d8     LIBCMTD:getqloc.obj
 0003:000090e4       ??_C@_07MHIPBHMG@america?$AA@ 0047a0e4     LIBCMTD:getqloc.obj
 0003:000090f0       ??_C@_03KIALPMKC@usa?$AA@  0047a0f0     LIBCMTD:getqloc.obj
 0003:000090f4       ??_C@_02FGJGKGGD@us?$AA@   0047a0f4     LIBCMTD:getqloc.obj
 0003:000090f8       ??_C@_02NEINDODK@uk?$AA@   0047a0f8     LIBCMTD:getqloc.obj
 0003:000090fc       ??_C@_05JMPCFJFJ@swiss?$AA@ 0047a0fc     LIBCMTD:getqloc.obj
 0003:00009104       ??_C@_0BA@HLOCPIOD@swedish?9finland?$AA@ 0047a104     LIBCMTD:getqloc.obj
 0003:00009118       ??_C@_0BC@PKCNIABK@spanish?9venezuela?$AA@ 0047a118     LIBCMTD:getqloc.obj
 0003:00009130       ??_C@_0BA@GBHHMIJI@spanish?9uruguay?$AA@ 0047a130     LIBCMTD:getqloc.obj
 0003:00009144       ??_C@_0BE@BHDOHPMC@spanish?9puerto?5rico?$AA@ 0047a144     LIBCMTD:getqloc.obj
 0003:0000915c       ??_C@_0N@KMOIDGGN@spanish?9peru?$AA@ 0047a15c     LIBCMTD:getqloc.obj
 0003:0000916c       ??_C@_0BB@HMHLPGPH@spanish?9paraguay?$AA@ 0047a16c     LIBCMTD:getqloc.obj
 0003:00009180       ??_C@_0P@MCPKNGFD@spanish?9panama?$AA@ 0047a180     LIBCMTD:getqloc.obj
 0003:00009194       ??_C@_0BC@IHOHGAIL@spanish?9nicaragua?$AA@ 0047a194     LIBCMTD:getqloc.obj
 0003:000091ac       ??_C@_0P@KLMJDNFJ@spanish?9modern?$AA@ 0047a1ac     LIBCMTD:getqloc.obj
 0003:000091c0       ??_C@_0BA@BPAPGBCM@spanish?9mexican?$AA@ 0047a1c0     LIBCMTD:getqloc.obj
 0003:000091d4       ??_C@_0BB@PDECHHHE@spanish?9honduras?$AA@ 0047a1d4     LIBCMTD:getqloc.obj
 0003:000091e8       ??_C@_0BC@KLHKFGDB@spanish?9guatemala?$AA@ 0047a1e8     LIBCMTD:getqloc.obj
 0003:00009200       ??_C@_0BE@MFOOKJAI@spanish?9el?5salvador?$AA@ 0047a200     LIBCMTD:getqloc.obj
 0003:00009218       ??_C@_0BA@FCOKFPFC@spanish?9ecuador?$AA@ 0047a218     LIBCMTD:getqloc.obj
 0003:0000922c       ??_C@_0BL@PLMGIMOO@spanish?9dominican?5republic?$AA@ 0047a22c     LIBCMTD:getqloc.obj
 0003:0000924c       ??_C@_0BD@HLGDNMHB@spanish?9costa?5rica?$AA@ 0047a24c     LIBCMTD:getqloc.obj
 0003:00009264       ??_C@_0BB@PKCBKCPE@spanish?9colombia?$AA@ 0047a264     LIBCMTD:getqloc.obj
 0003:00009278       ??_C@_0O@MCBIJGNE@spanish?9chile?$AA@ 0047a278     LIBCMTD:getqloc.obj
 0003:00009288       ??_C@_0BA@BEFEIGJJ@spanish?9bolivia?$AA@ 0047a288     LIBCMTD:getqloc.obj
 0003:0000929c       ??_C@_0BC@EMECMPD@spanish?9argentina?$AA@ 0047a29c     LIBCMTD:getqloc.obj
 0003:000092b4       ??_C@_0BF@EALFLENP@portuguese?9brazilian?$AA@ 0047a2b4     LIBCMTD:getqloc.obj
 0003:000092d0       ??_C@_0BC@HBLEBLNN@norwegian?9nynorsk?$AA@ 0047a2d0     LIBCMTD:getqloc.obj
 0003:000092e8       ??_C@_0BB@HMACDDCK@norwegian?9bokmal?$AA@ 0047a2e8     LIBCMTD:getqloc.obj
 0003:000092fc       ??_C@_09BAFFPPHE@norwegian?$AA@ 0047a2fc     LIBCMTD:getqloc.obj
 0003:00009308       ??_C@_0O@EAJFJDFG@italian?9swiss?$AA@ 0047a308     LIBCMTD:getqloc.obj
 0003:00009318       ??_C@_0O@CNOMPGD@irish?9english?$AA@ 0047a318     LIBCMTD:getqloc.obj
 0003:00009328       ??_C@_0N@EDHBGCKG@german?9swiss?$AA@ 0047a328     LIBCMTD:getqloc.obj
 0003:00009338       ??_C@_0BC@JACMHNBP@german?9luxembourg?$AA@ 0047a338     LIBCMTD:getqloc.obj
 0003:00009350       ??_C@_0BE@HBGMGFEG@german?9lichtenstein?$AA@ 0047a350     LIBCMTD:getqloc.obj
 0003:00009368       ??_C@_0BA@HKKBIBKL@german?9austrian?$AA@ 0047a368     LIBCMTD:getqloc.obj
 0003:0000937c       ??_C@_0N@GCAEPEBK@french?9swiss?$AA@ 0047a37c     LIBCMTD:getqloc.obj
 0003:0000938c       ??_C@_0BC@DJFJJCK@french?9luxembourg?$AA@ 0047a38c     LIBCMTD:getqloc.obj
 0003:000093a4       ??_C@_0BA@NNCEDFIC@french?9canadian?$AA@ 0047a3a4     LIBCMTD:getqloc.obj
 0003:000093b8       ??_C@_0P@CMPOCLM@french?9belgian?$AA@ 0047a3b8     LIBCMTD:getqloc.obj
 0003:000093cc       ??_C@_0M@GHHDJOK@english?9usa?$AA@ 0047a3cc     LIBCMTD:getqloc.obj
 0003:000093dc       ??_C@_0L@PLDJKEIL@english?9us?$AA@ 0047a3dc     LIBCMTD:getqloc.obj
 0003:000093ec       ??_C@_0L@HJCCDMNC@english?9uk?$AA@ 0047a3ec     LIBCMTD:getqloc.obj
 0003:000093fc       ??_C@_0BK@CKLIAGJB@english?9trinidad?5y?5tobago?$AA@ 0047a3fc     LIBCMTD:getqloc.obj
 0003:0000941c       ??_C@_0BF@JMJMGNNF@english?9south?5africa?$AA@ 0047a41c     LIBCMTD:getqloc.obj
 0003:00009438       ??_C@_0L@DKIIFDFD@english?9nz?$AA@ 0047a438     LIBCMTD:getqloc.obj
 0003:00009448       ??_C@_0BA@ONHGJCLH@english?9jamaica?$AA@ 0047a448     LIBCMTD:getqloc.obj
 0003:0000945c       ??_C@_0M@HJBGHOPO@english?9ire?$AA@ 0047a45c     LIBCMTD:getqloc.obj
 0003:0000946c       ??_C@_0BC@LFEKMIFB@english?9caribbean?$AA@ 0047a46c     LIBCMTD:getqloc.obj
 0003:00009484       ??_C@_0M@OLDPFKHI@english?9can?$AA@ 0047a484     LIBCMTD:getqloc.obj
 0003:00009494       ??_C@_0P@OMDEHBMP@english?9belize?$AA@ 0047a494     LIBCMTD:getqloc.obj
 0003:000094a8       ??_C@_0M@KFHFPFED@english?9aus?$AA@ 0047a4a8     LIBCMTD:getqloc.obj
 0003:000094b8       ??_C@_0BB@MNMBKDFE@english?9american?$AA@ 0047a4b8     LIBCMTD:getqloc.obj
 0003:000094cc       ??_C@_0O@KIDLNNBA@dutch?9belgian?$AA@ 0047a4cc     LIBCMTD:getqloc.obj
 0003:000094dc       ??_C@_0BE@JBKABBMH@chinese?9traditional?$AA@ 0047a4dc     LIBCMTD:getqloc.obj
 0003:000094f4       ??_C@_0BC@MJJMPKCG@chinese?9singapore?$AA@ 0047a4f4     LIBCMTD:getqloc.obj
 0003:0000950c       ??_C@_0BD@FDKADDCP@chinese?9simplified?$AA@ 0047a50c     LIBCMTD:getqloc.obj
 0003:00009524       ??_C@_0BB@DBEFDDME@chinese?9hongkong?$AA@ 0047a524     LIBCMTD:getqloc.obj
 0003:00009538       ??_C@_07DHNMFMCI@chinese?$AA@ 0047a538     LIBCMTD:getqloc.obj
 0003:00009544       ??_C@_03FNDDCHI@chi?$AA@   0047a544     LIBCMTD:getqloc.obj
 0003:00009548       ??_C@_03BMMIADDJ@chh?$AA@  0047a548     LIBCMTD:getqloc.obj
 0003:0000954c       ??_C@_08OAIPJDGI@canadian?$AA@ 0047a54c     LIBCMTD:getqloc.obj
 0003:00009558       ??_C@_07HBPMNPNJ@belgian?$AA@ 0047a558     LIBCMTD:getqloc.obj
 0003:00009564       ??_C@_0L@OEKOPBEL@australian?$AA@ 0047a564     LIBCMTD:getqloc.obj
 0003:00009574       ??_C@_0BB@MEIMBEDG@american?9english?$AA@ 0047a574     LIBCMTD:getqloc.obj
 0003:00009588       ??_C@_0BB@DFMDPDGB@american?5english?$AA@ 0047a588     LIBCMTD:getqloc.obj
 0003:0000959c       ??_C@_08IJLOKOLL@american?$AA@ 0047a59c     LIBCMTD:getqloc.obj
 0003:000095a8       ___rg_language             0047a5a8     LIBCMTD:getqloc.obj
 0003:00009818       ___rg_country              0047a818     LIBCMTD:getqloc.obj
 0003:000098f4       ___rglangidNotDefault      0047a8f4     LIBCMTD:getqloc.obj
 0003:0000990c       ??_C@_0BC@NFIEMBLL@Norwegian?9Nynorsk?$AA@ 0047a90c     LIBCMTD:getqloc.obj
 0003:00009928       ??_C@_1OM@OECHDGCF@?$AAs?$AAt?$AAr?$AAc?$AAp?$AAy?$AA_?$AAs?$AA?$CI?$AAl?$AAp?$AAO?$AAu?$AAt?$AAS?$AAt?$AAr?$AA?9?$AA?$DO?$AAs?$AAz?$AAL?$AAa?$AAn?$AAg?$AAu?$AAa?$AAg?$AAe?$AA?0?$AA?5?$AA?$CI@ 0047a928     LIBCMTD:getqloc.obj
 0003:00009a44       ??_C@_1CO@NJACLALJ@?$AA_?$AA_?$AAg?$AAe?$AAt?$AA_?$AAq?$AAu?$AAa?$AAl?$AAi?$AAf?$AAi?$AAe?$AAd?$AA_?$AAl?$AAo?$AAc?$AAa?$AAl?$AAe?$AA?$AA@ 0047aa44     LIBCMTD:getqloc.obj
 0003:00009a80       ??_C@_1GC@FECJGAE@?$AAf?$AA?3?$AA?2?$AAd?$AAd?$AA?2?$AAv?$AAc?$AAt?$AAo?$AAo?$AAl?$AAs?$AA?2?$AAc?$AAr?$AAt?$AA_?$AAb?$AAl?$AAd?$AA?2?$AAs?$AAe?$AAl?$AAf?$AA_?$AAx?$AA8?$AA6?$AA?2?$AAc@ 0047aa80     LIBCMTD:getqloc.obj
 0003:00009af8       ??_C@_03NFKLAGEF@OCP?$AA@  0047aaf8     LIBCMTD:getqloc.obj
 0003:00009afc       ??_C@_03DFHEHBHG@ACP?$AA@  0047aafc     LIBCMTD:getqloc.obj
 0003:00009b00       __pDestructExceptionObject 0047ab00     LIBCMTD:frame.obj
 0003:00009b04       ??_C@_0O@DPKOEFFH@bad?5exception?$AA@ 0047ab04     LIBCMTD:frame.obj
 0003:00009b18       ??_7bad_exception@std@@6B@ 0047ab18     LIBCMTD:frame.obj
 0003:00009b28       ??_C@_1HO@MLMGPAFH@?$AA?$CI?$AA?$CC?$AAi?$AAn?$AAc?$AAo?$AAn?$AAs?$AAi?$AAs?$AAt?$AAe?$AAn?$AAt?$AA?5?$AAI?$AAO?$AAB?$AA?5?$AAf?$AAi?$AAe?$AAl?$AAd?$AAs?$AA?$CC?$AA?0?$AA?5?$AAs?$AAt?$AAr?$AAe@ 0047ab28     LIBCMTD:_flsbuf.obj
 0003:00009bc0       ??_C@_1GC@GNCCMPNN@?$AAf?$AA?3?$AA?2?$AAd?$AAd?$AA?2?$AAv?$AAc?$AAt?$AAo?$AAo?$AAl?$AAs?$AA?2?$AAc?$AAr?$AAt?$AA_?$AAb?$AAl?$AAd?$AA?2?$AAs?$AAe?$AAl?$AAf?$AA_?$AAx?$AA8?$AA6?$AA?2?$AAc@ 0047abc0     LIBCMTD:_flsbuf.obj
 0003:00009c38       ??_C@_1BI@MFCLPIBM@?$AAs?$AAt?$AAr?$AA?5?$AA?$CB?$AA?$DN?$AA?5?$AAN?$AAU?$AAL?$AAL?$AA?$AA@ 0047ac38     LIBCMTD:_flsbuf.obj
 0003:00009c54       ??_C@_1O@CEDCILHN@?$AA?$CI?$AAn?$AAu?$AAl?$AAl?$AA?$CJ?$AA?$AA@ 0047ac54     LIBCMTD:output.obj
 0003:00009c64       ??_C@_06OJHGLDPL@?$CInull?$CJ?$AA@ 0047ac64     LIBCMTD:output.obj
 0003:00009c70       ___lookuptable             0047ac70     LIBCMTD:output.obj
 0003:00009cdc       ??_C@_0DA@NFBEBPEE@f?3?2dd?2vctools?2crt_bld?2self_x86?2c@ 0047acdc     LIBCMTD:output.obj
 0003:00009d18       ??_C@_1EK@PNGFDECN@?$AA?$CI?$AA?$CC?$AA?8?$AAn?$AA?8?$AA?5?$AAf?$AAo?$AAr?$AAm?$AAa?$AAt?$AA?5?$AAs?$AAp?$AAe?$AAc?$AAi?$AAf?$AAi?$AAe?$AAr?$AA?5?$AAd?$AAi?$AAs?$AAa?$AAb?$AAl?$AAe?$AAd?$AA?$CC@ 0047ad18     LIBCMTD:output.obj
 0003:00009d70       ??_C@_1CC@IFFHEMNF@?$AA?$CI?$AAc?$AAh?$AA?5?$AA?$CB?$AA?$DN?$AA?5?$AA_?$AAT?$AA?$CI?$AA?8?$AA?2?$AA0?$AA?8?$AA?$CJ?$AA?$CJ?$AA?$AA@ 0047ad70     LIBCMTD:output.obj
 0003:00009d98       ??_C@_1BAA@ODEGEDCK@?$AA?$CI?$AA?5?$AA?$CI?$AA_?$AAS?$AAt?$AAr?$AAe?$AAa?$AAm?$AA?9?$AA?$DO?$AA_?$AAf?$AAl?$AAa?$AAg?$AA?5?$AA?$CG?$AA?5?$AA_?$AAI?$AAO?$AAS?$AAT?$AAR?$AAG?$AA?$CJ?$AA?5?$AA?$HM?$AA?$HM?$AA?5@ 0047ad98     LIBCMTD:output.obj
 0003:00009ecc       ??_C@_1BE@IONLIDNC@?$AA_?$AAo?$AAu?$AAt?$AAp?$AAu?$AAt?$AA_?$AAl?$AA?$AA@ 0047aecc     LIBCMTD:output.obj
 0003:00009ee8       ??_C@_1GA@HHFOFBLN@?$AAf?$AA?3?$AA?2?$AAd?$AAd?$AA?2?$AAv?$AAc?$AAt?$AAo?$AAo?$AAl?$AAs?$AA?2?$AAc?$AAr?$AAt?$AA_?$AAb?$AAl?$AAd?$AA?2?$AAs?$AAe?$AAl?$AAf?$AA_?$AAx?$AA8?$AA6?$AA?2?$AAc@ 0047aee8     LIBCMTD:output.obj
 0003:00009f5c       ??_C@_1CC@FADMNIL@?$AA?$CI?$AAs?$AAt?$AAr?$AAe?$AAa?$AAm?$AA?5?$AA?$CB?$AA?$DN?$AA?5?$AAN?$AAU?$AAL?$AAL?$AA?$CJ?$AA?$AA@ 0047af5c     LIBCMTD:output.obj
 0003:00009f84       ??_C@_1BI@IGILPKD@?$AA_?$AAv?$AAs?$AAp?$AAr?$AAi?$AAn?$AAt?$AAf?$AA_?$AAl?$AA?$AA@ 0047af84     LIBCMTD:vsprintf.obj
 0003:00009fa0       ??_C@_1GE@DPADKNCG@?$AAf?$AA?3?$AA?2?$AAd?$AAd?$AA?2?$AAv?$AAc?$AAt?$AAo?$AAo?$AAl?$AAs?$AA?2?$AAc?$AAr?$AAt?$AA_?$AAb?$AAl?$AAd?$AA?2?$AAs?$AAe?$AAl?$AAf?$AA_?$AAx?$AA8?$AA6?$AA?2?$AAc@ 0047afa0     LIBCMTD:vsprintf.obj
 0003:0000a018       ??_C@_1CE@HMKDJHB@?$AA_?$AAv?$AAs?$AAc?$AAp?$AAr?$AAi?$AAn?$AAt?$AAf?$AA_?$AAh?$AAe?$AAl?$AAp?$AAe?$AAr?$AA?$AA@ 0047b018     LIBCMTD:vsprintf.obj
 0003:0000a048       ??_C@_1EC@FABAOFFO@?$AA?$CI?$AAc?$AAo?$AAu?$AAn?$AAt?$AA?5?$AA?$DN?$AA?$DN?$AA?5?$AA0?$AA?$CJ?$AA?5?$AA?$HM?$AA?$HM?$AA?5?$AA?$CI?$AAs?$AAt?$AAr?$AAi?$AAn?$AAg?$AA?5?$AA?$CB?$AA?$DN?$AA?5?$AAN?$AAU?$AAL?$AAL?$AA?$CJ@ 0047b048     LIBCMTD:vsnprnc.obj
 0003:0000a098       ??_C@_1CE@PCFPEIFI@?$AA_?$AAv?$AAs?$AAn?$AAp?$AAr?$AAi?$AAn?$AAt?$AAf?$AA_?$AAh?$AAe?$AAl?$AAp?$AAe?$AAr?$AA?$AA@ 0047b098     LIBCMTD:vsnprnc.obj
 0003:0000a0c4       ??_C@_1DA@HPBFKMEB@?$AA?$CI?$AA?$CC?$AAB?$AAu?$AAf?$AAf?$AAe?$AAr?$AA?5?$AAt?$AAo?$AAo?$AA?5?$AAs?$AAm?$AAa?$AAl?$AAl?$AA?$CC?$AA?0?$AA?5?$AA0?$AA?$CJ?$AA?$AA@ 0047b0c4     LIBCMTD:vsnprnc.obj
 0003:0000a100       ??_C@_1EE@OKCKIGFK@?$AAs?$AAt?$AAr?$AAi?$AAn?$AAg?$AA?5?$AA?$CB?$AA?$DN?$AA?5?$AAN?$AAU?$AAL?$AAL?$AA?5?$AA?$CG?$AA?$CG?$AA?5?$AAs?$AAi?$AAz?$AAe?$AAI?$AAn?$AAB?$AAy?$AAt?$AAe?$AAs?$AA?5?$AA?$DO?$AA?5@ 0047b100     LIBCMTD:vsnprnc.obj
 0003:0000a154       ??_C@_1BM@BLJALHEF@?$AA_?$AAv?$AAs?$AAp?$AAr?$AAi?$AAn?$AAt?$AAf?$AA_?$AAs?$AA_?$AAl?$AA?$AA@ 0047b154     LIBCMTD:vsnprnc.obj
 0003:0000a178       ??_C@_1BO@MLMCMBKN@?$AAf?$AAo?$AAr?$AAm?$AAa?$AAt?$AA?5?$AA?$CB?$AA?$DN?$AA?5?$AAN?$AAU?$AAL?$AAL?$AA?$AA@ 0047b178     LIBCMTD:vsnprnc.obj
 0003:0000a19c       ??_C@_1BO@MMPELNIM@?$AA_?$AAv?$AAs?$AAn?$AAp?$AAr?$AAi?$AAn?$AAt?$AAf?$AA_?$AAs?$AA_?$AAl?$AA?$AA@ 0047b19c     LIBCMTD:vsnprnc.obj
 0003:0000a1c0       ??_C@_1CG@JEHFHLNG@?$AA_?$AAm?$AAb?$AAs?$AAt?$AAo?$AAw?$AAc?$AAs?$AA_?$AAl?$AA_?$AAh?$AAe?$AAl?$AAp?$AAe?$AAr?$AA?$AA@ 0047b1c0     LIBCMTD:mbstowcs.obj
 0003:0000a1f0       ??_C@_1GE@LCCDHBMH@?$AAf?$AA?3?$AA?2?$AAd?$AAd?$AA?2?$AAv?$AAc?$AAt?$AAo?$AAo?$AAl?$AAs?$AA?2?$AAc?$AAr?$AAt?$AA_?$AAb?$AAl?$AAd?$AA?2?$AAs?$AAe?$AAl?$AAf?$AA_?$AAx?$AA8?$AA6?$AA?2?$AAc@ 0047b1f0     LIBCMTD:mbstowcs.obj
 0003:0000a268       ??_C@_1BE@EEKACIGI@?$AAs?$AA?5?$AA?$CB?$AA?$DN?$AA?5?$AAN?$AAU?$AAL?$AAL?$AA?$AA@ 0047b268     LIBCMTD:mbstowcs.obj
 0003:0000a280       ??_C@_1CO@JNPEPJAL@?$AAr?$AAe?$AAt?$AAs?$AAi?$AAz?$AAe?$AA?5?$AA?$DM?$AA?$DN?$AA?5?$AAs?$AAi?$AAz?$AAe?$AAI?$AAn?$AAW?$AAo?$AAr?$AAd?$AAs?$AA?$AA@ 0047b280     LIBCMTD:mbstowcs.obj
 0003:0000a2b8       ??_C@_1CM@LLECFMFH@?$AAb?$AAu?$AAf?$AAf?$AAe?$AAr?$AAS?$AAi?$AAz?$AAe?$AA?5?$AA?$DM?$AA?$DN?$AA?5?$AAI?$AAN?$AAT?$AA_?$AAM?$AAA?$AAX?$AA?$AA@ 0047b2b8     LIBCMTD:mbstowcs.obj
 0003:0000a2ec       ??_C@_1BM@PHENIGHD@?$AA_?$AAm?$AAb?$AAs?$AAt?$AAo?$AAw?$AAc?$AAs?$AA_?$AAs?$AA_?$AAl?$AA?$AA@ 0047b2ec     LIBCMTD:mbstowcs.obj
 0003:0000a310       ??_C@_1JA@JKDFMOPO@?$AA?$CI?$AAp?$AAw?$AAc?$AAs?$AA?5?$AA?$DN?$AA?$DN?$AA?5?$AAN?$AAU?$AAL?$AAL?$AA?5?$AA?$CG?$AA?$CG?$AA?5?$AAs?$AAi?$AAz?$AAe?$AAI?$AAn?$AAW?$AAo?$AAr?$AAd?$AAs?$AA?5?$AA?$DN?$AA?$DN?$AA?5@ 0047b310     LIBCMTD:mbstowcs.obj
 0003:0000a3bc       ??_C@_1CM@HABGDNLJ@?$AAl?$AAe?$AAn?$AAg?$AAt?$AAh?$AA?5?$AA?$DM?$AA?5?$AAs?$AAi?$AAz?$AAe?$AAI?$AAn?$AAT?$AAC?$AAh?$AAa?$AAr?$AAs?$AA?$AA@ 0047b3bc     LIBCMTD:xtoas.obj
 0003:0000a3f0       ??_C@_1DE@PCJGDBBD@?$AA2?$AA?5?$AA?$DM?$AA?$DN?$AA?5?$AAr?$AAa?$AAd?$AAi?$AAx?$AA?5?$AA?$CG?$AA?$CG?$AA?5?$AAr?$AAa?$AAd?$AAi?$AAx?$AA?5?$AA?$DM?$AA?$DN?$AA?5?$AA3?$AA6?$AA?$AA@ 0047b3f0     LIBCMTD:xtoas.obj
 0003:0000a430       ??_C@_1FA@MKGGAGEI@?$AAs?$AAi?$AAz?$AAe?$AAI?$AAn?$AAT?$AAC?$AAh?$AAa?$AAr?$AAs?$AA?5?$AA?$DO?$AA?5?$AA?$CI?$AAs?$AAi?$AAz?$AAe?$AA_?$AAt?$AA?$CJ?$AA?$CI?$AAi?$AAs?$AA_?$AAn?$AAe?$AAg?$AA?5?$AA?$DP@ 0047b430     LIBCMTD:xtoas.obj
 0003:0000a490       ??_C@_1CC@JNJFIMGE@?$AAs?$AAi?$AAz?$AAe?$AAI?$AAn?$AAT?$AAC?$AAh?$AAa?$AAr?$AAs?$AA?5?$AA?$DO?$AA?5?$AA0?$AA?$AA@ 0047b490     LIBCMTD:xtoas.obj
 0003:0000a4b8       ??_C@_1O@GIMBNLEI@?$AAx?$AAt?$AAo?$AAa?$AA_?$AAs?$AA?$AA@ 0047b4b8     LIBCMTD:xtoas.obj
 0003:0000a4c8       ??_C@_1FM@MFCBFCGB@?$AAf?$AA?3?$AA?2?$AAd?$AAd?$AA?2?$AAv?$AAc?$AAt?$AAo?$AAo?$AAl?$AAs?$AA?2?$AAc?$AAr?$AAt?$AA_?$AAb?$AAl?$AAd?$AA?2?$AAs?$AAe?$AAl?$AAf?$AA_?$AAx?$AA8?$AA6?$AA?2?$AAc@ 0047b4c8     LIBCMTD:xtoas.obj
 0003:0000a538       ??_C@_1BI@ICGGMGLK@?$AAb?$AAu?$AAf?$AA?5?$AA?$CB?$AA?$DN?$AA?5?$AAN?$AAU?$AAL?$AAL?$AA?$AA@ 0047b538     LIBCMTD:xtoas.obj
 0003:0000a554       ??_C@_1BC@MJJNBNFN@?$AAx?$AA6?$AA4?$AAt?$AAo?$AAa?$AA_?$AAs?$AA?$AA@ 0047b554     LIBCMTD:xtoas.obj
 0003:0000a56c       ??_C@_1CG@LLJCAOHF@?$AA_?$AAw?$AAc?$AAs?$AAt?$AAo?$AAm?$AAb?$AAs?$AA_?$AAl?$AA_?$AAh?$AAe?$AAl?$AAp?$AAe?$AAr?$AA?$AA@ 0047b56c     LIBCMTD:wcstombs.obj
 0003:0000a5a0       ??_C@_1GE@OAENIBOD@?$AAf?$AA?3?$AA?2?$AAd?$AAd?$AA?2?$AAv?$AAc?$AAt?$AAo?$AAo?$AAl?$AAs?$AA?2?$AAc?$AAr?$AAt?$AA_?$AAb?$AAl?$AAd?$AA?2?$AAs?$AAe?$AAl?$AAf?$AA_?$AAx?$AA8?$AA6?$AA?2?$AAc@ 0047b5a0     LIBCMTD:wcstombs.obj
 0003:0000a618       ??_C@_1BK@OIBENBPM@?$AAp?$AAw?$AAc?$AAs?$AA?5?$AA?$CB?$AA?$DN?$AA?5?$AAN?$AAU?$AAL?$AAL?$AA?$AA@ 0047b618     LIBCMTD:wcstombs.obj
 0003:0000a638       ??_C@_1CM@KEOGBFLI@?$AAs?$AAi?$AAz?$AAe?$AAI?$AAn?$AAB?$AAy?$AAt?$AAe?$AAs?$AA?5?$AA?$DO?$AA?5?$AAr?$AAe?$AAt?$AAs?$AAi?$AAz?$AAe?$AA?$AA@ 0047b638     LIBCMTD:wcstombs.obj
 0003:0000a66c       ??_C@_1BM@BDMCLLDL@?$AA_?$AAw?$AAc?$AAs?$AAt?$AAo?$AAm?$AAb?$AAs?$AA_?$AAs?$AA_?$AAl?$AA?$AA@ 0047b66c     LIBCMTD:wcstombs.obj
 0003:0000a690       ??_C@_1IM@MFGKHGBP@?$AA?$CI?$AAd?$AAs?$AAt?$AA?5?$AA?$CB?$AA?$DN?$AA?5?$AAN?$AAU?$AAL?$AAL?$AA?5?$AA?$CG?$AA?$CG?$AA?5?$AAs?$AAi?$AAz?$AAe?$AAI?$AAn?$AAB?$AAy?$AAt?$AAe?$AAs?$AA?5?$AA?$DO?$AA?5?$AA0?$AA?$CJ@ 0047b690     LIBCMTD:wcstombs.obj
 0003:0000a738       ??_C@_1CE@IGKFIJFD@?$AA_?$AAv?$AAs?$AAw?$AAp?$AAr?$AAi?$AAn?$AAt?$AAf?$AA_?$AAh?$AAe?$AAl?$AAp?$AAe?$AAr?$AA?$AA@ 0047b738     LIBCMTD:vswprnc.obj
 0003:0000a768       ??_C@_1GE@KINELFI@?$AAf?$AA?3?$AA?2?$AAd?$AAd?$AA?2?$AAv?$AAc?$AAt?$AAo?$AAo?$AAl?$AAs?$AA?2?$AAc?$AAr?$AAt?$AA_?$AAb?$AAl?$AAd?$AA?2?$AAs?$AAe?$AAl?$AAf?$AA_?$AAx?$AA8?$AA6?$AA?2?$AAc@ 0047b768     LIBCMTD:vswprnc.obj
 0003:0000a7e0       ??_C@_1EE@MPCHJFGP@?$AAs?$AAt?$AAr?$AAi?$AAn?$AAg?$AA?5?$AA?$CB?$AA?$DN?$AA?5?$AAN?$AAU?$AAL?$AAL?$AA?5?$AA?$CG?$AA?$CG?$AA?5?$AAs?$AAi?$AAz?$AAe?$AAI?$AAn?$AAW?$AAo?$AAr?$AAd?$AAs?$AA?5?$AA?$DO?$AA?5@ 0047b7e0     LIBCMTD:vswprnc.obj
 0003:0000a834       ??_C@_1BO@OALHJLCI@?$AA_?$AAv?$AAs?$AAw?$AAp?$AAr?$AAi?$AAn?$AAt?$AAf?$AA_?$AAs?$AA_?$AAl?$AA?$AA@ 0047b834     LIBCMTD:vswprnc.obj
 0003:0000a858       ??_C@_1CA@BKFKMJFF@?$AA_?$AAv?$AAs?$AAn?$AAw?$AAp?$AAr?$AAi?$AAn?$AAt?$AAf?$AA_?$AAs?$AA_?$AAl?$AA?$AA@ 0047b858     LIBCMTD:vswprnc.obj
 0003:0000a880       ??_C@_1O@NCBFODOE@?$AAx?$AAt?$AAo?$AAw?$AA_?$AAs?$AA?$AA@ 0047b880     LIBCMTD:xtows.obj
 0003:0000a890       ??_C@_1BC@HDEJCFPB@?$AAx?$AA6?$AA4?$AAt?$AAo?$AAw?$AA_?$AAs?$AA?$AA@ 0047b890     LIBCMTD:xtows.obj
 0003:0000a8a8       ??_C@_1BG@BBCDFOMA@?$AA_?$AAw?$AAo?$AAu?$AAt?$AAp?$AAu?$AAt?$AA_?$AAl?$AA?$AA@ 0047b8a8     LIBCMTD:woutput.obj
 0003:0000a8c4       ??_C@_1BK@EPLNBKAK@?$AA_?$AAv?$AAs?$AAw?$AAp?$AAr?$AAi?$AAn?$AAt?$AAf?$AA_?$AAl?$AA?$AA@ 0047b8c4     LIBCMTD:vswprint.obj
 0003:0000a8e4       ??_C@_1CG@IMMIEPNA@?$AA_?$AAv?$AAs?$AAc?$AAw?$AAp?$AAr?$AAi?$AAn?$AAt?$AAf?$AA_?$AAh?$AAe?$AAl?$AAp?$AAe?$AAr?$AA?$AA@ 0047b8e4     LIBCMTD:vswprint.obj
 0003:0000a914       ??_C@_1BG@GLLONOEH@?$AA_?$AAs?$AAt?$AAr?$AAi?$AAc?$AAm?$AAp?$AA_?$AAl?$AA?$AA@ 0047b914     LIBCMTD:stricmp.obj
 0003:0000a930       ??_C@_1GC@OILHAOLL@?$AAf?$AA?3?$AA?2?$AAd?$AAd?$AA?2?$AAv?$AAc?$AAt?$AAo?$AAo?$AAl?$AAs?$AA?2?$AAc?$AAr?$AAt?$AA_?$AAb?$AAl?$AAd?$AA?2?$AAs?$AAe?$AAl?$AAf?$AA_?$AAx?$AA8?$AA6?$AA?2?$AAc@ 0047b930     LIBCMTD:stricmp.obj
 0003:0000a9a8       ??_C@_1BC@JLGKKIIG@?$AA_?$AAs?$AAt?$AAr?$AAi?$AAc?$AAm?$AAp?$AA?$AA@ 0047b9a8     LIBCMTD:stricmp.obj
 0003:0000a9c0       ??_C@_1CC@JLPHKJPH@?$AAc?$AAo?$AAu?$AAn?$AAt?$AA?5?$AA?$DM?$AA?$DN?$AA?5?$AAI?$AAN?$AAT?$AA_?$AAM?$AAA?$AAX?$AA?$AA@ 0047b9c0     LIBCMTD:strnicmp.obj
 0003:0000a9e8       ??_C@_1BI@BJLEPLEF@?$AA_?$AAs?$AAt?$AAr?$AAn?$AAi?$AAc?$AAm?$AAp?$AA_?$AAl?$AA?$AA@ 0047b9e8     LIBCMTD:strnicmp.obj
 0003:0000aa08       ??_C@_1GE@CONPOJMA@?$AAf?$AA?3?$AA?2?$AAd?$AAd?$AA?2?$AAv?$AAc?$AAt?$AAo?$AAo?$AAl?$AAs?$AA?2?$AAc?$AAr?$AAt?$AA_?$AAb?$AAl?$AAd?$AA?2?$AAs?$AAe?$AAl?$AAf?$AA_?$AAx?$AA8?$AA6?$AA?2?$AAc@ 0047ba08     LIBCMTD:strnicmp.obj
 0003:0000aa80       ??_C@_1BE@BHJDFFNA@?$AA_?$AAs?$AAt?$AAr?$AAn?$AAi?$AAc?$AAm?$AAp?$AA?$AA@ 0047ba80     LIBCMTD:strnicmp.obj
 0003:0000aac4       ??_7type_info@@6B@         0047bac4     LIBCMTD:typinfo.obj
 0003:0000aad0       ??_7exception@std@@6B@     0047bad0     LIBCMTD:stdexcpt.obj
 0003:0000aadc       ??_C@_0BC@EOODALEL@Unknown?5exception?$AA@ 0047badc     LIBCMTD:stdexcpt.obj
 0003:0000aaf8       ??_7bad_cast@std@@6B@      0047baf8     LIBCMTD:stdexcpt.obj
 0003:0000ab08       ??_7bad_typeid@std@@6B@    0047bb08     LIBCMTD:stdexcpt.obj
 0003:0000ab18       ??_7__non_rtti_object@std@@6B@ 0047bb18     LIBCMTD:stdexcpt.obj
 0003:0000ab28       ??_C@_1GE@BDAODJCD@?$AAf?$AA?3?$AA?2?$AAd?$AAd?$AA?2?$AAv?$AAc?$AAt?$AAo?$AAo?$AAl?$AAs?$AA?2?$AAc?$AAr?$AAt?$AA_?$AAb?$AAl?$AAd?$AA?2?$AAs?$AAe?$AAl?$AAf?$AA_?$AAx?$AA8?$AA6?$AA?2?$AAc@ 0047bb28     LIBCMTD:dbgdel.obj
 0003:0000aba0       ??_C@_1JE@ECKHFIFP@?$AA?$CI?$AA?$CC?$AAI?$AAn?$AAv?$AAa?$AAl?$AAi?$AAd?$AA?5?$AAf?$AAi?$AAl?$AAe?$AA?5?$AAd?$AAe?$AAs?$AAc?$AAr?$AAi?$AAp?$AAt?$AAo?$AAr?$AA?4?$AA?5?$AAF?$AAi?$AAl?$AAe?$AA?5@ 0047bba0     LIBCMTD:lseeki64.obj
 0003:0000ac54       ??_C@_1CM@OKGMMMDH@?$AA?$CI?$AA_?$AAo?$AAs?$AAf?$AAi?$AAl?$AAe?$AA?$CI?$AAf?$AAh?$AA?$CJ?$AA?5?$AA?$CG?$AA?5?$AAF?$AAO?$AAP?$AAE?$AAN?$AA?$CJ?$AA?$AA@ 0047bc54     LIBCMTD:lseeki64.obj
 0003:0000ac88       ??_C@_1BE@KHFBJMNM@?$AA_?$AAl?$AAs?$AAe?$AAe?$AAk?$AAi?$AA6?$AA4?$AA?$AA@ 0047bc88     LIBCMTD:lseeki64.obj
 0003:0000aca0       ??_C@_1GE@MINKPNPH@?$AAf?$AA?3?$AA?2?$AAd?$AAd?$AA?2?$AAv?$AAc?$AAt?$AAo?$AAo?$AAl?$AAs?$AA?2?$AAc?$AAr?$AAt?$AA_?$AAb?$AAl?$AAd?$AA?2?$AAs?$AAe?$AAl?$AAf?$AA_?$AAx?$AA8?$AA6?$AA?2?$AAc@ 0047bca0     LIBCMTD:lseeki64.obj
 0003:0000ad18       ??_C@_1FO@LPCLHKGE@?$AA?$CI?$AAf?$AAh?$AA?5?$AA?$DO?$AA?$DN?$AA?5?$AA0?$AA?5?$AA?$CG?$AA?$CG?$AA?5?$AA?$CI?$AAu?$AAn?$AAs?$AAi?$AAg?$AAn?$AAe?$AAd?$AA?$CJ?$AAf?$AAh?$AA?5?$AA?$DM?$AA?5?$AA?$CI?$AAu?$AAn?$AAs?$AAi@ 0047bd18     LIBCMTD:lseeki64.obj
 0003:0000ad88       ??_C@_1O@KOFKDHPL@?$AA_?$AAw?$AAr?$AAi?$AAt?$AAe?$AA?$AA@ 0047bd88     LIBCMTD:write.obj
 0003:0000ad98       ??_C@_1FO@EPLDPDDL@?$AAf?$AA?3?$AA?2?$AAd?$AAd?$AA?2?$AAv?$AAc?$AAt?$AAo?$AAo?$AAl?$AAs?$AA?2?$AAc?$AAr?$AAt?$AA_?$AAb?$AAl?$AAd?$AA?2?$AAs?$AAe?$AAl?$AAf?$AA_?$AAx?$AA8?$AA6?$AA?2?$AAc@ 0047bd98     LIBCMTD:write.obj
 0003:0000ae08       ??_C@_1DI@CNMHHHLG@?$AAi?$AAs?$AAl?$AAe?$AAa?$AAd?$AAb?$AAy?$AAt?$AAe?$AA?$CI?$AA_?$AAd?$AAb?$AAc?$AAs?$AAB?$AAu?$AAf?$AAf?$AAe?$AAr?$AA?$CI?$AAf?$AAh?$AA?$CJ?$AA?$CJ?$AA?$AA@ 0047be08     LIBCMTD:write.obj
 0003:0000ae4c       ??_C@_1CC@EEOLPHGO@?$AA?$CI?$AA?$CI?$AAc?$AAn?$AAt?$AA?5?$AA?$CG?$AA?5?$AA1?$AA?$CJ?$AA?5?$AA?$DN?$AA?$DN?$AA?5?$AA0?$AA?$CJ?$AA?$AA@ 0047be4c     LIBCMTD:write.obj
 0003:0000ae74       ??_C@_1BM@NCANHCIP@?$AA_?$AAw?$AAr?$AAi?$AAt?$AAe?$AA_?$AAn?$AAo?$AAl?$AAo?$AAc?$AAk?$AA?$AA@ 0047be74     LIBCMTD:write.obj
 0003:0000ae98       ??_C@_1BM@KFJLMBPG@?$AA?$CI?$AAb?$AAu?$AAf?$AA?5?$AA?$CB?$AA?$DN?$AA?5?$AAN?$AAU?$AAL?$AAL?$AA?$CJ?$AA?$AA@ 0047be98     LIBCMTD:write.obj
 0003:0000aebc       ??_C@_0DB@JEHOCBEJ@f?3?2dd?2vctools?2crt_bld?2self_x86?2c@ 0047bebc     LIBCMTD:_getbuf.obj
 0003:0000aef8       ??_C@_1GC@DKMGNNCC@?$AAf?$AA?3?$AA?2?$AAd?$AAd?$AA?2?$AAv?$AAc?$AAt?$AAo?$AAo?$AAl?$AAs?$AA?2?$AAc?$AAr?$AAt?$AA_?$AAb?$AAl?$AAd?$AA?2?$AAs?$AAe?$AAl?$AAf?$AA_?$AAx?$AA8?$AA6?$AA?2?$AAc@ 0047bef8     LIBCMTD:_getbuf.obj
 0003:0000af70       ??_C@_1BA@LEBDGIHM@?$AA_?$AAi?$AAs?$AAa?$AAt?$AAt?$AAy?$AA?$AA@ 0047bf70     LIBCMTD:isatty.obj
 0003:0000af88       ??_C@_1GA@LPGDJDEN@?$AAf?$AA?3?$AA?2?$AAd?$AAd?$AA?2?$AAv?$AAc?$AAt?$AAo?$AAo?$AAl?$AAs?$AA?2?$AAc?$AAr?$AAt?$AA_?$AAb?$AAl?$AAd?$AA?2?$AAs?$AAe?$AAl?$AAf?$AA_?$AAx?$AA8?$AA6?$AA?2?$AAc@ 0047bf88     LIBCMTD:isatty.obj
 0003:0000affc       ??_C@_0CP@BNKDODJJ@f?3?2dd?2vctools?2crt_bld?2self_x86?2c@ 0047bffc     LIBCMTD:_file.obj
 0003:0000b034       ??_C@_1BA@JGHIEKKM@?$AA_?$AAf?$AAi?$AAl?$AAe?$AAn?$AAo?$AA?$AA@ 0047c034     LIBCMTD:fileno.obj
 0003:0000b048       ??_C@_1GA@PBJHELNC@?$AAf?$AA?3?$AA?2?$AAd?$AAd?$AA?2?$AAv?$AAc?$AAt?$AAo?$AAo?$AAl?$AAs?$AA?2?$AAc?$AAr?$AAt?$AA_?$AAb?$AAl?$AAd?$AA?2?$AAs?$AAe?$AAl?$AAf?$AA_?$AAx?$AA8?$AA6?$AA?2?$AAc@ 0047c048     LIBCMTD:fileno.obj
 0003:0000b0bc       ??_C@_1O@GKDHFACN@?$AAp?$AAr?$AAi?$AAn?$AAt?$AAf?$AA?$AA@ 0047c0bc     LIBCMTD:printf.obj
 0003:0000b0d0       ??_C@_1GA@LHEGHOAF@?$AAf?$AA?3?$AA?2?$AAd?$AAd?$AA?2?$AAv?$AAc?$AAt?$AAo?$AAo?$AAl?$AAs?$AA?2?$AAc?$AAr?$AAt?$AA_?$AAb?$AAl?$AAd?$AA?2?$AAs?$AAe?$AAl?$AAf?$AA_?$AAx?$AA8?$AA6?$AA?2?$AAc@ 0047c0d0     LIBCMTD:printf.obj
 0003:0000b144       ??_C@_1CA@CBMNPEO@?$AAs?$AAi?$AAz?$AAe?$AAI?$AAn?$AAB?$AAy?$AAt?$AAe?$AAs?$AA?5?$AA?$DO?$AA?5?$AA0?$AA?$AA@ 0047c144     LIBCMTD:wctomb.obj
 0003:0000b16c       ??_C@_1BI@IEADNOHF@?$AA_?$AAw?$AAc?$AAt?$AAo?$AAm?$AAb?$AA_?$AAs?$AA_?$AAl?$AA?$AA@ 0047c16c     LIBCMTD:wctomb.obj
 0003:0000b188       ??_C@_1GA@LDLHPOO@?$AAf?$AA?3?$AA?2?$AAd?$AAd?$AA?2?$AAv?$AAc?$AAt?$AAo?$AAo?$AAl?$AAs?$AA?2?$AAc?$AAr?$AAt?$AA_?$AAb?$AAl?$AAd?$AA?2?$AAs?$AAe?$AAl?$AAf?$AA_?$AAx?$AA8?$AA6?$AA?2?$AAc@ 0047c188     LIBCMTD:wctomb.obj
 0003:0000b1fc       ??_C@_1CO@HFMIILNF@?$AAs?$AAi?$AAz?$AAe?$AAI?$AAn?$AAB?$AAy?$AAt?$AAe?$AAs?$AA?5?$AA?$DM?$AA?$DN?$AA?5?$AAI?$AAN?$AAT?$AA_?$AAM?$AAA?$AAX?$AA?$AA@ 0047c1fc     LIBCMTD:wctomb.obj
 0003:0000b238       ??_C@_1FK@BCPANIEK@?$AA?$CI?$AA?$CC?$AAM?$AAi?$AAs?$AAs?$AAi?$AAn?$AAg?$AA?5?$AAp?$AAo?$AAs?$AAi?$AAt?$AAi?$AAo?$AAn?$AA?5?$AAi?$AAn?$AA?5?$AAt?$AAh?$AAe?$AA?5?$AAf?$AAo?$AAr?$AAm?$AAa?$AAt@ 0047c238     LIBCMTD:outputp.obj
 0003:0000b2a8       ??_C@_1FK@LNCFKALM@?$AA?$CI?$AA?$CI?$AAs?$AAt?$AAa?$AAt?$AAe?$AA?5?$AA?$DN?$AA?$DN?$AA?5?$AAS?$AAT?$AA_?$AAN?$AAO?$AAR?$AAM?$AAA?$AAL?$AA?$CJ?$AA?5?$AA?$HM?$AA?$HM?$AA?5?$AA?$CI?$AAs?$AAt?$AAa?$AAt?$AAe?$AA?5@ 0047c2a8     LIBCMTD:outputp.obj
 0003:0000b318       ??_C@_1JC@OACKELNN@?$AA_?$AAt?$AAv?$AAa?$AAl?$AAi?$AAd?$AAa?$AAt?$AAe?$AA_?$AAp?$AAa?$AAr?$AAa?$AAm?$AA_?$AAr?$AAe?$AAu?$AAs?$AAe?$AA?$CI?$AA?$CG?$AAp?$AAo?$AAs?$AA_?$AAv?$AAa?$AAl?$AAu@ 0047c318     LIBCMTD:outputp.obj
 0003:0000b3c8       ??_C@_1IK@NBGDDCBN@?$AA_?$AAt?$AAv?$AAa?$AAl?$AAi?$AAd?$AAa?$AAt?$AAe?$AA_?$AAp?$AAa?$AAr?$AAa?$AAm?$AA_?$AAr?$AAe?$AAu?$AAs?$AAe?$AA?$CI?$AA?$CG?$AAp?$AAo?$AAs?$AA_?$AAv?$AAa?$AAl?$AAu@ 0047c3c8     LIBCMTD:outputp.obj
 0003:0000b470       ??_C@_1DG@GOHGNKHE@?$AAp?$AAa?$AAs?$AAs?$AA?5?$AA?$DN?$AA?$DN?$AA?5?$AAF?$AAO?$AAR?$AAM?$AAA?$AAT?$AA_?$AAO?$AAU?$AAT?$AAP?$AAU?$AAT?$AA_?$AAP?$AAA?$AAS?$AAS?$AA?$AA@ 0047c470     LIBCMTD:outputp.obj
 0003:0000b4b0       ??_C@_1IM@DNGHAPLB@?$AA_?$AAt?$AAv?$AAa?$AAl?$AAi?$AAd?$AAa?$AAt?$AAe?$AA_?$AAp?$AAa?$AAr?$AAa?$AAm?$AA_?$AAr?$AAe?$AAu?$AAs?$AAe?$AA?$CI?$AA?$CG?$AAp?$AAo?$AAs?$AA_?$AAv?$AAa?$AAl?$AAu@ 0047c4b0     LIBCMTD:outputp.obj
 0003:0000b558       ??_C@_1IG@HJIMKDHC@?$AA_?$AAt?$AAv?$AAa?$AAl?$AAi?$AAd?$AAa?$AAt?$AAe?$AA_?$AAp?$AAa?$AAr?$AAa?$AAm?$AA_?$AAr?$AAe?$AAu?$AAs?$AAe?$AA?$CI?$AA?$CG?$AAp?$AAo?$AAs?$AA_?$AAv?$AAa?$AAl?$AAu@ 0047c558     LIBCMTD:outputp.obj
 0003:0000b5f8       ??_C@_1IG@FDCPLALG@?$AA_?$AAt?$AAv?$AAa?$AAl?$AAi?$AAd?$AAa?$AAt?$AAe?$AA_?$AAp?$AAa?$AAr?$AAa?$AAm?$AA_?$AAr?$AAe?$AAu?$AAs?$AAe?$AA?$CI?$AA?$CG?$AAp?$AAo?$AAs?$AA_?$AAv?$AAa?$AAl?$AAu@ 0047c5f8     LIBCMTD:outputp.obj
 0003:0000b698       ??_C@_1IK@MHEDJAMK@?$AA_?$AAt?$AAv?$AAa?$AAl?$AAi?$AAd?$AAa?$AAt?$AAe?$AA_?$AAp?$AAa?$AAr?$AAa?$AAm?$AA_?$AAr?$AAe?$AAu?$AAs?$AAe?$AA?$CI?$AA?$CG?$AAp?$AAo?$AAs?$AA_?$AAv?$AAa?$AAl?$AAu@ 0047c698     LIBCMTD:outputp.obj
 0003:0000b740       ??_C@_1EM@BNPHBBIA@?$AA?$CI?$AA?$CI?$AAt?$AAy?$AAp?$AAe?$AA_?$AAp?$AAo?$AAs?$AA?$DO?$AA?$DN?$AA0?$AA?$CJ?$AA?5?$AA?$CG?$AA?$CG?$AA?5?$AA?$CI?$AAt?$AAy?$AAp?$AAe?$AA_?$AAp?$AAo?$AAs?$AA?$DM?$AA_?$AAA?$AAR?$AAG@ 0047c740     LIBCMTD:outputp.obj
 0003:0000b7a0       ??_C@_1IK@EIEPDKHJ@?$AA_?$AAt?$AAv?$AAa?$AAl?$AAi?$AAd?$AAa?$AAt?$AAe?$AA_?$AAp?$AAa?$AAr?$AAa?$AAm?$AA_?$AAr?$AAe?$AAu?$AAs?$AAe?$AA?$CI?$AA?$CG?$AAp?$AAo?$AAs?$AA_?$AAv?$AAa?$AAl?$AAu@ 0047c7a0     LIBCMTD:outputp.obj
 0003:0000b848       ??_C@_1JG@JBJBOCFB@?$AA?$CI?$AA?$CI?$AAp?$AAr?$AAe?$AAc?$AAi?$AAs?$AA_?$AAp?$AAo?$AAs?$AA?5?$AA?$DO?$AA?$DN?$AA?5?$AA0?$AA?$CJ?$AA?5?$AA?$CG?$AA?$CG?$AA?5?$AA?$CI?$AA?$CK?$AAe?$AAn?$AAd?$AA_?$AAp?$AAo?$AAs?$AA?5@ 0047c848     LIBCMTD:outputp.obj
 0003:0000b900       ??_C@_1II@PIPIMLPF@?$AA_?$AAt?$AAv?$AAa?$AAl?$AAi?$AAd?$AAa?$AAt?$AAe?$AA_?$AAp?$AAa?$AAr?$AAa?$AAm?$AA_?$AAr?$AAe?$AAu?$AAs?$AAe?$AA?$CI?$AA?$CG?$AAp?$AAo?$AAs?$AA_?$AAv?$AAa?$AAl?$AAu@ 0047c900     LIBCMTD:outputp.obj
 0003:0000b9a8       ??_C@_1JE@NMBHOLFI@?$AA?$CI?$AA?$CI?$AAw?$AAi?$AAd?$AAt?$AAh?$AA_?$AAp?$AAo?$AAs?$AA?5?$AA?$DO?$AA?$DN?$AA?5?$AA0?$AA?$CJ?$AA?5?$AA?$CG?$AA?$CG?$AA?5?$AA?$CI?$AA?$CK?$AAe?$AAn?$AAd?$AA_?$AAp?$AAo?$AAs?$AA?5?$AA?$DN@ 0047c9a8     LIBCMTD:outputp.obj
 0003:0000ba60       ??_C@_1EE@DMAIGNBG@?$AA?$CI?$AA?$CC?$AAI?$AAn?$AAc?$AAo?$AAr?$AAr?$AAe?$AAc?$AAt?$AA?5?$AAf?$AAo?$AAr?$AAm?$AAa?$AAt?$AA?5?$AAs?$AAp?$AAe?$AAc?$AAi?$AAf?$AAi?$AAe?$AAr?$AA?$CC?$AA?0?$AA?5?$AA0@ 0047ca60     LIBCMTD:outputp.obj
 0003:0000bab8       ??_C@_1JC@PFJNKEIO@?$AA?$CI?$AA?$CI?$AAt?$AAy?$AAp?$AAe?$AA_?$AAp?$AAo?$AAs?$AA?5?$AA?$DO?$AA?$DN?$AA?5?$AA0?$AA?$CJ?$AA?5?$AA?$CG?$AA?$CG?$AA?5?$AA?$CI?$AA?$CK?$AAe?$AAn?$AAd?$AA_?$AAp?$AAo?$AAs?$AA?5?$AA?$DN?$AA?$DN@ 0047cab8     LIBCMTD:outputp.obj
 0003:0000bb68       ??_C@_1BI@KANOLAMF@?$AA_?$AAo?$AAu?$AAt?$AAp?$AAu?$AAt?$AA_?$AAp?$AA_?$AAl?$AA?$AA@ 0047cb68     LIBCMTD:outputp.obj
 0003:0000bb88       ___lookuptable_s           0047cb88     LIBCMTD:outputs.obj
 0003:0000bbf4       ??_C@_1BI@COFBLHCG@?$AA_?$AAo?$AAu?$AAt?$AAp?$AAu?$AAt?$AA_?$AAs?$AA_?$AAl?$AA?$AA@ 0047cbf4     LIBCMTD:outputs.obj
 0003:0000bc10       ??_C@_1BK@ONMFGLDB@?$AA_?$AAw?$AAo?$AAu?$AAt?$AAp?$AAu?$AAt?$AA_?$AAs?$AA_?$AAl?$AA?$AA@ 0047cc10     LIBCMTD:woutputs.obj
 0003:0000bc30       ??_C@_1BK@GDEKGMNC@?$AA_?$AAw?$AAo?$AAu?$AAt?$AAp?$AAu?$AAt?$AA_?$AAp?$AA_?$AAl?$AA?$AA@ 0047cc30     LIBCMTD:woutputp.obj
 0003:0000bc50       ??_C@_1GA@GFFDGGFH@?$AAf?$AA?3?$AA?2?$AAd?$AAd?$AA?2?$AAv?$AAc?$AAt?$AAo?$AAo?$AAl?$AAs?$AA?2?$AAc?$AAr?$AAt?$AA_?$AAb?$AAl?$AAd?$AA?2?$AAs?$AAe?$AAl?$AAf?$AA_?$AAx?$AA8?$AA6?$AA?2?$AAc@ 0047cc50     LIBCMTD:mbtowc.obj
 0003:0000bcc8       ??_C@_1NC@EINCOKCO@?$AA_?$AAl?$AAo?$AAc?$AA_?$AAu?$AAp?$AAd?$AAa?$AAt?$AAe?$AA?4?$AAG?$AAe?$AAt?$AAL?$AAo?$AAc?$AAa?$AAl?$AAe?$AAT?$AA?$CI?$AA?$CJ?$AA?9?$AA?$DO?$AAl?$AAo?$AAc?$AAi?$AAn?$AAf@ 0047ccc8     LIBCMTD:mbtowc.obj
 0003:0000bdc4       ??_C@_1O@HJNPHHHB@?$AAf?$AAp?$AAu?$AAt?$AAw?$AAc?$AA?$AA@ 0047cdc4     LIBCMTD:fputwc.obj
 0003:0000bdd8       ??_C@_1GA@BJIGKGEA@?$AAf?$AA?3?$AA?2?$AAd?$AAd?$AA?2?$AAv?$AAc?$AAt?$AAo?$AAo?$AAl?$AAs?$AA?2?$AAc?$AAr?$AAt?$AA_?$AAb?$AAl?$AAd?$AA?2?$AAs?$AAe?$AAl?$AAf?$AA_?$AAx?$AA8?$AA6?$AA?2?$AAc@ 0047cdd8     LIBCMTD:fputwc.obj
 0003:0000be4c       ??_C@_1BM@JMKHIAHP@?$AA?$CI?$AAs?$AAt?$AAr?$AA?5?$AA?$CB?$AA?$DN?$AA?5?$AAN?$AAU?$AAL?$AAL?$AA?$CJ?$AA?$AA@ 0047ce4c     LIBCMTD:fputwc.obj
 0003:0000be70       ??_C@_1HG@KNCBMCDD@?$AAf?$AA?3?$AA?2?$AAd?$AAd?$AA?2?$AAv?$AAc?$AAt?$AAo?$AAo?$AAl?$AAs?$AA?2?$AAc?$AAr?$AAt?$AA_?$AAb?$AAl?$AAd?$AA?2?$AAs?$AAe?$AAl?$AAf?$AA_?$AAx?$AA8?$AA6?$AA?2?$AAc@ 0047ce70     LIBCMTD:typname.obj
 0003:0000bf00       ??_C@_1CK@GELGGBDK@?$AAp?$AAN?$AAo?$AAd?$AAe?$AA?9?$AA?$DO?$AA_?$AAN?$AAe?$AAx?$AAt?$AA?5?$AA?$CB?$AA?$DN?$AA?5?$AAN?$AAU?$AAL?$AAL?$AA?$AA@ 0047cf00     LIBCMTD:typname.obj
 0003:0000bf38       ??_C@_1JK@NAFNEPGC@?$AAs?$AAt?$AAr?$AAc?$AAp?$AAy?$AA_?$AAs?$AA?5?$AA?$CI?$AA?$CI?$AAc?$AAh?$AAa?$AAr?$AA?5?$AA?$CK?$AA?$CJ?$AA?$CI?$AA?$CI?$AAt?$AAy?$AAp?$AAe?$AA_?$AAi?$AAn?$AAf?$AAo?$AA?5?$AA?$CK?$AA?$CJ@ 0047cf38     LIBCMTD:typname.obj
 0003:0000bff0       ??_C@_1CM@OOICDMK@?$AAt?$AAy?$AAp?$AAe?$AA_?$AAi?$AAn?$AAf?$AAo?$AA?3?$AA?3?$AA_?$AAN?$AAa?$AAm?$AAe?$AA_?$AAb?$AAa?$AAs?$AAe?$AA?$AA@ 0047cff0     LIBCMTD:typname.obj
 0003:0000c028       ??_C@_1GI@EAJKJPED@?$AAs?$AAt?$AAr?$AAc?$AAp?$AAy?$AA_?$AAs?$AA?5?$AA?$CI?$AAp?$AAT?$AAm?$AAp?$AAT?$AAy?$AAp?$AAe?$AAN?$AAa?$AAm?$AAe?$AA?0?$AA?5?$AAl?$AAe?$AAn?$AA?$CL?$AA2?$AA?0?$AA?5?$AA?$CI@ 0047d028     LIBCMTD:typname.obj
 0003:0000c0a4       ??_C@_1DO@OJJLFJPE@?$AAt?$AAy?$AAp?$AAe?$AA_?$AAi?$AAn?$AAf?$AAo?$AA?3?$AA?3?$AA_?$AAN?$AAa?$AAm?$AAe?$AA_?$AAb?$AAa?$AAs?$AAe?$AA_?$AAi?$AAn?$AAt?$AAe?$AAr?$AAn?$AAa?$AAl?$AA?$AA@ 0047d0a4     LIBCMTD:typname.obj
 0003:0000c0f0       ??_C@_0DB@KIKNCIEC@f?3?2dd?2vctools?2crt_bld?2self_x86?2c@ 0047d0f0     LIBCMTD:osfinfo.obj
 0003:0000c12c       ??_C@_1BO@EMBOBGKE@?$AA_?$AAg?$AAe?$AAt?$AA_?$AAo?$AAs?$AAf?$AAh?$AAa?$AAn?$AAd?$AAl?$AAe?$AA?$AA@ 0047d12c     LIBCMTD:osfinfo.obj
 0003:0000c150       ??_C@_1GC@MLKLDJJG@?$AAf?$AA?3?$AA?2?$AAd?$AAd?$AA?2?$AAv?$AAc?$AAt?$AAo?$AAo?$AAl?$AAs?$AA?2?$AAc?$AAr?$AAt?$AA_?$AAb?$AAl?$AAd?$AA?2?$AAs?$AAe?$AAl?$AAf?$AA_?$AAx?$AA8?$AA6?$AA?2?$AAc@ 0047d150     LIBCMTD:osfinfo.obj
 0003:0000c1c8       ??_C@_0DB@OLNNDFNH@f?3?2dd?2vctools?2crt_bld?2self_x86?2c@ 0047d1c8     LIBCMTD:_sftbuf.obj
 0003:0000c208       ??_C@_1GC@DGAFOCMO@?$AAf?$AA?3?$AA?2?$AAd?$AAd?$AA?2?$AAv?$AAc?$AAt?$AAo?$AAo?$AAl?$AAs?$AA?2?$AAc?$AAr?$AAt?$AA_?$AAb?$AAl?$AAd?$AA?2?$AAs?$AAe?$AAl?$AAf?$AA_?$AAx?$AA8?$AA6?$AA?2?$AAc@ 0047d208     LIBCMTD:_sftbuf.obj
 0003:0000c280       ??_C@_1CO@KCKAACMI@?$AAf?$AAl?$AAa?$AAg?$AA?5?$AA?$DN?$AA?$DN?$AA?5?$AA0?$AA?5?$AA?$HM?$AA?$HM?$AA?5?$AAf?$AAl?$AAa?$AAg?$AA?5?$AA?$DN?$AA?$DN?$AA?5?$AA1?$AA?$AA@ 0047d280     LIBCMTD:_sftbuf.obj
 0003:0000c2b8       ??_C@_1BO@JGFPDJCP@?$AAv?$AAp?$AAr?$AAi?$AAn?$AAt?$AAf?$AA_?$AAh?$AAe?$AAl?$AAp?$AAe?$AAr?$AA?$AA@ 0047d2b8     LIBCMTD:vprintf.obj
 0003:0000c2e0       ??_C@_1GC@DHFFJKMC@?$AAf?$AA?3?$AA?2?$AAd?$AAd?$AA?2?$AAv?$AAc?$AAt?$AAo?$AAo?$AAl?$AAs?$AA?2?$AAc?$AAr?$AAt?$AA_?$AAb?$AAl?$AAd?$AA?2?$AAs?$AAe?$AAl?$AAf?$AA_?$AAx?$AA8?$AA6?$AA?2?$AAc@ 0047d2e0     LIBCMTD:vprintf.obj
 0003:0000c358       ??_C@_1BA@PCFLFGNC@?$AAw?$AAc?$AAs?$AAt?$AAo?$AAx?$AAl?$AA?$AA@ 0047d358     LIBCMTD:wcstol.obj
 0003:0000c370       ??_C@_1GA@CADFOND@?$AAf?$AA?3?$AA?2?$AAd?$AAd?$AA?2?$AAv?$AAc?$AAt?$AAo?$AAo?$AAl?$AAs?$AA?2?$AAc?$AAr?$AAt?$AA_?$AAb?$AAl?$AAd?$AA?2?$AAs?$AAe?$AAl?$AAf?$AA_?$AAx?$AA8?$AA6?$AA?2?$AAc@ 0047d370     LIBCMTD:wcstol.obj
 0003:0000c3e4       ??_C@_0BK@CFCOFLF@?5Complete?5Object?5Locator?8?$AA@ 0047d3e4     LIBCMTD:undname.obj
 0003:0000c404       ??_C@_0BN@MECKDCOJ@?5Class?5Hierarchy?5Descriptor?8?$AA@ 0047d404     LIBCMTD:undname.obj
 0003:0000c428       ??_C@_0BD@LGICGFMM@?5Base?5Class?5Array?8?$AA@ 0047d428     LIBCMTD:undname.obj
 0003:0000c440       ??_C@_0BM@LDKODKLH@?5Base?5Class?5Descriptor?5at?5?$CI?$AA@ 0047d440     LIBCMTD:undname.obj
 0003:0000c464       ??_C@_0BC@DAFEJGAK@?5Type?5Descriptor?8?$AA@ 0047d464     LIBCMTD:undname.obj
 0003:0000c47c       ??_C@_0BM@PMGGMLDN@?$GAlocal?5static?5thread?5guard?8?$AA@ 0047d47c     LIBCMTD:undname.obj
 0003:0000c4a0       ??_C@_0CL@FGIJHLCE@?$GAmanaged?5vector?5copy?5constructor@ 0047d4a0     LIBCMTD:undname.obj
 0003:0000c4d4       ??_C@_0CJ@GJELGAMM@?$GAvector?5vbase?5copy?5constructor?5i@ 0047d4d4     LIBCMTD:undname.obj
 0003:0000c508       ??_C@_0CD@CGAJBKEJ@?$GAvector?5copy?5constructor?5iterato@ 0047d508     LIBCMTD:undname.obj
 0003:0000c534       ??_C@_0CB@PDBIFEP@?$GAdynamic?5atexit?5destructor?5for?5?8@ 0047d534     LIBCMTD:undname.obj
 0003:0000c55c       ??_C@_0BL@CLIPGLGB@?$GAdynamic?5initializer?5for?5?8?$AA@ 0047d55c     LIBCMTD:undname.obj
 0003:0000c57c       ??_C@_0CM@FCBBDIGB@?$GAeh?5vector?5vbase?5copy?5constructo@ 0047d57c     LIBCMTD:undname.obj
 0003:0000c5b0       ??_C@_0CG@HLDDJMAG@?$GAeh?5vector?5copy?5constructor?5iter@ 0047d5b0     LIBCMTD:undname.obj
 0003:0000c5e0       ??_C@_0CF@IMGKMJNO@?$GAmanaged?5vector?5destructor?5itera@ 0047d5e0     LIBCMTD:undname.obj
 0003:0000c60c       ??_C@_0CG@CFDHKGGD@?$GAmanaged?5vector?5constructor?5iter@ 0047d60c     LIBCMTD:undname.obj
 0003:0000c63c       ??_C@_0BN@CKNJLHMB@?$GAplacement?5delete?$FL?$FN?5closure?8?$AA@ 0047d63c     LIBCMTD:undname.obj
 0003:0000c660       ??_C@_0BL@CNOONJFP@?$GAplacement?5delete?5closure?8?$AA@ 0047d660     LIBCMTD:undname.obj
 0003:0000c680       ??_C@_0P@HJKNJFNN@?$GAomni?5callsig?8?$AA@ 0047d680     LIBCMTD:undname.obj
 0003:0000c694       ??_C@_09LBNFPBCA@?5delete?$FL?$FN?$AA@ 0047d694     LIBCMTD:undname.obj
 0003:0000c6a0       ??_C@_06FHBGPFGH@?5new?$FL?$FN?$AA@ 0047d6a0     LIBCMTD:undname.obj
 0003:0000c6a8       ??_C@_0CE@IIHCMGGL@?$GAlocal?5vftable?5constructor?5closu@ 0047d6a8     LIBCMTD:undname.obj
 0003:0000c6d4       ??_C@_0BA@KKLDJDLB@?$GAlocal?5vftable?8?$AA@ 0047d6d4     LIBCMTD:undname.obj
 0003:0000c6e8       ??_C@_05KHLCHHI@?$GARTTI?$AA@ 0047d6e8     LIBCMTD:undname.obj
 0003:0000c6f0       ??_C@_03KLGMFNMG@?$GAEH?$AA@ 0047d6f0     LIBCMTD:undname.obj
 0003:0000c6f4       ??_C@_0BA@KBCDOMBN@?$GAudt?5returning?8?$AA@ 0047d6f4     LIBCMTD:undname.obj
 0003:0000c708       ??_C@_0BL@LLKPOHJI@?$GAcopy?5constructor?5closure?8?$AA@ 0047d708     LIBCMTD:undname.obj
 0003:0000c728       ??_C@_0CH@OOJPLCPH@?$GAeh?5vector?5vbase?5constructor?5ite@ 0047d728     LIBCMTD:undname.obj
 0003:0000c758       ??_C@_0CA@GCEOPDGL@?$GAeh?5vector?5destructor?5iterator?8?$AA@ 0047d758     LIBCMTD:undname.obj
 0003:0000c780       ??_C@_0CB@JONCMFFK@?$GAeh?5vector?5constructor?5iterator?8@ 0047d780     LIBCMTD:undname.obj
 0003:0000c7a8       ??_C@_0BL@NILFHHPC@?$GAvirtual?5displacement?5map?8?$AA@ 0047d7a8     LIBCMTD:undname.obj
 0003:0000c7c8       ??_C@_0CE@IKBNEHA@?$GAvector?5vbase?5constructor?5iterat@ 0047d7c8     LIBCMTD:undname.obj
 0003:0000c7f4       ??_C@_0BN@LFPFMEDL@?$GAvector?5destructor?5iterator?8?$AA@ 0047d7f4     LIBCMTD:undname.obj
 0003:0000c818       ??_C@_0BO@PFGOCPJJ@?$GAvector?5constructor?5iterator?8?$AA@ 0047d818     LIBCMTD:undname.obj
 0003:0000c83c       ??_C@_0BN@IMDCHIKM@?$GAscalar?5deleting?5destructor?8?$AA@ 0047d83c     LIBCMTD:undname.obj
 0003:0000c860       ??_C@_0BO@OBMKPJIG@?$GAdefault?5constructor?5closure?8?$AA@ 0047d860     LIBCMTD:undname.obj
 0003:0000c884       ??_C@_0BN@DEGPLNFK@?$GAvector?5deleting?5destructor?8?$AA@ 0047d884     LIBCMTD:undname.obj
 0003:0000c8a8       ??_C@_0BD@JDLKDPAB@?$GAvbase?5destructor?8?$AA@ 0047d8a8     LIBCMTD:undname.obj
 0003:0000c8c0       ??_C@_08OBABFOLI@?$GAstring?8?$AA@ 0047d8c0     LIBCMTD:undname.obj
 0003:0000c8cc       ??_C@_0BF@KDPPACIK@?$GAlocal?5static?5guard?8?$AA@ 0047d8cc     LIBCMTD:undname.obj
 0003:0000c8e8       ??_C@_08LLFFHHDJ@?$GAtypeof?8?$AA@ 0047d8e8     LIBCMTD:undname.obj
 0003:0000c8f4       ??_C@_07FEEIOKP@?$GAvcall?8?$AA@ 0047d8f4     LIBCMTD:undname.obj
 0003:0000c900       ??_C@_09BLBHBJP@?$GAvbtable?8?$AA@ 0047d900     LIBCMTD:undname.obj
 0003:0000c90c       ??_C@_09IFPLHPGF@?$GAvftable?8?$AA@ 0047d90c     LIBCMTD:undname.obj
 0003:0000c918       ??_C@_02MHEGNOJ@?$FO?$DN?$AA@ 0047d918     LIBCMTD:undname.obj
 0003:0000c91c       ??_C@_02DHLNPPGH@?$HM?$DN?$AA@ 0047d91c     LIBCMTD:undname.obj
 0003:0000c920       ??_C@_02FGJGFEAB@?$CG?$DN?$AA@ 0047d920     LIBCMTD:undname.obj
 0003:0000c924       ??_C@_03CDNPDDLA@?$DM?$DM?$DN?$AA@ 0047d924     LIBCMTD:undname.obj
 0003:0000c928       ??_C@_03IKFCCPFF@?$DO?$DO?$DN?$AA@ 0047d928     LIBCMTD:undname.obj
 0003:0000c92c       ??_C@_02FENAOKFI@?$CF?$DN?$AA@ 0047d92c     LIBCMTD:undname.obj
 0003:0000c930       ??_C@_02FJEHGPIO@?1?$DN?$AA@ 0047d930     LIBCMTD:undname.obj
 0003:0000c934       ??_C@_02FKMDLLOA@?9?$DN?$AA@ 0047d934     LIBCMTD:undname.obj
 0003:0000c938       ??_C@_02FOEOMHFC@?$CL?$DN?$AA@ 0047d938     LIBCMTD:undname.obj
 0003:0000c93c       ??_C@_02FPIMKNGF@?$CK?$DN?$AA@ 0047d93c     LIBCMTD:undname.obj
 0003:0000c940       ??_C@_02NONPIBCD@?$HM?$HM?$AA@ 0047d940     LIBCMTD:undname.obj
 0003:0000c944       ??_C@_02PPKAJPJL@?$CG?$CG?$AA@ 0047d944     LIBCMTD:undname.obj
 0003:0000c948       ??_C@_01DNKMNLPK@?$HM?$AA@ 0047d948     LIBCMTD:undname.obj
 0003:0000c94c       ??_C@_01JKBOJNNK@?$FO?$AA@ 0047d94c     LIBCMTD:undname.obj
 0003:0000c950       ??_C@_01PJKLJHI@?$HO?$AA@  0047d950     LIBCMTD:undname.obj
 0003:0000c954       ??_C@_02HCKGKOFO@?$CI?$CJ?$AA@ 0047d954     LIBCMTD:undname.obj
 0003:0000c958       ??_C@_01IHBHIGKO@?0?$AA@   0047d958     LIBCMTD:undname.obj
 0003:0000c95c       ??_C@_02EEKDKGMJ@?$DO?$DN?$AA@ 0047d95c     LIBCMTD:undname.obj
 0003:0000c960       ??_C@_01PPODPGHN@?$DO?$AA@ 0047d960     LIBCMTD:undname.obj
 0003:0000c964       ??_C@_02EHCHHCKH@?$DM?$DN?$AA@ 0047d964     LIBCMTD:undname.obj
 0003:0000c968       ??_C@_01MNNFJEPP@?$DM?$AA@ 0047d968     LIBCMTD:undname.obj
 0003:0000c96c       ??_C@_01FGNFDNOH@?$CF?$AA@ 0047d96c     LIBCMTD:undname.obj
 0003:0000c970       ??_C@_01KMDKNFGN@?1?$AA@   0047d970     LIBCMTD:undname.obj
 0003:0000c974       ??_C@_03MNHNFDLC@?9?$DO?$CK?$AA@ 0047d974     LIBCMTD:undname.obj
 0003:0000c978       ??_C@_01HNPIGOCE@?$CG?$AA@ 0047d978     LIBCMTD:undname.obj
 0003:0000c97c       ??_C@_01MIFGBAGJ@?$CL?$AA@ 0047d97c     LIBCMTD:undname.obj
 0003:0000c980       ??_C@_01JOAMLHOP@?9?$AA@   0047d980     LIBCMTD:undname.obj
 0003:0000c984       ??_C@_02BAABKJLB@?9?9?$AA@ 0047d984     LIBCMTD:undname.obj
 0003:0000c988       ??_C@_02ECNGHCIF@?$CL?$CL?$AA@ 0047d988     LIBCMTD:undname.obj
 0003:0000c98c       ??_C@_01NBENCBCI@?$CK?$AA@ 0047d98c     LIBCMTD:undname.obj
 0003:0000c990       ??_C@_02HBOOOICD@?9?$DO?$AA@ 0047d990     LIBCMTD:undname.obj
 0003:0000c994       ??_C@_08LHJFAFGD@operator?$AA@ 0047d994     LIBCMTD:undname.obj
 0003:0000c9a0       ??_C@_02GPECMEKF@?$FL?$FN?$AA@ 0047d9a0     LIBCMTD:undname.obj
 0003:0000c9a4       ??_C@_02FDNJECIE@?$CB?$DN?$AA@ 0047d9a4     LIBCMTD:undname.obj
 0003:0000c9a8       ??_C@_02EGOFBIJA@?$DN?$DN?$AA@ 0047d9a8     LIBCMTD:undname.obj
 0003:0000c9ac       ??_C@_01DCLJPIOD@?$CB?$AA@ 0047d9ac     LIBCMTD:undname.obj
 0003:0000c9b0       ??_C@_02FODMEDOG@?$DM?$DM?$AA@ 0047d9b0     LIBCMTD:undname.obj
 0003:0000c9b4       ??_C@_02GPIOPFAK@?$DO?$DO?$AA@ 0047d9b4     LIBCMTD:undname.obj
 0003:0000c9b8       ??_C@_07FPCDHGMM@?5delete?$AA@ 0047d9b8     LIBCMTD:undname.obj
 0003:0000c9c4       ??_C@_04NIHEBCM@?5new?$AA@ 0047d9c4     LIBCMTD:undname.obj
 0003:0000c9cc       ??_C@_0M@GFIIJFMG@__unaligned?$AA@ 0047d9cc     LIBCMTD:undname.obj
 0003:0000c9dc       ??_C@_0L@PILCLIHE@__restrict?$AA@ 0047d9dc     LIBCMTD:undname.obj
 0003:0000c9ec       ??_C@_07JOMMBBKO@__ptr64?$AA@ 0047d9ec     LIBCMTD:undname.obj
 0003:0000c9f8       ??_C@_06GHPCKEAG@__eabi?$AA@ 0047d9f8     LIBCMTD:undname.obj
 0003:0000ca00       ??_C@_09HIJEGCPM@__clrcall?$AA@ 0047da00     LIBCMTD:undname.obj
 0003:0000ca0c       ??_C@_0L@JMKHOMEK@__fastcall?$AA@ 0047da0c     LIBCMTD:undname.obj
 0003:0000ca1c       ??_C@_0L@NPHFGOKO@__thiscall?$AA@ 0047da1c     LIBCMTD:undname.obj
 0003:0000ca2c       ??_C@_09IFJBGAPI@__stdcall?$AA@ 0047da2c     LIBCMTD:undname.obj
 0003:0000ca38       ??_C@_08GHMPAG@__pascal?$AA@ 0047da38     LIBCMTD:undname.obj
 0003:0000ca44       ??_C@_07KOLFKCDI@__cdecl?$AA@ 0047da44     LIBCMTD:undname.obj
 0003:0000ca50       ??_C@_08EHJDFFNH@__based?$CI?$AA@ 0047da50     LIBCMTD:undname.obj
 0003:0000cc34       ??_C@_04HEJADOOB@CV?3?5?$AA@ 0047dc34     LIBCMTD:undname.obj
 0003:0000cc3c       ??_C@_02MOLJINC@?3?3?$AA@  0047dc3c     LIBCMTD:undname.obj
 0003:0000cc40       ??_C@_01GEODFPGF@?8?$AA@   0047dc40     LIBCMTD:undname.obj
 0003:0000cc44       ??_C@_01NLNLIGKH@?$GA?$AA@ 0047dc44     LIBCMTD:undname.obj
 0003:0000cc48       ??_C@_0O@KHGCOMHP@generic?9type?9?$AA@ 0047dc48     LIBCMTD:undname.obj
 0003:0000cc58       ??_C@_0BE@JAEOCHPE@template?9parameter?9?$AA@ 0047dc58     LIBCMTD:undname.obj
 0003:0000cc70       ??_C@_02OHHJMEON@?8?8?$AA@ 0047dc70     LIBCMTD:undname.obj
 0003:0000cc74       ??_C@_0BG@JNJLAMPM@?$GAanonymous?5namespace?8?$AA@ 0047dc74     LIBCMTD:undname.obj
 0003:0000cc90       ??_C@_0BN@IBLMMFAP@?$GAnon?9type?9template?9parameter?$AA@ 0047dc90     LIBCMTD:undname.obj
 0003:0000ccb4       ??_C@_0BE@EODMJLIF@?$GAtemplate?9parameter?$AA@ 0047dcb4     LIBCMTD:undname.obj
 0003:0000cccc       ??_C@_04GKJNKENE@void?$AA@ 0047dccc     LIBCMTD:undname.obj
 0003:0000ccd4       ??_C@_04HIBGFPH@NULL?$AA@  0047dcd4     LIBCMTD:undname.obj
 0003:0000ccdc       ??_C@_0M@DHNBOJMP@extern?5?$CCC?$CC?5?$AA@ 0047dcdc     LIBCMTD:undname.obj
 0003:0000ccec       ??_C@_08KJLFOPNE@?$FLthunk?$FN?3?$AA@ 0047dcec     LIBCMTD:undname.obj
 0003:0000ccf8       ??_C@_08GPDDCMKI@public?3?5?$AA@ 0047dcf8     LIBCMTD:undname.obj
 0003:0000cd04       ??_C@_0M@GAIFPFIP@protected?3?5?$AA@ 0047dd04     LIBCMTD:undname.obj
 0003:0000cd14       ??_C@_09LAPHOOG@private?3?5?$AA@ 0047dd14     LIBCMTD:undname.obj
 0003:0000cd20       ??_C@_08NIEOINHE@virtual?5?$AA@ 0047dd20     LIBCMTD:undname.obj
 0003:0000cd2c       ??_C@_07PGOEDBHP@static?5?$AA@ 0047dd2c     LIBCMTD:undname.obj
 0003:0000cd38       ??_C@_0DA@HGFJFBBE@?$GAtemplate?5static?5data?5member?5des@ 0047dd38     LIBCMTD:undname.obj
 0003:0000cd74       ??_C@_0DB@ILEFOCIJ@?$GAtemplate?5static?5data?5member?5con@ 0047dd74     LIBCMTD:undname.obj
 0003:0000cdb0       ??_C@_0CB@KJDOOODE@?$GAlocal?5static?5destructor?5helper?8@ 0047ddb0     LIBCMTD:undname.obj
 0003:0000cdd8       ??_C@_0L@HNGCOGAE@?$GAadjustor?$HL?$AA@ 0047ddd8     LIBCMTD:undname.obj
 0003:0000cde8       ??_C@_0L@GHPFDFH@?$GAvtordisp?$HL?$AA@ 0047dde8     LIBCMTD:undname.obj
 0003:0000cdf8       ??_C@_0N@CBHHHENL@?$GAvtordispex?$HL?$AA@ 0047ddf8     LIBCMTD:undname.obj
 0003:0000ce08       ??_C@_01CLKCMJKC@?5?$AA@   0047de08     LIBCMTD:undname.obj
 0003:0000ce0c       ??_C@_02IGFCGPIL@?$HN?8?$AA@ 0047de0c     LIBCMTD:undname.obj
 0003:0000ce10       ??_C@_03OPGICMGF@?$HN?8?5?$AA@ 0047de10     LIBCMTD:undname.obj
 0003:0000ce14       ??_C@_02KCKGHPCA@?$CJ?5?$AA@ 0047de14     LIBCMTD:undname.obj
 0003:0000ce18       ??_C@_05BEFAKPML@void?5?$AA@ 0047de18     LIBCMTD:undname.obj
 0003:0000ce20       ??_C@_0P@GCOCNKDM@std?3?3nullptr_t?$AA@ 0047de20     LIBCMTD:undname.obj
 0003:0000ce34       ??_C@_08PABEKFH@volatile?$AA@ 0047de34     LIBCMTD:undname.obj
 0003:0000ce40       ??_C@_0M@ELJOJFFH@?0?$DMellipsis?$DO?$AA@ 0047de40     LIBCMTD:undname.obj
 0003:0000ce50       ??_C@_04EENFHACM@?0?4?4?4?$AA@ 0047de50     LIBCMTD:undname.obj
 0003:0000ce58       ??_C@_0L@EGPHHEKN@?$DMellipsis?$DO?$AA@ 0047de58     LIBCMTD:undname.obj
 0003:0000ce68       ??_C@_07HDJPLPEK@?5throw?$CI?$AA@ 0047de68     LIBCMTD:undname.obj
 0003:0000ce74       ??_C@_09EFNPDFFP@?5volatile?$AA@ 0047de74     LIBCMTD:undname.obj
 0003:0000ce80       ??_C@_05BNCCCJPP@const?$AA@ 0047de80     LIBCMTD:undname.obj
 0003:0000ce88       ??_C@_07EDHNAJHC@signed?5?$AA@ 0047de88     LIBCMTD:undname.obj
 0003:0000ce94       ??_C@_09EBBEKKIH@unsigned?5?$AA@ 0047de94     LIBCMTD:undname.obj
 0003:0000cea0       ??_C@_07NFANNNEC@UNKNOWN?$AA@ 0047dea0     LIBCMTD:undname.obj
 0003:0000ceac       ??_C@_06GCICPBLB@__w64?5?$AA@ 0047deac     LIBCMTD:undname.obj
 0003:0000ceb4       ??_C@_07CLGGIAMF@wchar_t?$AA@ 0047deb4     LIBCMTD:undname.obj
 0003:0000cec0       ??_C@_09EEKGDCPH@?$DMunknown?$DO?$AA@ 0047dec0     LIBCMTD:undname.obj
 0003:0000cecc       ??_C@_08GAHOLHEO@__int128?$AA@ 0047decc     LIBCMTD:undname.obj
 0003:0000ced8       ??_C@_07LFCOJCAC@__int64?$AA@ 0047ded8     LIBCMTD:undname.obj
 0003:0000cee4       ??_C@_07OFLPPHGP@__int32?$AA@ 0047dee4     LIBCMTD:undname.obj
 0003:0000cef0       ??_C@_07ICFHOGAF@__int16?$AA@ 0047def0     LIBCMTD:undname.obj
 0003:0000cefc       ??_C@_06EBGKOKIG@__int8?$AA@ 0047defc     LIBCMTD:undname.obj
 0003:0000cf04       ??_C@_04DDKJGDCM@bool?$AA@ 0047df04     LIBCMTD:undname.obj
 0003:0000cf0c       ??_C@_06BNJCAIGJ@double?$AA@ 0047df0c     LIBCMTD:undname.obj
 0003:0000cf14       ??_C@_05CJIMAING@long?5?$AA@ 0047df14     LIBCMTD:undname.obj
 0003:0000cf1c       ??_C@_05KNFBNCOH@float?$AA@ 0047df1c     LIBCMTD:undname.obj
 0003:0000cf24       ??_C@_04GOKPGOLB@long?$AA@ 0047df24     LIBCMTD:undname.obj
 0003:0000cf2c       ??_C@_03JBIPMCLC@int?$AA@  0047df2c     LIBCMTD:undname.obj
 0003:0000cf30       ??_C@_05BFKKPKCG@short?$AA@ 0047df30     LIBCMTD:undname.obj
 0003:0000cf38       ??_C@_04ENMBGAPA@char?$AA@ 0047df38     LIBCMTD:undname.obj
 0003:0000cf40       ??_C@_05LJGMCFOG@enum?5?$AA@ 0047df40     LIBCMTD:undname.obj
 0003:0000cf48       ??_C@_0N@DLIEFKNA@cointerface?5?$AA@ 0047df48     LIBCMTD:undname.obj
 0003:0000cf58       ??_C@_08KOFANOFK@coclass?5?$AA@ 0047df58     LIBCMTD:undname.obj
 0003:0000cf64       ??_C@_06LJBABKPM@class?5?$AA@ 0047df64     LIBCMTD:undname.obj
 0003:0000cf6c       ??_C@_07DIBCDNGL@struct?5?$AA@ 0047df6c     LIBCMTD:undname.obj
 0003:0000cf78       ??_C@_06MOJHIBMG@union?5?$AA@ 0047df78     LIBCMTD:undname.obj
 0003:0000cf80       ??_C@_0P@GCIFDJCJ@?$GAunknown?5ecsu?8?$AA@ 0047df80     LIBCMTD:undname.obj
 0003:0000cf94       ??_C@_04LAHKHJMA@int?5?$AA@ 0047df94     LIBCMTD:undname.obj
 0003:0000cf9c       ??_C@_06EHJMALKF@short?5?$AA@ 0047df9c     LIBCMTD:undname.obj
 0003:0000cfa4       ??_C@_05CIHEBHNO@char?5?$AA@ 0047dfa4     LIBCMTD:undname.obj
 0003:0000cfac       ??_C@_06LIJLOJAG@const?5?$AA@ 0047dfac     LIBCMTD:undname.obj
 0003:0000cfb4       ??_C@_09GAIEOBLP@volatile?5?$AA@ 0047dfb4     LIBCMTD:undname.obj
 0003:0000cfc0       ??_C@_0O@GKABPPIF@cli?3?3pin_ptr?$DM?$AA@ 0047dfc0     LIBCMTD:undname.obj
 0003:0000cfd0       ??_C@_0M@EALIELKG@cli?3?3array?$DM?$AA@ 0047dfd0     LIBCMTD:undname.obj
 0003:0000cfe0       ??_C@_02GOGNNPBN@?$CJ?$FL?$AA@ 0047dfe0     LIBCMTD:undname.obj
 0003:0000cfe4       ??_C@_06EEGAIFAK@?$HLflat?$HN?$AA@ 0047dfe4     LIBCMTD:undname.obj
 0003:0000cfec       ??_C@_02MDINNEEG@s?5?$AA@  0047dfec     LIBCMTD:undname.obj
 0003:0000cff0       ??_C@_05JIBOFOHK@?$HLfor?5?$AA@ 0047dff0     LIBCMTD:undname.obj
 0003:0000cff8       ??_7DNameNode@@6B@         0047dff8     LIBCMTD:undname.obj
 0003:0000d008       ??_7charNode@@6B@          0047e008     LIBCMTD:undname.obj
 0003:0000d018       ??_7pcharNode@@6B@         0047e018     LIBCMTD:undname.obj
 0003:0000d028       ??_7pDNameNode@@6B@        0047e028     LIBCMTD:undname.obj
 0003:0000d038       ??_7DNameStatusNode@@6B@   0047e038     LIBCMTD:undname.obj
 0003:0000d048       ??_C@_04OKOHEJBO@?5?$DP?$DP?5?$AA@ 0047e048     LIBCMTD:undname.obj
 0003:0000d050       ??_7pairNode@@6B@          0047e050     LIBCMTD:undname.obj
 0003:0000d060       ??_C@_1BA@BALFACEM@?$AAC?$AAO?$AAN?$AAO?$AAU?$AAT?$AA$?$AA?$AA@ 0047e060     LIBCMTD:initcon.obj
 0003:0000d074       ??_C@_1O@EGMJNCOI@?$AAf?$AAc?$AAl?$AAo?$AAs?$AAe?$AA?$AA@ 0047e074     LIBCMTD:fclose.obj
 0003:0000d088       ??_C@_1GA@KMIDAPAP@?$AAf?$AA?3?$AA?2?$AAd?$AAd?$AA?2?$AAv?$AAc?$AAt?$AAo?$AAo?$AAl?$AAs?$AA?2?$AAc?$AAr?$AAt?$AA_?$AAb?$AAl?$AAd?$AA?2?$AAs?$AAe?$AAl?$AAf?$AA_?$AAx?$AA8?$AA6?$AA?2?$AAc@ 0047e088     LIBCMTD:fclose.obj
 0003:0000d0fc       ??_C@_1BO@JINCABEC@?$AA_?$AAf?$AAc?$AAl?$AAo?$AAs?$AAe?$AA_?$AAn?$AAo?$AAl?$AAo?$AAc?$AAk?$AA?$AA@ 0047e0fc     LIBCMTD:fclose.obj
 0003:0000d120       ??_C@_1DG@LNNHNFHJ@?$AA?$CI?$AA_?$AAo?$AAs?$AAf?$AAi?$AAl?$AAe?$AA?$CI?$AAf?$AAi?$AAl?$AAe?$AAd?$AAe?$AAs?$AA?$CJ?$AA?5?$AA?$CG?$AA?5?$AAF?$AAO?$AAP?$AAE?$AAN?$AA?$CJ?$AA?$AA@ 0047e120     LIBCMTD:commit.obj
 0003:0000d160       ??_C@_1BA@FLNMBBIM@?$AA_?$AAc?$AAo?$AAm?$AAm?$AAi?$AAt?$AA?$AA@ 0047e160     LIBCMTD:commit.obj
 0003:0000d178       ??_C@_1GA@BOPCOCFN@?$AAf?$AA?3?$AA?2?$AAd?$AAd?$AA?2?$AAv?$AAc?$AAt?$AAo?$AAo?$AAl?$AAs?$AA?2?$AAc?$AAr?$AAt?$AA_?$AAb?$AAl?$AAd?$AA?2?$AAs?$AAe?$AAl?$AAf?$AA_?$AAx?$AA8?$AA6?$AA?2?$AAc@ 0047e178     LIBCMTD:commit.obj
 0003:0000d1f0       ??_C@_1HC@KFLBHHBC@?$AA?$CI?$AAf?$AAi?$AAl?$AAe?$AAd?$AAe?$AAs?$AA?5?$AA?$DO?$AA?$DN?$AA?5?$AA0?$AA?5?$AA?$CG?$AA?$CG?$AA?5?$AA?$CI?$AAu?$AAn?$AAs?$AAi?$AAg?$AAn?$AAe?$AAd?$AA?$CJ?$AAf?$AAi?$AAl?$AAe?$AAd@ 0047e1f0     LIBCMTD:commit.obj
 0003:0000d278       ??_C@_1O@EDEJGJBM@?$AA_?$AAc?$AAl?$AAo?$AAs?$AAe?$AA?$AA@ 0047e278     LIBCMTD:close.obj
 0003:0000d288       ??_C@_1FO@NNGNFGFH@?$AAf?$AA?3?$AA?2?$AAd?$AAd?$AA?2?$AAv?$AAc?$AAt?$AAo?$AAo?$AAl?$AAs?$AA?2?$AAc?$AAr?$AAt?$AA_?$AAb?$AAl?$AAd?$AA?2?$AAs?$AAe?$AAl?$AAf?$AA_?$AAx?$AA8?$AA6?$AA?2?$AAc@ 0047e288     LIBCMTD:close.obj
 0003:0000d2f8       ??_C@_1GE@MIMBMOF@?$AAf?$AA?3?$AA?2?$AAd?$AAd?$AA?2?$AAv?$AAc?$AAt?$AAo?$AAo?$AAl?$AAs?$AA?2?$AAc?$AAr?$AAt?$AA_?$AAb?$AAl?$AAd?$AA?2?$AAs?$AAe?$AAl?$AAf?$AA_?$AAx?$AA8?$AA6?$AA?2?$AAc@ 0047e2f8     LIBCMTD:_freebuf.obj
 0003:0000d370       ??_C@_1BO@KIJENGPH@?$AAs?$AAt?$AAr?$AAe?$AAa?$AAm?$AA?5?$AA?$CB?$AA?$DN?$AA?5?$AAN?$AAU?$AAL?$AAL?$AA?$AA@ 0047e370     LIBCMTD:_freebuf.obj
 0003:0000d8d4       ??_R4bad_exception@std@@6B@ 0047e8d4     LIBCMTD:frame.obj
 0003:0000d8ec       ??_R3bad_exception@std@@8  0047e8ec     LIBCMTD:frame.obj
 0003:0000d900       ??_R2bad_exception@std@@8  0047e900     LIBCMTD:frame.obj
 0003:0000d90c       ??_R1A@?0A@EA@bad_exception@std@@8 0047e90c     LIBCMTD:frame.obj
 0003:0000d930       ??_R1A@?0A@EA@exception@std@@8 0047e930     LIBCMTD:frame.obj
 0003:0000d954       ??_R3exception@std@@8      0047e954     LIBCMTD:frame.obj
 0003:0000d968       ??_R2exception@std@@8      0047e968     LIBCMTD:frame.obj
 0003:0000d970       ??_R4type_info@@6B@        0047e970     LIBCMTD:typinfo.obj
 0003:0000d988       ??_R3type_info@@8          0047e988     LIBCMTD:typinfo.obj
 0003:0000d99c       ??_R2type_info@@8          0047e99c     LIBCMTD:typinfo.obj
 0003:0000d9a4       ??_R1A@?0A@EA@type_info@@8 0047e9a4     LIBCMTD:typinfo.obj
 0003:0000d9c8       ??_R4exception@std@@6B@    0047e9c8     LIBCMTD:stdexcpt.obj
 0003:0000d9e0       ??_R4bad_cast@std@@6B@     0047e9e0     LIBCMTD:stdexcpt.obj
 0003:0000d9f8       ??_R3bad_cast@std@@8       0047e9f8     LIBCMTD:stdexcpt.obj
 0003:0000da0c       ??_R2bad_cast@std@@8       0047ea0c     LIBCMTD:stdexcpt.obj
 0003:0000da18       ??_R1A@?0A@EA@bad_cast@std@@8 0047ea18     LIBCMTD:stdexcpt.obj
 0003:0000da3c       ??_R4bad_typeid@std@@6B@   0047ea3c     LIBCMTD:stdexcpt.obj
 0003:0000da54       ??_R3bad_typeid@std@@8     0047ea54     LIBCMTD:stdexcpt.obj
 0003:0000da68       ??_R2bad_typeid@std@@8     0047ea68     LIBCMTD:stdexcpt.obj
 0003:0000da74       ??_R1A@?0A@EA@bad_typeid@std@@8 0047ea74     LIBCMTD:stdexcpt.obj
 0003:0000da98       ??_R4__non_rtti_object@std@@6B@ 0047ea98     LIBCMTD:stdexcpt.obj
 0003:0000dab0       ??_R3__non_rtti_object@std@@8 0047eab0     LIBCMTD:stdexcpt.obj
 0003:0000dac4       ??_R2__non_rtti_object@std@@8 0047eac4     LIBCMTD:stdexcpt.obj
 0003:0000dad4       ??_R1A@?0A@EA@__non_rtti_object@std@@8 0047ead4     LIBCMTD:stdexcpt.obj
 0003:0000dc04       ___rtc_iaa                 0047ec04     LIBCMTD:_initsect_.obj
 0003:0000de0c       ___rtc_izz                 0047ee0c     LIBCMTD:_initsect_.obj
 0003:0000df10       ___rtc_taa                 0047ef10     LIBCMTD:_initsect_.obj
 0003:0000e118       ___rtc_tzz                 0047f118     LIBCMTD:_initsect_.obj
 0003:0000e7fc       __TI2?AVbad_exception@std@@ 0047f7fc     LIBCMTD:frame.obj
 0003:0000e810       __CTA2?AVbad_exception@std@@ 0047f810     LIBCMTD:frame.obj
 0003:0000e820       __CT??_R0?AVbad_exception@std@@@8??0bad_exception@std@@QAE@ABV01@@Z12 0047f820     LIBCMTD:frame.obj
 0003:0000e840       __CT??_R0?AVexception@std@@@8??0exception@std@@QAE@ABV01@@Z12 0047f840     LIBCMTD:frame.obj
 0004:00000000       ___security_cookie         00480000     LIBCMTD:gs_cookie.obj
 0004:00000004       ___security_cookie_complement 00480004     LIBCMTD:gs_cookie.obj
 0004:00000008       ___app_type                00480008     LIBCMTD:wincrt0.obj
 0004:0000000c       ?_RTC_ErrorLevels@@3PAHA   0048000c     LIBCMTD:_error_.obj
 0004:00000028       ___badioinfo               00480028     LIBCMTD:ioinit.obj
 0004:00000074       __crtDbgFlag               00480074     LIBCMTD:dbgheap.obj
 0004:00000078       ___crtDebugFillThreshold   00480078     LIBCMTD:dbgheap.obj
 0004:00000080       __crtBreakAlloc            00480080     LIBCMTD:dbgheap.obj
 0004:0000008c       ___flsindex                0048008c     LIBCMTD:tidtable.obj
 0004:00000090       ___getvalueindex           00480090     LIBCMTD:tidtable.obj
 0004:000000a0       ___clocalestr              004800a0     LIBCMTD:nlsdata2.obj
 0004:000000a8       ___lc_time_c               004800a8     LIBCMTD:nlsdata2.obj
 0004:00000258       ___initiallocinfo          00480258     LIBCMTD:nlsdata2.obj
 0004:0000035c       ___ptlocinfo               0048035c     LIBCMTD:nlsdata2.obj
 0004:00000360       ___initiallocalestructinfo 00480360     LIBCMTD:nlsdata2.obj
 0004:00000530       ___initialmbcinfo          00480530     LIBCMTD:mbctype.obj
 0004:00000750       __mbctype                  00480750     LIBCMTD:mbctype.obj
 0004:00000858       __mbcasemap                00480858     LIBCMTD:mbctype.obj
 0004:00000958       ___ptmbcinfo               00480958     LIBCMTD:mbctype.obj
 0004:00000b58       ___globallocalestatus      00480b58     LIBCMTD:glstatus.obj
 0004:00000b60       __pfnAllocHook             00480b60     LIBCMTD:dbghook.obj
 0004:00000b64       __cfltcvt_tab              00480b64     LIBCMTD:cmiscdat.obj
 0004:00000d00       __crtAssertBusy            00480d00     LIBCMTD:dbgrptt.obj
 0004:00000d04       __CrtDbgMode               00480d04     LIBCMTD:dbgrptt.obj
 0004:00000d10       __CrtDbgFile               00480d10     LIBCMTD:dbgrptt.obj
 0004:00000d30       __pctype                   00480d30     LIBCMTD:ctype.obj
 0004:00000d34       __pwctype                  00480d34     LIBCMTD:ctype.obj
 0004:00000d40       ___lconv_static_decimal    00480d40     LIBCMTD:lconv.obj
 0004:00000d44       ___lconv_static_W_decimal  00480d44     LIBCMTD:lconv.obj
 0004:00000d48       ___lconv_c                 00480d48     LIBCMTD:lconv.obj
 0004:00000d98       ___lconv                   00480d98     LIBCMTD:lconv.obj
 0004:00000db0       ___mb_cur_max              00480db0     LIBCMTD:nlsdata1.obj
 0004:00000db4       ___decimal_point           00480db4     LIBCMTD:nlsdata1.obj
 0004:00000db8       ___decimal_point_length    00480db8     LIBCMTD:nlsdata1.obj
 0004:00000dc0       ??_R0?AVbad_exception@std@@@8 00480dc0     LIBCMTD:frame.obj
 0004:00000de8       ??_R0?AVexception@std@@@8  00480de8     LIBCMTD:frame.obj
 0004:00000e10       ___abort_behavior          00480e10     LIBCMTD:abort.obj
 0004:00000e14       ___nullstring              00480e14     LIBCMTD:output.obj
 0004:00000e18       ___wnullstring             00480e18     LIBCMTD:output.obj
 0004:00000e20       __NLG_Destination          00480e20     LIBCMTD:exsup.obj
 0004:00000e34       ??_R0?AVtype_info@@@8      00480e34     LIBCMTD:typinfo.obj
 0004:00000e50       ??_R0?AVbad_cast@std@@@8   00480e50     LIBCMTD:stdexcpt.obj
 0004:00000e70       ??_R0?AVbad_typeid@std@@@8 00480e70     LIBCMTD:stdexcpt.obj
 0004:00000e94       ??_R0?AV__non_rtti_object@std@@@8 00480e94     LIBCMTD:stdexcpt.obj
 0004:00000ec0       __iob                      00480ec0     LIBCMTD:_file.obj
 0004:000011c0       __confh                    004811c0     LIBCMTD:initcon.obj
 0004:00001304       __aenvptr                  00481304     LIBCMTD:wincrt0.obj
 0004:00001308       __wenvptr                  00481308     LIBCMTD:wincrt0.obj
 0004:0000130c       ___error_mode              0048130c     LIBCMTD:wincrt0.obj
 0004:00001314       ?wsprintffp@@3P6AHPADPBDZZA 00481314     LIBCMTD:_error_.obj
 0004:000016ec       __umaskval                 004816ec     LIBCMTD:crt0dat.obj
 0004:000016f0       ___argc                    004816f0     LIBCMTD:crt0dat.obj
 0004:000016f4       ___argv                    004816f4     LIBCMTD:crt0dat.obj
 0004:000016f8       ___wargv                   004816f8     LIBCMTD:crt0dat.obj
 0004:000016fc       __environ                  004816fc     LIBCMTD:crt0dat.obj
 0004:00001700       ___initenv                 00481700     LIBCMTD:crt0dat.obj
 0004:00001704       __wenviron                 00481704     LIBCMTD:crt0dat.obj
 0004:00001708       ___winitenv                00481708     LIBCMTD:crt0dat.obj
 0004:0000170c       __pgmptr                   0048170c     LIBCMTD:crt0dat.obj
 0004:00001710       __wpgmptr                  00481710     LIBCMTD:crt0dat.obj
 0004:00001714       __exitflag                 00481714     LIBCMTD:crt0dat.obj
 0004:00001718       __C_Termination_Done       00481718     LIBCMTD:crt0dat.obj
 0004:0000171c       __C_Exit_Done              0048171c     LIBCMTD:crt0dat.obj
 0004:00001880       ?_pfnDumpClient@@3P6AXPAXI@ZA 00481880     LIBCMTD:dbgheap.obj
 0004:00001888       ___crtDebugCheckCount      00481888     LIBCMTD:dbgheap.obj
 0004:00001898       _gpFlsAlloc                00481898     LIBCMTD:tidtable.obj
 0004:0000189c       _gpFlsGetValue             0048189c     LIBCMTD:tidtable.obj
 0004:000018a0       _gpFlsSetValue             004818a0     LIBCMTD:tidtable.obj
 0004:000018a4       _gpFlsFree                 004818a4     LIBCMTD:tidtable.obj
 0004:000018ac       __crtheap                  004818ac     LIBCMTD:heapinit.obj
 0004:0000201c       ___locale_changed          0048201c     LIBCMTD:setlocal.obj
 0004:00002020       ___pInvalidArgHandler      00482020     LIBCMTD:invarg.obj
 0004:00002028       ___mbulinfo                00482028     LIBCMTD:mbctype.obj
 0004:00002034       ___mbcodepage              00482034     LIBCMTD:mbctype.obj
 0004:00002038       ___ismbcodepage            00482038     LIBCMTD:mbctype.obj
 0004:0000203c       ___mblcid                  0048203c     LIBCMTD:mbctype.obj
 0004:00002048       ?__pInconsistency@@3P6AXXZA 00482048     LIBCMTD:hooks.obj
 0004:0000221c       ___pPurecall               0048221c     LIBCMTD:inithelp.obj
 0004:00002220       ?_pnhHeap@@3P6AHI@ZA       00482220     LIBCMTD:handler.obj
 0004:00002224       __newmode                  00482224     LIBCMTD:_newmode.obj
 0004:00002258       ___lconv_static_null       00482258     LIBCMTD:lconv.obj
 0004:0000225c       ___lconv_static_W_null     0048225c     LIBCMTD:lconv.obj
 0004:00002260       __cflush                   00482260     LIBCMTD:_file.obj
 0004:00002274       __stdbuf                   00482274     LIBCMTD:_sftbuf.obj
 0004:00002294       ?pArgList@UnDecorator@@0PAVReplicator@@A 00482294     LIBCMTD:undname.obj
 0004:00002298       ?pZNameList@UnDecorator@@0PAVReplicator@@A 00482298     LIBCMTD:undname.obj
 0004:0000229c       ?pTemplateArgList@UnDecorator@@0PAVReplicator@@A 0048229c     LIBCMTD:undname.obj
 0004:000022a0       ?gName@UnDecorator@@0PBDB  004822a0     LIBCMTD:undname.obj
 0004:000022a4       ?name@UnDecorator@@0PBDB   004822a4     LIBCMTD:undname.obj
 0004:00002368       ___piob                    00482368     <common>
 0004:000026c0       __bufin                    004826c0     <common>
 0004:000036c0       __nstream                  004836c0     <common>
 0004:000036c4       ___sse2_available          004836c4     <common>
 0004:000036d0       __pfnReportHook            004836d0     <common>
 0004:000036e0       __pReportHookListW         004836e0     <common>
 0004:000036e4       __pReportHookList          004836e4     <common>
 0004:000036e8       __debugger_hook_dummy      004836e8     <common>
 0004:000036f4       ___setlc_active            004836f4     <common>
 0004:00003704       ___unguarded_readlc_active 00483704     <common>
 0004:00003708       __nhandle                  00483708     <common>
 0004:00003760       ___pioinfo                 00483760     <common>
 0004:00003860       ___env_initialized         00483860     <common>
 0004:00003870       ___onexitend               00483870     <common>
 0004:00003874       ___onexitbegin             00483874     <common>
 0004:00003878       ___mbctype_initialized     00483878     <common>
 0004:0000387c       __FPinit                   0048387c     <common>
 0004:00003880       ___dyn_tls_init_callback   00483880     <common>
 0004:00003884       __acmdln                   00483884     <common>
 0004:00003894       __NoHeapEnableTerminationOnCorruption 00483894     <common>
 0005:00000000       __IMPORT_DESCRIPTOR_KERNEL32 00484000     kernel32:KERNEL32.dll
 0005:00000014       __IMPORT_DESCRIPTOR_USER32 00484014     user32:USER32.dll
 0005:00000028       __IMPORT_DESCRIPTOR_VMProtectSDK32 00484028     VMProtectSDK32:VMProtectSDK32.dll
 0005:0000003c       __NULL_IMPORT_DESCRIPTOR   0048403c     kernel32:KERNEL32.dll
 0005:00000288       __imp__GetModuleHandleA@4  00484288     kernel32:KERNEL32.dll
 0005:0000028c       __imp__CloseHandle@4       0048428c     kernel32:KERNEL32.dll
 0005:00000290       __imp__CreateFileW@28      00484290     kernel32:KERNEL32.dll
 0005:00000294       __imp__SetStdHandle@8      00484294     kernel32:KERNEL32.dll
 0005:00000298       __imp__GetConsoleMode@8    00484298     kernel32:KERNEL32.dll
 0005:0000029c       __imp__GetConsoleCP@0      0048429c     kernel32:KERNEL32.dll
 0005:000002a0       __imp__SetFilePointer@16   004842a0     kernel32:KERNEL32.dll
 0005:000002a4       __imp__IsProcessorFeaturePresent@4 004842a4     kernel32:KERNEL32.dll
 0005:000002a8       __imp__LCMapStringW@24     004842a8     kernel32:KERNEL32.dll
 0005:000002ac       __imp__GetUserDefaultLCID@0 004842ac     kernel32:KERNEL32.dll
 0005:000002b0       __imp__EnumSystemLocalesA@8 004842b0     kernel32:KERNEL32.dll
 0005:000002b4       __imp__IsValidLocale@8     004842b4     kernel32:KERNEL32.dll
 0005:000002b8       __imp__GetCommandLineA@0   004842b8     kernel32:KERNEL32.dll
 0005:000002bc       __imp__HeapSetInformation@16 004842bc     kernel32:KERNEL32.dll
 0005:000002c0       __imp__GetStartupInfoW@4   004842c0     kernel32:KERNEL32.dll
 0005:000002c4       __imp__WideCharToMultiByte@32 004842c4     kernel32:KERNEL32.dll
 0005:000002c8       __imp__IsDebuggerPresent@0 004842c8     kernel32:KERNEL32.dll
 0005:000002cc       __imp__MultiByteToWideChar@24 004842cc     kernel32:KERNEL32.dll
 0005:000002d0       __imp__RaiseException@16   004842d0     kernel32:KERNEL32.dll
 0005:000002d4       __imp__lstrlenA@4          004842d4     kernel32:KERNEL32.dll
 0005:000002d8       __imp__GetProcAddress@8    004842d8     kernel32:KERNEL32.dll
 0005:000002dc       __imp__LoadLibraryW@4      004842dc     kernel32:KERNEL32.dll
 0005:000002e0       __imp__TerminateProcess@8  004842e0     kernel32:KERNEL32.dll
 0005:000002e4       __imp__GetCurrentProcess@0 004842e4     kernel32:KERNEL32.dll
 0005:000002e8       __imp__UnhandledExceptionFilter@4 004842e8     kernel32:KERNEL32.dll
 0005:000002ec       __imp__SetUnhandledExceptionFilter@4 004842ec     kernel32:KERNEL32.dll
 0005:000002f0       __imp__QueryPerformanceCounter@4 004842f0     kernel32:KERNEL32.dll
 0005:000002f4       __imp__GetTickCount@0      004842f4     kernel32:KERNEL32.dll
 0005:000002f8       __imp__GetCurrentThreadId@0 004842f8     kernel32:KERNEL32.dll
 0005:000002fc       __imp__GetCurrentProcessId@0 004842fc     kernel32:KERNEL32.dll
 0005:00000300       __imp__GetSystemTimeAsFileTime@4 00484300     kernel32:KERNEL32.dll
 0005:00000304       __imp__InterlockedIncrement@4 00484304     kernel32:KERNEL32.dll
 0005:00000308       __imp__InterlockedDecrement@4 00484308     kernel32:KERNEL32.dll
 0005:0000030c       __imp__DecodePointer@4     0048430c     kernel32:KERNEL32.dll
 0005:00000310       __imp__GetModuleHandleW@4  00484310     kernel32:KERNEL32.dll
 0005:00000314       __imp__ExitProcess@4       00484314     kernel32:KERNEL32.dll
 0005:00000318       __imp__GetModuleFileNameA@12 00484318     kernel32:KERNEL32.dll
 0005:0000031c       __imp__FreeEnvironmentStringsW@4 0048431c     kernel32:KERNEL32.dll
 0005:00000320       __imp__GetEnvironmentStringsW@0 00484320     kernel32:KERNEL32.dll
 0005:00000324       __imp__SetHandleCount@4    00484324     kernel32:KERNEL32.dll
 0005:00000328       __imp__GetStdHandle@4      00484328     kernel32:KERNEL32.dll
 0005:0000032c       __imp__InitializeCriticalSectionAndSpinCount@8 0048432c     kernel32:KERNEL32.dll
 0005:00000330       __imp__GetFileType@4       00484330     kernel32:KERNEL32.dll
 0005:00000334       __imp__DeleteCriticalSection@4 00484334     kernel32:KERNEL32.dll
 0005:00000338       __imp__HeapValidate@12     00484338     kernel32:KERNEL32.dll
 0005:0000033c       __imp__IsBadReadPtr@8      0048433c     kernel32:KERNEL32.dll
 0005:00000340       __imp__EncodePointer@4     00484340     kernel32:KERNEL32.dll
 0005:00000344       __imp__TlsAlloc@0          00484344     kernel32:KERNEL32.dll
 0005:00000348       __imp__TlsGetValue@4       00484348     kernel32:KERNEL32.dll
 0005:0000034c       __imp__TlsSetValue@8       0048434c     kernel32:KERNEL32.dll
 0005:00000350       __imp__TlsFree@4           00484350     kernel32:KERNEL32.dll
 0005:00000354       __imp__SetLastError@4      00484354     kernel32:KERNEL32.dll
 0005:00000358       __imp__GetLastError@0      00484358     kernel32:KERNEL32.dll
 0005:0000035c       __imp__GetCurrentThread@0  0048435c     kernel32:KERNEL32.dll
 0005:00000360       __imp__HeapCreate@12       00484360     kernel32:KERNEL32.dll
 0005:00000364       __imp__HeapDestroy@4       00484364     kernel32:KERNEL32.dll
 0005:00000368       __imp__GetModuleFileNameW@12 00484368     kernel32:KERNEL32.dll
 0005:0000036c       __imp__WriteFile@20        0048436c     kernel32:KERNEL32.dll
 0005:00000370       __imp__HeapFree@12         00484370     kernel32:KERNEL32.dll
 0005:00000374       __imp__HeapAlloc@12        00484374     kernel32:KERNEL32.dll
 0005:00000378       __imp__GetProcessHeap@0    00484378     kernel32:KERNEL32.dll
 0005:0000037c       __imp__VirtualQuery@12     0048437c     kernel32:KERNEL32.dll
 0005:00000380       __imp__FreeLibrary@4       00484380     kernel32:KERNEL32.dll
 0005:00000384       __imp__RtlUnwind@16        00484384     kernel32:KERNEL32.dll
 0005:00000388       __imp__GetACP@0            00484388     kernel32:KERNEL32.dll
 0005:0000038c       __imp__GetOEMCP@0          0048438c     kernel32:KERNEL32.dll
 0005:00000390       __imp__GetCPInfo@8         00484390     kernel32:KERNEL32.dll
 0005:00000394       __imp__IsValidCodePage@4   00484394     kernel32:KERNEL32.dll
 0005:00000398       __imp__EnterCriticalSection@4 00484398     kernel32:KERNEL32.dll
 0005:0000039c       __imp__LeaveCriticalSection@4 0048439c     kernel32:KERNEL32.dll
 0005:000003a0       __imp__FatalAppExitA@8     004843a0     kernel32:KERNEL32.dll
 0005:000003a4       __imp__SetConsoleCtrlHandler@8 004843a4     kernel32:KERNEL32.dll
 0005:000003a8       __imp__InterlockedExchange@8 004843a8     kernel32:KERNEL32.dll
 0005:000003ac       __imp__GetLocaleInfoW@16   004843ac     kernel32:KERNEL32.dll
 0005:000003b0       __imp__HeapReAlloc@16      004843b0     kernel32:KERNEL32.dll
 0005:000003b4       __imp__HeapSize@12         004843b4     kernel32:KERNEL32.dll
 0005:000003b8       __imp__HeapQueryInformation@20 004843b8     kernel32:KERNEL32.dll
 0005:000003bc       __imp__OutputDebugStringA@4 004843bc     kernel32:KERNEL32.dll
 0005:000003c0       __imp__WriteConsoleW@20    004843c0     kernel32:KERNEL32.dll
 0005:000003c4       __imp__OutputDebugStringW@4 004843c4     kernel32:KERNEL32.dll
 0005:000003c8       __imp__GetStringTypeW@16   004843c8     kernel32:KERNEL32.dll
 0005:000003cc       __imp__GetLocaleInfoA@16   004843cc     kernel32:KERNEL32.dll
 0005:000003d0       __imp__FlushFileBuffers@4  004843d0     kernel32:KERNEL32.dll
 0005:000003d4       \177KERNEL32_NULL_THUNK_DATA 004843d4     kernel32:KERNEL32.dll
 0005:00000440       __imp__DialogBoxParamA@20  00484440     user32:USER32.dll
 0005:00000444       __imp__SetFocus@4          00484444     user32:USER32.dll
 0005:00000448       __imp__GetDlgItem@8        00484448     user32:USER32.dll
 0005:0000044c       __imp__EndDialog@8         0048444c     user32:USER32.dll
 0005:00000450       __imp__GetDlgItemTextA@16  00484450     user32:USER32.dll
 0005:00000454       __imp__MessageBoxA@16      00484454     user32:USER32.dll
 0005:00000458       \177USER32_NULL_THUNK_DATA 00484458     user32:USER32.dll
 0005:00000488       __imp__VMProtectDecryptStringA@4 00484488     VMProtectSDK32:VMProtectSDK32.dll
 0005:0000048c       __imp__VMProtectBegin@4    0048448c     VMProtectSDK32:VMProtectSDK32.dll
 0005:00000490       __imp__VMProtectEnd@0      00484490     VMProtectSDK32:VMProtectSDK32.dll
 0005:00000494       \177VMProtectSDK32_NULL_THUNK_DATA 00484494     VMProtectSDK32:VMProtectSDK32.dll

 entry point at        0002:00000ca3

 Static symbols

 0004:000022a8       ?outputString@UnDecorator@@0PADA 004822a8     LIBCMTD:undname.obj
 0004:000022ac       ?maxStringLength@UnDecorator@@0HA 004822ac     LIBCMTD:undname.obj
 0004:000022b0       ?disableFlags@UnDecorator@@0KA 004822b0     LIBCMTD:undname.obj
 0004:000022b4       ?m_pGetParameter@UnDecorator@@0P6APADJ@ZA 004822b4     LIBCMTD:undname.obj
 0004:000022b8       ?fExplicitTemplateParams@UnDecorator@@0_NA 004822b8     LIBCMTD:undname.obj
 0004:000022b9       ?fGetTemplateArgumentList@UnDecorator@@0_NA 004822b9     LIBCMTD:undname.obj
 0004:00002328       ?nodes@?1??make@DNameStatusNode@@SAPAV2@W4DNameStatus@@@Z@4PAV2@A 00482328     LIBCMTD:undname.obj
 0004:00002364       ??_B?1??make@DNameStatusNode@@SAPAV1@W4DNameStatus@@@Z@51 00482364     LIBCMTD:undname.obj
